:020000040800F2
:1000000000000220A90300083D8000084980000884
:10001000518000085980000861800008000000003D
:1000200000000000000000000000000075800008D3
:100030006980000800000000818000082188000815
:10004000F9030008F9030008F9030008F9030008A0
:10005000F9030008F9030008F9030008F903000890
:10006000F9030008F9030008F9030008F903000880
:10007000F9030008F9030008F9030008F903000870
:10008000F9030008F9030008F9030008F903000860
:10009000F9030008F9030008F9030008F903000850
:1000A000F9030008F9030008F9030008F903000840
:1000B000F90300088D800008A1800008F9030008FA
:1000C000F9030008F9030008F9030008F903000820
:1000D000F9030008659C0008F9030008F90300080B
:1000E000F9030008F9030008F9030008F903000800
:1000F000F9030008F9030008F9030008F9030008F0
:10010000F9030008F9030008F9030008F9030008DF
:10011000F9030008F9030008F9030008F9030008CF
:10012000C5800008F9030008F9030008AD80000845
:10013000F9030008F9030008F9030008F9030008AF
:10014000F9030008F9030008F9030008F90300089F
:10015000F9030008F9030008F9030008F90300088F
:10016000F9030008F9030008F9030008F90300087F
:10017000F9030008F9030008F90300080000000073
:10018000F9030008F9030008F9030008F90300085F
:10019000F9030008F9030008F9030008F90300084F
:1001A000F9030008F9030008F903000880B58EB0D0
:1001B00000AF40F6D803C2F200034BF6BA22CCF6E9
:1001C000DE221A6044F6D843C2F200034BF6BA228C
:1001D000CCF6DE221A6040F6D803C2F200033B637D
:1001E00044F6DC43C2F20003FB623B6BBB6207E0F8
:1001F000BB6A4FF000021A60BB6A03F10403BB62E2
:10020000FA6ABB6A9A42F3D840F6D803C2F20003F6
:100210001B68002B06D144F6D843C2F200031B68CA
:10022000002B00D0FEE740F20003C2F200034BF6C1
:10023000BA22CCF6DE221A6040F6D403C2F20003E2
:100240004BF6BA22CCF6DE221A6043F64C03C0F617
:1002500002037B6240F20003C2F200033B6240F6FD
:10026000D803C2F20003FB613B6ABB610BE07B6A0F
:100270001A68BB691A60BB6903F10403BB617B6A3E
:1002800003F104037B62FA69BB699A42EFD840F23A
:100290000003C2F200031A6845F27863C1F2342306
:1002A0009A420BD140F6D403C2F200031A6840F61A
:1002B000D403C2F200031B689A4200D0FEE70DF09F
:1002C00047FC07F104023B461046194607F0F0FDD3
:1002D00040F20042C0F6000240F20043C0F60003C4
:1002E000D31A4FEAA3037B614FF000033B610BE09D
:1002F00040F20043C0F600033A6953F822309847B1
:100300003B6903F101033B617A693B699A42EFDC87
:1003100040F20042C0F6000240F20043C0F6000383
:10032000D31A4FEAA3037B614FF000033B610BE05C
:1003300040F20043C0F600033A6953F82230984770
:100340003B6903F101033B617A693B699A42EFDC47
:100350007A683B681046194609F090FC03467B63B7
:1003600040F20042C0F6000240F20043C0F6000333
:10037000D31A4FEAA303FB60FB68BB600DE0BB68C8
:1003800003F1FF3240F20043C0F6000353F822307D
:100390009847BB6803F1FF33BB60BB68002BEEDC02
:1003A000786B07F0E1FD00BF80B500AFFFF7FEFE00
:1003B00080B400AFFEE700BF80B400AFFEE700BF2F
:1003C00080B400AFFEE700BF80B400AFFEE700BF1F
:1003D00080B400AFFEE700BF80B400AFFEE700BF0F
:1003E00080B400AFFEE700BF80B400AFFEE700BFFF
:1003F00080B400AFFEE700BF80B400AFFEE700BFEF
:1004000080B487B000AFF860B9601346FB804FF04E
:1004100000037B61FB6893F83930DBB27B617B6959
:10042000012B02D07B69122B54D1BB68002B02D068
:10043000FB88002B02D14FF001034DE0FB6893F8DD
:100440003830012B02D14FF0020345E0FB684FF03A
:10045000010283F83820FB68BA689A62FB68FA8860
:100460009A85FB68FA88DA85FB684FF0000283F80A
:100470003A20FB6893F83930DBB2122B05D1FB68C8
:100480004FF0320283F8392004E0FB684FF022027B
:1004900083F83920FB681B68FA681268D26842F456
:1004A0008072DA60FB681B68FA681268526942F071
:1004B00001025A61FB684FF0000283F83820FB68A4
:1004C0001B68FA681268D26842F02002DA604FF0C6
:1004D000000301E04FF00203184607F11C07BD4678
:1004E00080BC704780B584B000AF78604FF00003E7
:1004F000FB604FF00003BB607B681B681B6803F068
:100500000103FB607B681B68DB6803F48073BB60DE
:10051000FB68002B14D0BB68002B11D07B681B68D4
:100520007A681268126822F001021A607B6893F8F8
:100530003A30DBB243F00103DAB27B6883F83A2049
:100540007B681B681B6803F00203002B0CBF0023B1
:100550000123FB607B681B685B6903F00103BB60E0
:10056000FB68002B14D0BB68002B11D07B681B6884
:100570007A681268126822F002021A607B6893F8A7
:100580003A30DBB243F00403DAB27B6883F83A20F6
:100590007B681B681B6803F00403002B0CBF00235F
:1005A0000123FB607B681B685B6903F00103BB6090
:1005B000FB68002B14D0BB68002B11D07B681B6834
:1005C0007A681268126822F004021A607B6893F855
:1005D0003A30DBB243F00203DAB27B6883F83A20A8
:1005E0007B681B681B6803F00803002B0CBF00230B
:1005F0000123FB607B681B685B6903F00103BB6040
:10060000FB68002B14D0BB68002B11D07B681B68E3
:100610007A681268126822F008021A607B6893F800
:100620003A30DBB243F00803DAB27B6883F83A2051
:100630007B681B681B6803F02003002B0CBF0023A2
:100640000123FB607B681B68DB6803F02003BB6051
:10065000FB68002B0DD0BB68002B0AD0786800F037
:10066000F5F87B681B687A681268126822F020022D
:100670001A607B681B681B6803F04003002B0CBFEB
:1006800000230123FB607B681B68DB6803F04003E9
:10069000BB60FB68002B0DD0BB68002B0AD07868CC
:1006A00000F038F87B681B687A681268126822F0DC
:1006B00040021A607B6893F83A30DBB2002B07D017
:1006C0007B684FF0010283F83920786800F018F851
:1006D00007F11007BD4680BD80B483B000AF7860DD
:1006E00007F10C07BD4680BC704700BF80B483B0E3
:1006F00000AF786007F10C07BD4680BC704700BFB3
:1007000080B483B000AF786007F10C07BD4680BCB1
:10071000704700BF80B584B000AF78604FF0000331
:10072000FB607B6893F83930DBB2FB60FB68122B0F
:1007300003D0FB68322B40F081807B6893F838301F
:10074000012B02D14FF002037AE07B684FF00102E7
:1007500083F838207B689B68B3F5805F1DD17B6888
:100760001B6ABB607B681A68BB681B884FEAC3536F
:100770004FEAD35353607B681B69002B06D17B681B
:100780001B6A03F102027B681A6210E07B681B6A35
:1007900003F101027B681A6209E07B681A687B68D2
:1007A0001B6A1978516003F101027B681A627B6849
:1007B000DB8C03F1FF339AB27B68DA847B68DB8CD5
:1007C000002B33D17B681B687A681268D26822F0EC
:1007D0004002DA607B6893F83930DBB2322B05D106
:1007E0007B684FF0220283F8392014E07B681B6895
:1007F0007A681268D26822F48072DA607B681B68BB
:100800007A681268526922F001025A617B684FF0DF
:10081000010283F839207B684FF0000283F838200A
:100820007868FFF759FF4FF0000309E07B684FF04D
:10083000000283F838204FF0000301E04FF002037C
:10084000184607F11007BD4680BD00BF80B584B0D3
:1008500000AF78604FF00003FB607B6893F839309D
:10086000DBB2FB60FB68222B03D0FB68322B40F02D
:10087000A7807B6893F83830012B02D14FF0020338
:10088000A0E07B684FF0010283F838207B689B680A
:10089000B3F5805F27D17B689B6ABB607B681B696F
:1008A000002B11D17B681B685B689BB24FEAC35376
:1008B0004FEAD3539AB2BB681A807B689B6A03F1F4
:1008C00002027B689A622CE07B681B685B689BB2C3
:1008D000DBB29AB2BB681A807B689B6A03F10102A3
:1008E0007B689A621DE07B681B69002B0BD17B68DB
:1008F0009B6A7A6812685268D2B21A7003F10102D8
:100900007B689A620DE07B689B6A7A68126852681D
:10091000D2B202F07F02D2B21A7003F101027B68F8
:100920009A627B68DB8D03F1FF339AB27B68DA85CC
:100930007B68DB8D002B3BD100BF7B681B681B688D
:1009400003F02003002BF8D17B681B687A681268DB
:10095000D26822F02002DA607B6893F83930DBB28B
:10096000322B05D17B684FF0120283F8392014E056
:100970007B681B687A681268D26822F48072DA6039
:100980007B681B687A681268526922F001025A611A
:100990007B684FF0010283F839207B684FF000023A
:1009A00083F838207868FFF7A1FE4FF0000309E0D4
:1009B0007B684FF0000283F838204FF0000301E01D
:1009C0004FF00203184607F11007BD4680BD00BF77
:1009D00080B483B000AF786007F10C07BD4680BCDF
:1009E000704700BF80B483B000AF786007F10C0798
:1009F000BD4680BC704700BF80B582B000AF786054
:100A00007B68002B02D14FF00103C4E07B681A68B9
:100A10004FF00003C4F201039A426CD07B681B685C
:100A2000B3F1804F67D07B681A684FF48063C4F2DB
:100A300000039A425FD07B681A684FF40063C4F2E7
:100A400000039A4257D07B681A684FF44063C4F29F
:100A500000039A424FD07B681A684FF48053C4F267
:100A600000039A4247D07B681A684FF4A053C4F23F
:100A700000039A423FD07B681A684FF48063C4F247
:100A800001039A4237D07B681A684FF48043C4F25E
:100A900001039A422FD07B681A684FF48843C4F24E
:100AA00001039A4227D07B681A684FF49043C4F23E
:100AB00001039A421FD07B681A684FF4C053C4F2F6
:100AC00000039A4217D07B681A684FF4E053C4F2CF
:100AD00000039A420FD07B681A684FF40053C4F2A7
:100AE00000039A4207D046F2DC00C0F601004FF046
:100AF000D10107F0D1F97B689B68002B17D07B6888
:100B00009B68102B13D07B689B68202B0FD07B68D1
:100B10009B68402B0BD07B689B68602B07D046F20C
:100B2000DC00C0F601004FF0D20107F0B5F97B6898
:100B30001B69002B11D07B681B69B3F5807F0CD03B
:100B40007B681B69B3F5007F07D046F2DC00C0F676
:100B500001004FF0D30107F09FF97B6893F839301B
:100B6000DBB2002B02D1786800F01AF87B684FF0F6
:100B7000020283F839207B681A687B6803F104035A
:100B80001046194600F00AFA7B684FF0010283F81C
:100B900039204FF00003184607F10807BD4680BD15
:100BA00080B483B000AF786007F10C07BD4680BC0D
:100BB000704700BF80B582B000AF78607B681A686C
:100BC0004FF00003C4F201039A426CD07B681B68AB
:100BD000B3F1804F67D07B681A684FF48063C4F22A
:100BE00000039A425FD07B681A684FF40063C4F236
:100BF00000039A4257D07B681A684FF44063C4F2EE
:100C000000039A424FD07B681A684FF48053C4F2B5
:100C100000039A4247D07B681A684FF4A053C4F28D
:100C200000039A423FD07B681A684FF48063C4F295
:100C300001039A4237D07B681A684FF48043C4F2AC
:100C400001039A422FD07B681A684FF48843C4F29C
:100C500001039A4227D07B681A684FF49043C4F28C
:100C600001039A421FD07B681A684FF4C053C4F244
:100C700000039A4217D07B681A684FF4E053C4F21D
:100C800000039A420FD07B681A684FF40053C4F2F5
:100C900000039A4207D046F2DC00C0F6010040F2A1
:100CA0005B1107F0F9F87B681B687A681268D268F4
:100CB00042F00102DA607B681B687A681268126889
:100CC00042F001021A604FF00003184607F10807CE
:100CD000BD4680BD80B582B000AF78607B681B6880
:100CE0001B6903F00203002B27D07B681B68DB68BD
:100CF00003F00203002B20D07B681B687A6812681F
:100D0000126922F002021A617B684FF001021A7622
:100D10007B681B689B6903F00303002B03D0786892
:100D200000F01EF905E0786800F010F9786800F02E
:100D300021F97B684FF000021A767B681B681B69FB
:100D400003F00403002B27D07B681B68DB6803F0EB
:100D50000403002B20D07B681B687A681268126934
:100D600022F004021A617B684FF002021A767B6857
:100D70001B689B6903F44073002B03D0786800F074
:100D8000EFF805E0786800F0E1F8786800F0F2F834
:100D90007B684FF000021A767B681B681B6903F0C2
:100DA0000803002B27D07B681B68DB6803F008036F
:100DB000002B20D07B681B687A681268126922F0C9
:100DC00008021A617B684FF004021A767B681B6880
:100DD0009B6903F00303002B03D0786800F0C0F890
:100DE00005E0786800F0B2F8786800F0C3F87B6836
:100DF0004FF000021A767B681B681B6903F0100332
:100E0000002B27D07B681B68DB6803F01003002BE6
:100E100020D07B681B687A681268126922F0100281
:100E20001A617B684FF008021A767B681B689B6921
:100E300003F44073002B03D0786800F091F805E0CC
:100E4000786800F083F8786800F094F87B684FF0D9
:100E500000021A767B681B681B6903F00103DBB292
:100E6000002B12D07B681B68DB6803F00103DBB248
:100E7000002B0AD07B681B687A681268126922F01E
:100E800001021A6178680BF0C3F87B681B681B6964
:100E900003F08003002B11D07B681B68DB6803F034
:100EA0008003002B0AD07B681B687A68126812697D
:100EB00022F080021A617868FFF794FD7B681B6856
:100EC0001B6903F04003002B11D07B681B68DB68B3
:100ED00003F04003002B0AD07B681B687A68126815
:100EE000126922F040021A61786800F04DF87B68C0
:100EF0001B681B6903F02003002B11D07B681B6863
:100F0000DB6803F02003002B0AD07B681B687A683B
:100F10001268126922F020021A617868FFF758FD02
:100F200007F10807BD4680BD80B483B000AF78608C
:100F30007B681B687A681268126922F001021A61E4
:100F400007F10C07BD4680BC704700BF80B483B07A
:100F500000AF786007F10C07BD4680BC704700BF4A
:100F600080B483B000AF786007F10C07BD4680BC49
:100F7000704700BF80B483B000AF786007F10C0702
:100F8000BD4680BC704700BF80B483B000AF7860BE
:100F900007F10C07BD4680BC704700BF80B485B028
:100FA00000AF786039604FF00003FB607B681B681E
:100FB000FB607A684FF00003C4F201039A421FD02D
:100FC0007B68B3F1804F1BD07A684FF48063C4F222
:100FD00000039A4214D07A684FF40063C4F200030D
:100FE0009A420DD07A684FF44063C4F200039A42EB
:100FF00006D07A684FF48063C4F201039A4202D1AA
:101000004FF0010301E04FF00003002B08D0FB6814
:1010100023F07003FB603B685B68FA681343FB6076
:101020007A684FF00003C4F201039A4249D07B680A
:10103000B3F1804F45D07A684FF48063C4F2000367
:101040009A423ED07A684FF40063C4F200039A4299
:1010500037D07A684FF44063C4F200039A4230D02C
:101060007A684FF48063C4F201039A4229D07A6807
:101070004FF48043C4F201039A4222D07A684FF4BD
:101080008843C4F201039A421BD07A684FF490431C
:10109000C4F201039A4214D07A684FF4C053C4F2E8
:1010A00000039A420DD07A684FF4E053C4F2000373
:1010B0009A4206D07A684FF40053C4F200039A4271
:1010C00002D14FF0010301E04FF00003002B08D0E4
:1010D000FB6823F44073FB603B68DB68FA681343EA
:1010E000FB607B68FA681A603B689A687B68DA6222
:1010F0003B681A687B689A627A684FF00003C4F212
:1011000001039A4206D07A684FF48063C4F2010367
:101110009A4202D14FF0010301E04FF00003002B8F
:1011200003D03B681A697B681A637B684FF0010241
:101130005A6107F11407BD4680BC704780B582B084
:1011400000AF78607B68002B02D14FF0010332E1E1
:101150007B685B68002B0CD07B685B68B3F5827F93
:1011600007D046F20C10C0F601004FF0A50106F0C2
:1011700093FE7B689B68002B11D07B689B68B3F55E
:10118000806F0CD07B689B68B3F5004F07D046F2A8
:101190000C10C0F601004FF0A60106F07DFE7B6842
:1011A000DB68B3F5006F0BD07B68DB68002B07D0E2
:1011B00046F20C10C0F601004FF0A70106F06CFEDD
:1011C0007B681B69002B0BD07B681B69022B07D047
:1011D00046F20C10C0F601004FF0A80106F05CFECC
:1011E0007B685B69002B0BD07B685B69012B07D0A8
:1011F00046F20C10C0F601004FF0A90106F04CFEBB
:101200007B689B69B3F5007F10D07B689B69002BDE
:101210000CD07B689B69B3F5802F07D046F20C1089
:10122000C0F601004FF0AA0106F036FE7B68DB69CC
:10123000002B23D07B68DB69082B1FD07B68DB6920
:10124000102B1BD07B68DB69182B17D07B68DB6900
:10125000202B13D07B68DB69282B0FD07B68DB69E0
:10126000302B0BD07B68DB69382B07D046F20C1093
:10127000C0F601004FF0AB0106F00EFE7B681B6A62
:10128000002B0BD07B681B6A802B07D046F20C101A
:10129000C0F601004FF0AC0106F0FEFD7B685B6A12
:1012A000002B0BD07B685B6A102B07D046F20C102A
:1012B000C0F601004FF0AD0106F0EEFD7B689B6AC1
:1012C000002B0CD07B689B6AB3F5005F07D046F219
:1012D0000C10C0F601004FF0AE0106F0DDFD7B689A
:1012E000DB6A002B05D07B68DA6A4FF6FF739A42FF
:1012F00007D946F20C10C0F601004FF0AF0106F01E
:10130000CBFD7B6893F85130DBB2002B02D17868BB
:1013100000F056F87B684FF0020283F851207B689A
:101320001B687A681268126822F040021A607B68B3
:101330001B687A6851687A68926811437A68D26843
:1013400011437A68126911437A68526911437A68C5
:10135000926902F4007211437A68D26911437A6883
:10136000126A11437A68926A0A431A607B681B68A2
:101370007A6892694FEA124202F004017A68526A6E
:101380000A435A607B681B687A68D26A1A617B6874
:101390001B687A681268D26922F40062DA617B689D
:1013A0004FF0000283F852207B684FF0010283F86F
:1013B00051204FF00003184607F10807BD4680BDD5
:1013C00080B483B000AF786007F10C07BD4680BCE5
:1013D000704700BF80B584B000AFF860B9603B6073
:1013E0001346FB80FB6893F85130DBB2012B40F0D1
:1013F0004F81BB68002B02D0FB88002B02D14FF03D
:10140000010347E1FB689B68002B0CD0FB689B68DD
:10141000B3F5004F07D046F20C10C0F601004FF4B0
:10142000AE7106F039FDFB6893F85030012B02D104
:101430004FF002032EE1FB684FF0010283F85020C9
:10144000FB684FF0120283F85120FB684FF0000256
:1014500083F85220FB68BA681A63FB68FA889A8698
:10146000FB68FA88DA86FB684FF00002DA64FB68F2
:101470004FF000029A64FB684FF000029A87FB6805
:101480004FF00002DA87FB689B6AB3F5005F0FD16B
:10149000FB681B68FA681268126822F400521A602E
:1014A000FB681B68FA681268126842F400521A60FE
:1014B000FB689B68B3F5004F07D1FB681B68FA68AF
:1014C0001268126842F480421A60FB681B681B684D
:1014D00003F04003002B07D1FB681B68FA68126811
:1014E000126842F040021A60FB68DB68002B42D1B0
:1014F000FB681A68FB681B6B1978D16003F1010265
:10150000FB681A63FB68DB8E03F1FF339AB2FB685A
:10151000DA861EE0F8684FF002014FF000023B68E7
:1015200000F0BEF80346002B02D04FF00303B1E0F9
:10153000FB681A68FB681B6B1978D16003F1010224
:10154000FB681A63FB68DB8E03F1FF339AB2FB681A
:10155000DA86FB68DB8E002BDCD1FB689B6AB3F577
:10156000005F4ED1FB681B68FA681268126842F48B
:1015700080521A6045E0FB681B68FA68126B12889B
:10158000DA60FB681B6B03F10202FB681A63FB68FD
:10159000DB8E03F1FF339AB2FB68DA8620E0F8684D
:1015A0004FF002014FF000023B6800F079F803466B
:1015B000002B02D04FF003036CE0FB681B68FA6855
:1015C000126B1288DA60FB681B6B03F10202FB6886
:1015D0001A63FB68DB8E03F1FF339AB2FB68DA868D
:1015E000FB68DB8E002BDAD1FB689B6AB3F5005FEA
:1015F00007D1FB681B68FA681268126842F48052CF
:101600001A60F8684FF002014FF000023B6800F0EA
:1016100047F80346002B0CD0FB6893F85230DBB23E
:1016200043F02003DAB2FB6883F852204FF0030343
:1016300030E0F8684FF080014FF001023B6800F0A5
:101640002FF80346002B0CD0FB6893F85230DBB226
:1016500043F02003DAB2FB6883F852204FF0030313
:1016600018E0FB689B68002B05D1FB681B68DB68F2
:10167000FB681B689B68FB684FF0010283F85120F0
:10168000FB684FF0000283F850204FF0000301E0A8
:101690004FF00203184607F11007BD4680BD00BF9A
:1016A00080B586B000AFF860B9603B601346FB714F
:1016B0004FF000037B6106F0E3FB02463B68D31862
:1016C0007B61FB79002B40F083803BE03B68B3F10A
:1016D000FF3F37D006F0D4FB02467B699A4231D3F4
:1016E000FB681B68FA681268526822F0E0025A60D0
:1016F000FB681B68FA681268126822F040021A60E0
:10170000FB689B6AB3F5005F0FD1FB681B68FA6842
:101710001268126822F400521A60FB681B68FA68AB
:101720001268126842F400521A60FB684FF001021E
:1017300083F85120FB684FF0000283F850204FF0EF
:10174000030351E0FB681B689B681A46BB681A409C
:10175000BB689A42BAD145E03B68B3F1FF3F38D04D
:1017600006F08EFB02467B699A4232D3FB681B6807
:10177000FA681268526822F0E0025A60FB681B683F
:10178000FA681268126822F040021A60FB689B6ACD
:10179000B3F5005F0FD1FB681B68FA681268126826
:1017A00022F400521A60FB681B68FA68126812681B
:1017B00042F400521A60FB684FF0010283F8512096
:1017C000FB684FF0000283F850204FF003030BE05A
:1017D00000BFFB681B689B681A46BB681A40BB6861
:1017E0009A42B9D04FF00003184607F11807BD46DA
:1017F00080BD00BF80B483B000AF03463960FB7189
:1018000097F90730002B10DA4FF46D43CEF2000346
:10181000FA7902F00F02A2F104013A68D2B24FEA5B
:101820000212D2B25B181A760DE04FF46143CEF289
:10183000000397F907103A68D2B24FEA0212D2B207
:101840005B1883F8002307F10C07BD4680BC704786
:1018500080B582B000AF78607B6803F1FF326FF033
:101860007F439A4202D94FF001031DE04EF210036C
:10187000CEF200037A6802F1FF325A604FF0FF3077
:101880004FF00F01FFF7B6FF4EF21003CEF2000348
:101890004FF000029A604EF21003CEF200034FF0B8
:1018A00007021A604FF00003184607F10807BD460B
:1018B00080BD00BF90B595B000AF78604FF00003D9
:1018C000FB647B681B680F2B07D946F24C10C0F6EF
:1018D00001004FF49D7106F0DFFA7B681B6803F08E
:1018E0000103DBB2002B00F0A6807B685B68002B55
:1018F0000FD07B685B68012B0BD07B685B68052B86
:1019000007D046F24C10C0F6010040F23F1106F03D
:10191000C3FA4FF46053C4F202039B6803F00C0354
:10192000042B11D04FF46053C4F202039B6803F000
:101930000C03082B18D14FF46053C4F202035B6808
:1019400003F48003002B0FD04FF46053C4F2020362
:101950001B6803F40033002B6CD07B685B68012BA1
:1019600068D04FF0010358E343F60203C4F20203C8
:101970004FF000021A7006F083FA034603F59C53F9
:1019800003F10803FB6408E006F07AFA0246FB6CF8
:101990009A4202D34FF003033FE34FF46053C4F283
:1019A00002031B6803F40033002BEDD143F602035E
:1019B000C4F202037A685268D2B21A707B685B681C
:1019C000012B1BD106F05CFA034603F59C5303F18F
:1019D0000803FB6408E006F053FA0246FB6C9A42E7
:1019E00002D34FF0030318E34FF46053C4F2020331
:1019F0001B6803F40033002BEDD01CE006F040FA26
:101A0000034603F59C5303F10803FB6408E006F06A
:101A100037FA0246FB6C9A4202D34FF00303FCE212
:101A20004FF46053C4F202031B6803F40033002B2D
:101A3000EDD100E000BF7B681B6803F00203002BC0
:101A400000F0AE807B68DB68002B0BD07B68DB6826
:101A5000012B07D046F24C10C0F6010040F27F1176
:101A600006F01AFA7B681B691F2B07D946F24C1047
:101A7000C0F601004FF4C07106F00EFA4FF4605347
:101A8000C4F202039B6803F00C03002B11D04FF447
:101A90006053C4F202039B6803F00C03082B18D1B7
:101AA0004FF46053C4F202035B6803F48003002B1D
:101AB0000FD14FF46053C4F202031B6803F002031A
:101AC000002B6CD07B68DB68012B68D04FF00103E2
:101AD000A3E27B68DB68002B40D04FF00003C4F228
:101AE00047234FF001021A6006F0CAF9034603F1DA
:101AF0006403FB6408E006F0C3F90246FB6C9A42FB
:101B000002D34FF0030388E24FF46053C4F20203A0
:101B10001B6803F00203002BEDD04FF46053C4F2B6
:101B200002034FF46052C4F20202126822F0F8017C
:101B30007A6810694FF0F802BA64BA6C92FAA2F4AB
:101B40007C647A6C3A643A6CB2FA82F4FC63FA6BA5
:101B5000D2B200FA02F20A431A6021E04FF0000309
:101B6000C4F247234FF000021A6006F089F90346D9
:101B700003F16403FB6408E006F082F90246FB6CA3
:101B80009A4202D34FF0030347E24FF46053C4F28A
:101B900002031B6803F00203002BEDD100E000BF3D
:101BA0007B681B6803F00803002B54D07B685B69DB
:101BB000002B0BD07B685B69012B07D046F24C10E1
:101BC000C0F601004FF4DC7106F066F97B685B69D2
:101BD000002B20D04FF46863C4F247234FF001027A
:101BE0001A6006F04DF9034603F16403FB6408E054
:101BF00006F046F90246FB6C9A4202D34FF003030B
:101C00000BE24FF46053C4F202035B6F03F0020374
:101C1000002BEDD01FE04FF46863C4F247234FF070
:101C200000021A6006F02CF9034603F16403FB641A
:101C300008E006F025F90246FB6C9A4202D34FF009
:101C40000303EAE14FF46053C4F202035B6F03F055
:101C50000203002BEDD17B681B6803F00403002B0B
:101C600000F0AA807B689B68002B0FD07B689B6884
:101C7000012B0BD07B689B68052B07D046F24C10DC
:101C8000C0F601004FF4F17106F006F94FF460530D
:101C9000C4F202034FF46052C4F20202126C42F02A
:101CA00080521A644FF4E043C4F200034FF4E04260
:101CB000C4F20002126842F480721A6006F0E0F882
:101CC000034603F16403FB6408E006F0D9F802461A
:101CD000FB6C9A4202D34FF003039EE14FF4E043C2
:101CE000C4F200031B6803F48073002BEDD043F6AD
:101CF0007003C4F202034FF000021A7006F0C0F83D
:101D0000034603F59C5303F10803FB6408E006F067
:101D1000B7F80246FB6C9A4202D34FF003037CE112
:101D20004FF46053C4F202031B6F03F00203002B55
:101D3000EDD143F67003C4F202037A689268D2B21E
:101D40001A707B689B68012B1BD106F099F803463B
:101D500003F59C5303F10803FB6408E006F090F8D8
:101D60000246FB6C9A4202D34FF0030355E14FF455
:101D70006053C4F202031B6F03F00203002BEDD08B
:101D80001AE006F07DF8034603F59C5303F10803BF
:101D9000FB6408E006F074F80246FB6C9A4202D33A
:101DA0004FF0030339E14FF46053C4F202031B6F99
:101DB00003F00203002BEDD17B689B69002B0FD051
:101DC0007B689B69012B0BD07B689B69022B07D03A
:101DD00046F24C10C0F6010040F2262106F05CF8F5
:101DE0007B689B69002B00F016814FF46053C4F2AE
:101DF00002039B6803F00C03082B00F009817B6849
:101E00009B69022B40F0E3807B68DB69002B0CD0E0
:101E10007B68DB69B3F5800F07D046F24C10C0F643
:101E2000010040F22F2106F037F87B681B6A3F2B38
:101E300007D946F24C10C0F601004FF40C7106F0C1
:101E40002BF87B685B6ABF2B04D97B685B6AB3F5B0
:101E5000D87F07D946F24C10C0F6010040F231217C
:101E600006F01AF87B689B6A022B13D07B689B6A8A
:101E7000042B0FD07B689B6A062B0BD07B689B6A78
:101E8000082B07D046F24C10C0F6010040F2322178
:101E900006F002F87B68DB6A032B03D97B68DB6AF8
:101EA0000F2B07D946F24C10C0F6010040F2332147
:101EB00005F0F2FF4FF06003C4F247234FF0000239
:101EC0001A6005F0DDFF034603F16403FB6408E0DC
:101ED00005F0D6FF0246FB6C9A4202D34FF0030393
:101EE0009BE04FF46053C4F202031B6803F00073DD
:101EF000002BEDD14FF46053C4F202037A68116AEB
:101F00007A68506A47F6C072BA63BA6B92FAA2F462
:101F10007C637A6B3A633A6BB2FA82F4FC62FA6AD7
:101F2000D2B200FA02F211437A68926A4FEA520280
:101F300002F1FF304FF44032BA62BA6A92FAA2F468
:101F40007C627A6A3A623A6AB2FA82F4FC61FA69AD
:101F5000D2B200FA02F211437A68D26911437A6868
:101F6000D06A4FF07062BA61BA6992FAA2F47C61E9
:101F70007A693A613A69B2FA82F4FC60FA68D2B2DC
:101F800000FA02F20A4342F000525A604FF0600336
:101F9000C4F247234FF001021A6005F071FF0346B7
:101FA00003F16403FB6408E005F06AFF0246FB6C82
:101FB0009A4202D34FF003032FE04FF46053C4F270
:101FC00002031B6803F00073002BEDD023E04FF0F9
:101FD0006003C4F247234FF000021A6005F050FF7F
:101FE000034603F16403FB6408E005F049FF024681
:101FF000FB6C9A4202D34FF003030EE04FF46053A0
:10200000C4F202031B6803F00073002BEDD102E061
:102010004FF0010301E04FF00003184607F15407A9
:10202000BD4690BD80B584B000AF786039604FF098
:102030000003FB607B681B68002B03D07B681B6878
:102040000F2B07D946F24C10C0F6010040F2962142
:1020500005F022FF3B68002B34D03B68012B31D0C8
:102060003B68022B2ED03B68032B2BD03B68042B04
:1020700028D03B68052B25D03B68062B22D03B6837
:10208000072B1FD03B68082B1CD03B68092B19D0AD
:102090003B680A2B16D03B680B2B13D03B680C2BEC
:1020A00010D03B680D2B0DD03B680E2B0AD03B683F
:1020B0000F2B07D046F24C10C0F6010040F29721DA
:1020C00005F0EAFE4FF47053C4F202031B6803F0FC
:1020D0000F023B689A4280F0B7804FF47053C4F20D
:1020E00002033A68D2B21A704FF47053C4F202037A
:1020F0001B6803F00F023B689A4202D04FF00103C5
:1021000015E27B681B6803F00103DBB2002B00F0D3
:1021100051817B685B68002B0FD07B685B68012B6B
:102120000BD07B685B68022B07D046F24C10C0F6E0
:10213000010040F2AD2105F0AFFE7B685B68012B2A
:102140000BD14FF46053C4F202031B6803F4003355
:10215000002B1ED14FF00103E9E17B685B68022B85
:102160000BD14FF46053C4F202031B6803F00073F9
:10217000002B0ED14FF00103D9E14FF46053C4F2AC
:1021800002031B6803F00203002B02D14FF001038E
:10219000CDE14FF46053C4F202034FF46052C4F235
:1021A0000202926822F003017A6852680A439A6038
:1021B00005F066FE034603F59C5303F10803FB603C
:1021C0007B685B68012B13D108E005F059FE0246DD
:1021D000FB689A4202D34FF00303A8E14FF4605327
:1021E000C4F202039B6803F00C03042BEDD1E1E081
:1021F0007B685B68022B1CD108E005F041FE0246BB
:10220000FB689A4202D34FF0030390E14FF460530E
:10221000C4F202039B6803F00C03082BEDD1C9E064
:1022200005F02EFE0246FB689A4203D34FF00303EB
:102230007DE100BF4FF46053C4F202039B6803F0DA
:102240000C03002BECD1B5E07B681B6803F00103A5
:10225000DBB2002B00F09A807B685B68002B0FD00C
:102260007B685B68012B0BD07B685B68022B07D017
:1022700046F24C10C0F6010040F2F52105F00CFECC
:102280007B685B68012B0BD14FF46053C4F20203EF
:102290001B6803F40033002B1ED14FF0010346E10D
:1022A0007B685B68022B0BD14FF46053C4F20203CE
:1022B0001B6803F00073002B0ED14FF0010336E1D1
:1022C0004FF46053C4F202031B6803F00203002BB7
:1022D00002D14FF001032AE14FF46053C4F202032C
:1022E0004FF46052C4F20202926822F003017A684D
:1022F00052680A439A6005F0C3FD034603F59C53F8
:1023000003F10803FB607B685B68012B13D108E0D5
:1023100005F0B6FD0246FB689A4202D34FF0030374
:1023200005E14FF46053C4F202039B6803F00C0311
:10233000042BEDD12AE07B685B68022B1CD108E0FE
:1023400005F09EFD0246FB689A4202D34FF003035C
:10235000EDE04FF46053C4F202039B6803F00C03FA
:10236000082BEDD112E005F08BFD0246FB689A4286
:1023700003D34FF00303DAE000BF4FF46053C4F21D
:1023800002039B6803F00C03002BECD14FF4705355
:10239000C4F202033A68D2B21A704FF47053C4F216
:1023A00002031B6803F00F023B689A4202D04FF011
:1023B0000103BCE07B681B6803F00203002B3AD0EA
:1023C0007B689B68002B27D07B689B68802B23D081
:1023D0007B689B68902B1FD07B689B68A02B1BD0D1
:1023E0007B689B68B02B17D07B689B68C02B13D091
:1023F0007B689B68D02B0FD07B689B68E02B0BD051
:102400007B689B68F02B07D046F24C10C0F60100A9
:1024100040F2453105F040FD4FF46053C4F2020331
:102420004FF46052C4F20202926822F0F0017A681E
:1024300092680A439A607B681B6803F00403002BD0
:102440002ED07B68DB68002B1BD07B68DB68B3F584
:10245000805F16D07B68DB68B3F5A05F11D07B6826
:10246000DB68B3F5C05F0CD07B68DB68B3F5E05F79
:1024700007D046F24C10C0F601004FF4537105F03E
:102480000BFD4FF46053C4F202034FF46052C4F2E8
:102490000202926822F4E0517A68D2680A439A6094
:1024A0007B681B6803F00803002B30D07B681B6936
:1024B000002B1BD07B681B69B3F5805F16D07B684F
:1024C0001B69B3F5A05F11D07B681B69B3F5C05FD2
:1024D0000CD07B681B69B3F5E05F07D046F24C1067
:1024E000C0F6010040F2533105F0D6FC4FF46053C2
:1024F000C4F202034FF46052C4F20202926822F462
:1025000060417A6812694FEAC2020A439A6000F099
:10251000D7F8024644F6D353C1F26203A3FB021379
:102520004FEA93131846FFF793F94FF0000318464C
:1025300007F11007BD4680BD90B494B000AF4FF0D6
:1025400000037B644FF00003FB644FF000033B6427
:102550004FF00003BB644FF46053C4F202039B6866
:1025600003F00C03042B0AD0082B0ED0002B40F0F4
:102570009A804FF41053C0F2F403BB6499E04FF417
:102580005853C0F26E13BB6493E04FF46053C4F22F
:1025900002035B6803F03F037B644FF46053C4F2B3
:1025A00002035B6803F480024FF48003FB63FB6B60
:1025B00093FAA3F4BC63BB6B7B637B6BB3FA83F4CA
:1025C0003C633B6BDBB222FA03F3002B24D04FF4C5
:1025D0005853C0F26E137A6CB3FBF2F24FF46053AF
:1025E000C4F202035B68194647F6C0730B4047F616
:1025F000C071F962F96A91FAA1F4BC62B96A7962B0
:10260000796AB1FA81F43C62396AC9B223FA01F3FA
:1026100003FB02F3FB6423E04FF41053C0F2F40316
:102620007A6CB3FBF2F24FF46053C4F202035B68BE
:10263000194647F6C0730B4047F6C071F961F96956
:1026400091FAA1F4BC61B96979617969B1FA81F44F
:102650003C613969C9B223FA01F303FB02F3FB645D
:102660004FF46053C4F202035B6803F440324FF44A
:102670004033FB60FB6893FAA3F4BC60BB687B60EB
:102680007B68B3FA83F43C603B68DBB222FA03F365
:1026900003F101034FEA43033B64FA6C3B6CB2FB6A
:1026A000F3F3BB6405E04FF41053C0F2F403BB64D2
:1026B00000BFBB6C184607F15007BD4690BC704781
:1026C00090B585B000AFFFF737FF02464FF4605377
:1026D000C4F202039B6803F0F0014FF0F003FB60CB
:1026E000FB6893FAA3F4BC60BB687B607B68B3FAB9
:1026F00083F43C603B68DBB221FA03F146F23C1301
:10270000C0F601035B5C22FA03F240F20C03C2F252
:1027100000031A6040F20C03C2F200031B68184663
:1027200007F11407BD4690BD90B587B000AF786043
:1027300039604FF000033B614FF00003FB604FF046
:102740000003BB603B681B68002B07D146F27C107E
:10275000C0F601004FF0C30105F09EFB3B685B68CB
:10276000002B4BD03B685B68012B47D03B685B6814
:10277000112B43D03B685B68022B3FD03B685B6802
:10278000122B3BD03B685A684FF00003C1F2110393
:102790009A4233D03B685A684FF00003C1F22103DC
:1027A0009A422BD03B685A684FF00003C1F23103C4
:1027B0009A4223D03B685A684FF00003C1F21203DB
:1027C0009A421BD03B685A684FF00003C1F22203C3
:1027D0009A4213D03B685A684FF00003C1F23203AB
:1027E0009A420BD03B685B68032B07D046F27C1003
:1027F000C0F601004FF0C40105F04EFB3B689B683A
:10280000002B0FD03B689B68012B0BD03B689B686B
:10281000022B07D046F27C10C0F601004FF0C50134
:1028200005F03AFB4FF000037B61F5E27B694FF066
:10283000010202FA03F33B613B681A683B691340EB
:10284000FB60FA683B699A4240F0E2823B685B6851
:10285000022B04D03B685B68122B40F0FA803B6887
:102860001B69002B00F0BB803B681B69092B00F043
:10287000B6803B681B69002B00F0B1803B681B6988
:10288000002B00F0AC803B681B69002B00F0A78098
:102890003B681B69002B00F0A2803B681B69012B81
:1028A00000F09D803B681B69012B00F098803B681D
:1028B0001B69022B00F093803B681B69022B00F020
:1028C0008E803B681B69022B00F089803B681B6986
:1028D000032B00F084803B681B69042B7FD03B688E
:1028E0001B69042B7BD03B681B69042B77D03B68AA
:1028F0001B69052B73D03B681B69052B6FD03B68A8
:102900001B69092B6BD03B681B69062B67D03B68A2
:102910001B69092B63D03B681B69072B5FD03B68A1
:102920001B69072B5BD03B681B69072B57D03B68A3
:102930001B69082B53D03B681B69082B4FD03B68A1
:102940001B69082B4BD03B681B69092B47D03B68A0
:102950001B69092B43D03B681B690A2B3FD03B689E
:102960001B690A2B3BD03B681B690B2B37D03B689C
:102970001B690C2B33D03B681B690C2B2FD03B6899
:102980001B690D2B2BD03B681B690F2B27D03B6895
:102990001B69052B23D03B681B69052B1FD03B68A7
:1029A0001B69052B1BD03B681B69082B17D03B68A4
:1029B0001B69082B13D03B681B690C2B0FD03B689D
:1029C0001B69062B0BD03B681B690E2B07D046F208
:1029D0007C10C0F601004FF0D60105F05DFA3B68AF
:1029E0001A697B6903F007034FEA830302FA03F3D2
:1029F000BB607B694FEAD3027B694FEAD3017B68F6
:102A000001F1080153F8213019467B6903F00703EF
:102A10004FEA83034FF00F0000FA03F36FEA03035A
:102A200019407B6802F1080243F822107B694FEAE3
:102A3000D3027B694FEAD3017B6801F1080153F8A7
:102A400021301946BB6819437B6802F1080243F83C
:102A500022107B681B681A467B694FEA43034FF0DC
:102A6000030101FA03F36FEA03031A407B681A605B
:102A70007B681B681A463B685B6803F003017B694F
:102A80004FEA430301FA03F31A437B681A603B6879
:102A90005B68012B0BD03B685B68022B07D03B685F
:102AA0005B68112B03D03B685B68122B4FD13B68EE
:102AB000DB68002B13D03B68DB68012B0FD03B6831
:102AC000DB68022B0BD03B68DB68032B07D046F298
:102AD0007C10C0F601004FF0E60105F0DDF97B68DF
:102AE0009B681A467B694FEA43034FF0030101FAE2
:102AF00003F36FEA03031A407B689A607B689B6864
:102B00001A463B68D9687B694FEA430301FA03F32D
:102B10001A437B689A607B685B681A467B694FF052
:102B2000010101FA03F36FEA03031A407B685A605C
:102B30007B685B681A463B685B6803F010034FEAEA
:102B400013117B6901FA03F31A437B685A607B68AF
:102B5000DB681A467B694FEA43034FF0030101FA31
:102B600003F36FEA03031A407B68DA607B68DB6873
:102B70001A463B6899687B694FEA430301FA03F3FD
:102B80001A437B68DA603B685B6803F08053002B74
:102B900000F03E814FF46053C4F202034FF46052E0
:102BA000C4F20202526C42F480425A647B6903F020
:102BB00003034FEA83034FF00F0202FA03F3BB60F3
:102BC0004FF46053C4F201037A694FEA92004FF464
:102BD0006052C4F2010279694FEA910101F10201E8
:102BE00052F821201146BA686FEA0202114000F142
:102BF000020243F822104FF46053C4F201037A69D1
:102C00004FEA92004FF46052C4F2010279694FEA30
:102C1000910101F1020152F8212011467C684FF028
:102C20000002C4F2020294425CD07C684FF48062DD
:102C3000C4F20202944252D07C684FF40062C4F2A3
:102C40000202944248D07C684FF44062C4F202020F
:102C500094423ED07C684FF48052C4F20202944207
:102C600034D07C684FF4A052C4F2020294422AD0BD
:102C70007C684FF4C052C4F20202944220D07C68B7
:102C80004FF4E052C4F20202944216D07C684FF432
:102C90000052C4F2020294420CD07C684FF41052ED
:102CA000C4F20202944202D14FF0090201E04FF057
:102CB0000A0201E04FF0080201E04FF0070201E0D4
:102CC0004FF0060201E04FF0050201E04FF0040270
:102CD00001E04FF0030201E04FF0020201E04FF08B
:102CE000010201E04FF000027C6904F003044FEAA6
:102CF000840402FA04F2114300F1020243F82210A4
:102D00004FF47053C4F201034FF47052C4F2010245
:102D100012681146FA686FEA02020A401A604FF41C
:102D20007053C4F201034FF47052C4F201025268AE
:102D30001146FA686FEA02020A405A603B685B6813
:102D400003F48033002B0CD04FF47053C4F2010312
:102D50004FF47052C4F2010212681146FA680A4335
:102D60001A603B685B6803F40033002B0CD04FF40F
:102D70007053C4F201034FF47052C4F2010252685E
:102D80001146FA680A435A604FF47053C4F20103C3
:102D90004FF47052C4F2010292681146FA686FEA69
:102DA00002020A409A604FF47053C4F201034FF4D8
:102DB0007052C4F20102D2681146FA686FEA020248
:102DC0000A40DA603B685B6803F48013002B0CD088
:102DD0004FF47053C4F201034FF47052C4F2010275
:102DE00092681146FA680A439A603B685B6803F48C
:102DF0000013002B0CD04FF47053C4F201034FF4B6
:102E00007052C4F20102D2681146FA680A43DA60CD
:102E10007B6903F101037B617B690F2B7FF606ADB4
:102E200007F11C07BD4690BD80B584B000AF786047
:102E30000B467B807B88012B3CD07B88022B39D0D2
:102E40007B88042B36D07B88082B33D07B88102BD3
:102E500030D07B88202B2DD07B88402B2AD07B88BC
:102E6000802B27D07B88B3F5807F23D07B88B3F578
:102E7000007F1FD07B88B3F5806F1BD07B88B3F5B4
:102E8000006F17D07B88B3F5805F13D07B88B3F5D4
:102E9000005F0FD07B88B3F5804F0BD07B88B3F5F4
:102EA000004F07D046F27C10C0F6010040F27511C9
:102EB00004F0F2FF7B681B691A467B881340002BE5
:102EC00003D04FF00103FB7302E04FF00003FB73EC
:102ED000FB7B184607F11007BD4680BD80B582B068
:102EE00000AF786013460A467A807B707B88012B9E
:102EF0003CD07B88022B39D07B88042B36D07B8852
:102F0000082B33D07B88102B30D07B88202B2DD002
:102F10007B88402B2AD07B88802B27D07B88B3F5F9
:102F2000807F23D07B88B3F5007F1FD07B88B3F5EB
:102F3000806F1BD07B88B3F5006F17D07B88B3F50B
:102F4000805F13D07B88B3F5005F0FD07B88B3F52B
:102F5000804F0BD07B88B3F5004F07D046F27C1032
:102F6000C0F601004FF4CB7104F096FF7B78002B84
:102F70000AD07B78012B07D046F27C10C0F6010006
:102F800040F2971104F088FF7B78002B03D07B6818
:102F90007A881A8302E07B687A885A8307F10807E7
:102FA000BD4680BD80B582B000AF78607B681B688D
:102FB0001A4646F25843C4F202039A4240F2938002
:102FC0004FF4C843C4F202035B681A467B68196871
:102FD00046F21003C4F2020399427BD07B68196861
:102FE00046F21043C4F20203994270D07B6819681C
:102FF00046F27003C4F20203994265D07B681968F7
:1030000046F27043C4F2020399425AD07B681968B1
:1030100046F22803C4F2020399424FD07B68196834
:1030200046F22843C4F20203994244D07B681968EF
:1030300046F28803C4F20203994239D07B681968CA
:1030400046F28843C4F2020399422ED07B68196885
:1030500046F24003C4F20203994223D07B68196808
:1030600046F24043C4F20203994218D07B681968C3
:1030700046F2A003C4F2020399420DD07B6819689E
:1030800046F2A043C4F20203994202D14FF4002356
:1030900001E04FF0007301E04FF4002301E04FF432
:1030A000002301E04FF4002301E04FF4007301E03E
:1030B0004FF4007301E04FF4007301E04FF400732C
:1030C00001E04FF0080301E04FF0080301E04FF08A
:1030D000080301E04FF008031340002B0CBF00234E
:1030E0000123DBB2CBE17B681B681A4646F2B803CA
:1030F000C4F202039A4240F293804FF4C843C4F2F0
:1031000002031B681A467B68196846F21003C4F272
:10311000020399427BD07B68196846F21043C4F2DF
:103120000203994270D07B68196846F27003C4F2BA
:103130000203994265D07B68196846F27043C4F275
:10314000020399425AD07B68196846F22803C4F2F8
:10315000020399424FD07B68196846F22843C4F2B3
:103160000203994244D07B68196846F28803C4F28E
:103170000203994239D07B68196846F28843C4F249
:10318000020399422ED07B68196846F24003C4F2CC
:103190000203994223D07B68196846F24043C4F287
:1031A0000203994218D07B68196846F2A003C4F262
:1031B000020399420DD07B68196846F2A043C4F21D
:1031C0000203994202D14FF4002301E04FF0007353
:1031D00001E04FF4002301E04FF4002301E04FF43D
:1031E000002301E04FF4007301E04FF4007301E0AD
:1031F0004FF4007301E04FF4007301E04FF0080357
:1032000001E04FF0080301E04FF0080301E04FF048
:1032100008031340002B0CBF00230123DBB22EE177
:103220007B681B681A4646F25803C4F202039A42AE
:1032300040F293804FF4C043C4F202035B681A4625
:103240007B68196846F21003C4F2020399427BD0EE
:103250007B68196846F21043C4F20203994270D0A9
:103260007B68196846F27003C4F20203994265D084
:103270007B68196846F27043C4F2020399425AD03F
:103280007B68196846F22803C4F2020399424FD0C2
:103290007B68196846F22843C4F20203994244D07D
:1032A0007B68196846F28803C4F20203994239D058
:1032B0007B68196846F28843C4F2020399422ED013
:1032C0007B68196846F24003C4F20203994223D096
:1032D0007B68196846F24043C4F20203994218D051
:1032E0007B68196846F2A003C4F2020399420DD02C
:1032F0007B68196846F2A043C4F20203994202D1E6
:103300004FF4002301E04FF0007301E04FF400237D
:1033100001E04FF4002301E04FF4002301E04FF4FB
:10332000007301E04FF4007301E04FF4007301E01B
:103330004FF4007301E04FF0080301E04FF0080381
:1033400001E04FF0080301E04FF008031340002BA9
:103350000CBF00230123DBB291E04FF4C043C4F261
:1033600002031B681A467B68196846F21003C4F210
:10337000020399427BD07B68196846F21043C4F27D
:103380000203994270D07B68196846F27003C4F258
:103390000203994265D07B68196846F27043C4F213
:1033A000020399425AD07B68196846F22803C4F296
:1033B000020399424FD07B68196846F22843C4F251
:1033C0000203994244D07B68196846F28803C4F22C
:1033D0000203994239D07B68196846F28843C4F2E7
:1033E000020399422ED07B68196846F24003C4F26A
:1033F0000203994223D07B68196846F24043C4F225
:103400000203994218D07B68196846F2A003C4F2FF
:10341000020399420DD07B68196846F2A043C4F2BA
:103420000203994202D14FF4002301E04FF00073F0
:1034300001E04FF4002301E04FF4002301E04FF4DA
:10344000002301E04FF4007301E04FF4007301E04A
:103450004FF4007301E04FF4007301E04FF00803F4
:1034600001E04FF0080301E04FF0080301E04FF0E6
:1034700008031340002B0CBF00230123DBB2002BF9
:1034800000F091827B681B681B6803F00403002B2B
:1034900000F089827B681B687A681268126822F0E3
:1034A00004021A607B681B681A4646F25843C4F24D
:1034B00002039A4240F293804FF4C843C4F20203DD
:1034C0004FF4C842C4F20202D26811467A6810680A
:1034D00046F21002C4F2020290427BD07A68106871
:1034E00046F21042C4F20202904270D07A6810682C
:1034F00046F27002C4F20202904265D07A68106807
:1035000046F27042C4F2020290425AD07A681068C1
:1035100046F22802C4F2020290424FD07A68106844
:1035200046F22842C4F20202904244D07A681068FF
:1035300046F28802C4F20202904239D07A681068DA
:1035400046F28842C4F2020290422ED07A68106895
:1035500046F24002C4F20202904223D07A68106818
:1035600046F24042C4F20202904218D07A681068D3
:1035700046F2A002C4F2020290420DD07A681068AE
:1035800046F2A042C4F20202904202D14FF400225D
:1035900001E04FF0007201E04FF4002201E04FF42F
:1035A000002201E04FF4002201E04FF4007201E03C
:1035B0004FF4007201E04FF4007201E04FF400722A
:1035C00001E04FF0080201E04FF0080201E04FF087
:1035D000080201E04FF008020A43DA60CBE17B68A1
:1035E0001B681A4646F2B803C4F202039A4240F23C
:1035F00093804FF4C843C4F202034FF4C842C4F2AC
:103600000202926811467A68106846F21002C4F20B
:10361000020290427BD07A68106846F21042C4F2EF
:103620000202904270D07A68106846F27002C4F2CA
:103630000202904265D07A68106846F27042C4F285
:10364000020290425AD07A68106846F22802C4F208
:10365000020290424FD07A68106846F22842C4F2C3
:103660000202904244D07A68106846F28802C4F29E
:103670000202904239D07A68106846F28842C4F259
:10368000020290422ED07A68106846F24002C4F2DC
:103690000202904223D07A68106846F24042C4F297
:1036A0000202904218D07A68106846F2A002C4F272
:1036B000020290420DD07A68106846F2A042C4F22D
:1036C0000202904202D14FF4002201E04FF000725A
:1036D00001E04FF4002201E04FF4002201E04FF43A
:1036E000002201E04FF4007201E04FF4007201E0AB
:1036F0004FF4007201E04FF4007201E04FF0080255
:1037000001E04FF0080201E04FF0080201E04FF045
:1037100008020A439A602EE17B681B681A4646F24B
:103720005803C4F202039A4240F293804FF4C0431C
:10373000C4F202034FF4C042C4F20202D26811463E
:103740007A68106846F21002C4F2020290427BD0FE
:103750007A68106846F21042C4F20202904270D0B9
:103760007A68106846F27002C4F20202904265D094
:103770007A68106846F27042C4F2020290425AD04F
:103780007A68106846F22802C4F2020290424FD0D2
:103790007A68106846F22842C4F20202904244D08D
:1037A0007A68106846F28802C4F20202904239D068
:1037B0007A68106846F28842C4F2020290422ED023
:1037C0007A68106846F24002C4F20202904223D0A6
:1037D0007A68106846F24042C4F20202904218D061
:1037E0007A68106846F2A002C4F2020290420DD03C
:1037F0007A68106846F2A042C4F20202904202D1F6
:103800004FF4002201E04FF0007201E04FF400227B
:1038100001E04FF4002201E04FF4002201E04FF4F8
:10382000007201E04FF4007201E04FF4007201E019
:103830004FF4007201E04FF0080201E04FF008027F
:1038400001E04FF0080201E04FF008020A43DA609D
:1038500091E04FF4C043C4F202034FF4C042C4F2FB
:103860000202926811467A68106846F21002C4F2A9
:10387000020290427BD07A68106846F21042C4F28D
:103880000202904270D07A68106846F27002C4F268
:103890000202904265D07A68106846F27042C4F223
:1038A000020290425AD07A68106846F22802C4F2A6
:1038B000020290424FD07A68106846F22842C4F261
:1038C0000202904244D07A68106846F28802C4F23C
:1038D0000202904239D07A68106846F28842C4F2F7
:1038E000020290422ED07A68106846F24002C4F27A
:1038F0000202904223D07A68106846F24042C4F235
:103900000202904218D07A68106846F2A002C4F20F
:10391000020290420DD07A68106846F2A042C4F2CA
:103920000202904202D14FF4002201E04FF00072F7
:1039300001E04FF4002201E04FF4002201E04FF4D7
:10394000002201E04FF4007201E04FF4007201E048
:103950004FF4007201E04FF4007201E04FF00802F2
:1039600001E04FF0080201E04FF0080201E04FF0E3
:1039700008020A439A607B68DB6C43F001027B68B3
:10398000DA647B684FF0040283F835207B684FF0DF
:10399000000283F834207B689B6C002B03D07B688B
:1039A0009B6C786898477B681B681A4646F25843B8
:1039B000C4F202039A4240F29C804FF4C843C4F21E
:1039C00002035B681A467B68196846F21003C4F26A
:1039D0000203994200F082807B68196846F2104326
:1039E000C4F20203994274D07B68196846F27003EE
:1039F000C4F20203994267D07B68196846F27043AB
:103A0000C4F2020399425AD07B68196846F228032F
:103A1000C4F2020399424FD07B68196846F22843EA
:103A2000C4F20203994244D07B68196846F28803C5
:103A3000C4F20203994239D07B68196846F2884380
:103A4000C4F2020399422ED07B68196846F2400303
:103A5000C4F20203994223D07B68196846F24043BE
:103A6000C4F20203994218D07B68196846F2A00399
:103A7000C4F2020399420DD07B68196846F2A04354
:103A8000C4F20203994202D14FF4803301E04FF4B3
:103A9000800301E04FF4803301E04FF4803301E014
:103AA0004FF4803301E04FF0400301E04FF040035A
:103AB00001E04FF0400301E04FF0400303E04FF01E
:103AC0000103C0F2800303E04FF00103C0F2800362
:103AD00003E04FF00103C0F2800303E04FF0010365
:103AE000C0F280031340002B0CBF00230123DBB284
:103AF000E6E17B681B681A4646F2B803C4F202038B
:103B00009A4240F29C804FF4C843C4F202031B68FF
:103B10001A467B68196846F21003C4F20203994200
:103B200000F082807B68196846F21043C4F20203F9
:103B3000994274D07B68196846F27003C4F202039C
:103B4000994267D07B68196846F27043C4F2020359
:103B500099425AD07B68196846F22803C4F20203DE
:103B600099424FD07B68196846F22843C4F2020399
:103B7000994244D07B68196846F28803C4F2020374
:103B8000994239D07B68196846F28843C4F202032F
:103B900099422ED07B68196846F24003C4F20203B2
:103BA000994223D07B68196846F24043C4F202036D
:103BB000994218D07B68196846F2A003C4F2020348
:103BC00099420DD07B68196846F2A043C4F2020303
:103BD000994202D14FF4803301E04FF4800301E0B9
:103BE0004FF4803301E04FF4803301E04FF4803331
:103BF00001E04FF0400301E04FF0400301E04FF0DF
:103C0000400301E04FF0400303E04FF00103C0F236
:103C1000800303E04FF00103C0F2800303E04FF0A4
:103C20000103C0F2800303E04FF00103C0F2800300
:103C30001340002B0CBF00230123DBB240E17B6863
:103C40001B681A4646F25803C4F202039A4240F235
:103C50009C804FF4C043C4F202035B681A467B6841
:103C6000196846F21003C4F20203994200F0828000
:103C70007B68196846F21043C4F20203994274D07B
:103C80007B68196846F27003C4F20203994267D058
:103C90007B68196846F27043C4F2020399425AD015
:103CA0007B68196846F22803C4F2020399424FD098
:103CB0007B68196846F22843C4F20203994244D053
:103CC0007B68196846F28803C4F20203994239D02E
:103CD0007B68196846F28843C4F2020399422ED0E9
:103CE0007B68196846F24003C4F20203994223D06C
:103CF0007B68196846F24043C4F20203994218D027
:103D00007B68196846F2A003C4F2020399420DD001
:103D10007B68196846F2A043C4F20203994202D1BB
:103D20004FF4803301E04FF4800301E04FF480331F
:103D300001E04FF4803301E04FF4803301E04FF0B5
:103D4000400301E04FF0400301E04FF0400301E089
:103D50004FF0400303E04FF00103C0F2800303E0A3
:103D60004FF00103C0F2800303E04FF00103C0F203
:103D7000800303E04FF00103C0F280031340002BE7
:103D80000CBF00230123DBB29AE04FF4C043C4F21E
:103D900002031B681A467B68196846F21003C4F2D6
:103DA0000203994200F082807B68196846F2104352
:103DB000C4F20203994274D07B68196846F270031A
:103DC000C4F20203994267D07B68196846F27043D7
:103DD000C4F2020399425AD07B68196846F228035C
:103DE000C4F2020399424FD07B68196846F2284317
:103DF000C4F20203994244D07B68196846F28803F2
:103E0000C4F20203994239D07B68196846F28843AC
:103E1000C4F2020399422ED07B68196846F240032F
:103E2000C4F20203994223D07B68196846F24043EA
:103E3000C4F20203994218D07B68196846F2A003C5
:103E4000C4F2020399420DD07B68196846F2A04380
:103E5000C4F20203994202D14FF4803301E04FF4DF
:103E6000800301E04FF4803301E04FF4803301E040
:103E70004FF4803301E04FF0400301E04FF0400386
:103E800001E04FF0400301E04FF0400303E04FF04A
:103E90000103C0F2800303E04FF00103C0F280038E
:103EA00003E04FF00103C0F2800303E04FF0010391
:103EB000C0F280031340002B0CBF00230123DBB2B0
:103EC000002B00F0B5827B681B685B6903F0800300
:103ED000002B00F0AD827B681B687A68126852691B
:103EE00022F080025A617B681B681A4646F25843EA
:103EF000C4F202039A4240F29C804FF4C842C4F2DA
:103F000002024FF4C843C4F20203DB6819467B681F
:103F1000186846F21003C4F20203984200F082804F
:103F20007B68186846F21043C4F20203984274D0CA
:103F30007B68186846F27003C4F20203984267D0A7
:103F40007B68186846F27043C4F2020398425AD064
:103F50007B68186846F22803C4F2020398424FD0E7
:103F60007B68186846F22843C4F20203984244D0A2
:103F70007B68186846F28803C4F20203984239D07D
:103F80007B68186846F28843C4F2020398422ED038
:103F90007B68186846F24003C4F20203984223D0BB
:103FA0007B68186846F24043C4F20203984218D076
:103FB0007B68186846F2A003C4F2020398420DD051
:103FC0007B68186846F2A043C4F20203984202D10B
:103FD0004FF4803301E04FF4800301E04FF480336D
:103FE00001E04FF4803301E04FF4803301E04FF003
:103FF000400301E04FF0400301E04FF0400301E0D7
:104000004FF0400303E04FF00103C0F2800303E0F0
:104010004FF00103C0F2800303E04FF00103C0F250
:10402000800303E04FF00103C0F280030B43D36031
:10403000E6E17B681B681A4646F2B803C4F2020345
:104040009A4240F29C804FF4C842C4F202024FF4FC
:10405000C843C4F202039B6819467B68186846F29D
:104060001003C4F20203984200F082807B68186853
:1040700046F21043C4F20203984274D07B68186879
:1040800046F27003C4F20203984267D07B68186856
:1040900046F27043C4F2020398425AD07B68186813
:1040A00046F22803C4F2020398424FD07B68186896
:1040B00046F22843C4F20203984244D07B68186851
:1040C00046F28803C4F20203984239D07B6818682C
:1040D00046F28843C4F2020398422ED07B681868E7
:1040E00046F24003C4F20203984223D07B6818686A
:1040F00046F24043C4F20203984218D07B68186825
:1041000046F2A003C4F2020398420DD07B681868FF
:1041100046F2A043C4F20203984202D14FF4803326
:1041200001E04FF4800301E04FF4803301E04FF4ED
:10413000803301E04FF4803301E04FF0400301E0B1
:104140004FF0400301E04FF0400301E04FF0400327
:1041500003E04FF00103C0F2800303E04FF00103DE
:10416000C0F2800303E04FF00103C0F2800303E0DC
:104170004FF00103C0F280030B43936040E17B6882
:104180001B681A4646F25803C4F202039A4240F2F0
:104190009C804FF4C042C4F202024FF4C043C4F208
:1041A0000203DB6819467B68186846F21003C4F204
:1041B0000203984200F082807B68186846F2104340
:1041C000C4F20203984274D07B68186846F2700308
:1041D000C4F20203984267D07B68186846F27043C5
:1041E000C4F2020398425AD07B68186846F228034A
:1041F000C4F2020398424FD07B68186846F2284305
:10420000C4F20203984244D07B68186846F28803DF
:10421000C4F20203984239D07B68186846F288439A
:10422000C4F2020398422ED07B68186846F240031D
:10423000C4F20203984223D07B68186846F24043D8
:10424000C4F20203984218D07B68186846F2A003B3
:10425000C4F2020398420DD07B68186846F2A0436E
:10426000C4F20203984202D14FF4803301E04FF4CC
:10427000800301E04FF4803301E04FF4803301E02C
:104280004FF4803301E04FF0400301E04FF0400372
:1042900001E04FF0400301E04FF0400303E04FF036
:1042A0000103C0F2800303E04FF00103C0F280037A
:1042B00003E04FF00103C0F2800303E04FF001037D
:1042C000C0F280030B43D3609AE04FF4C042C4F2C3
:1042D00002024FF4C043C4F202039B6819467B6894
:1042E000186846F21003C4F20203984200F082807C
:1042F0007B68186846F21043C4F20203984274D0F7
:104300007B68186846F27003C4F20203984267D0D3
:104310007B68186846F27043C4F2020398425AD090
:104320007B68186846F22803C4F2020398424FD013
:104330007B68186846F22843C4F20203984244D0CE
:104340007B68186846F28803C4F20203984239D0A9
:104350007B68186846F28843C4F2020398422ED064
:104360007B68186846F24003C4F20203984223D0E7
:104370007B68186846F24043C4F20203984218D0A2
:104380007B68186846F2A003C4F2020398420DD07D
:104390007B68186846F2A043C4F20203984202D137
:1043A0004FF4803301E04FF4800301E04FF4803399
:1043B00001E04FF4803301E04FF4803301E04FF02F
:1043C000400301E04FF0400301E04FF0400301E003
:1043D0004FF0400303E04FF00103C0F2800303E01D
:1043E0004FF00103C0F2800303E04FF00103C0F27D
:1043F000800303E04FF00103C0F280030B4393609E
:104400007B68DB6C43F002027B68DA647B684FF008
:10441000040283F835207B684FF0000283F83420D3
:104420007B689B6C002B03D07B689B6C78689847FB
:104430007B681B681A4646F25843C4F202039A424C
:1044400040F29C804FF4C843C4F202035B681A46F2
:104450007B68196846F21003C4F20203994200F027
:1044600082807B68196846F21043C4F202039942C5
:1044700074D07B68196846F27003C4F20203994253
:1044800067D07B68196846F27043C4F20203994210
:104490005AD07B68196846F22803C4F20203994295
:1044A0004FD07B68196846F22843C4F20203994250
:1044B00044D07B68196846F28803C4F2020399422B
:1044C00039D07B68196846F28843C4F202039942E6
:1044D0002ED07B68196846F24003C4F20203994269
:1044E00023D07B68196846F24043C4F20203994224
:1044F00018D07B68196846F2A003C4F202039942FF
:104500000DD07B68196846F2A043C4F202039942B9
:1045100002D14FF4802301E04FF0807301E04FF4AB
:10452000802301E04FF4802301E04FF4802301E079
:104530004FF4807301E04FF4807301E04FF4807317
:1045400001E04FF4807303E04FF00403C0F28003F6
:1045500003E04FF00403C0F2800303E04FF00403D4
:10456000C0F2800303E04FF00403C0F28003134065
:10457000002B0CBF00230123DBB2E6E17B681B6844
:104580001A4646F2B803C4F202039A4240F29C80F3
:104590004FF4C843C4F202031B681A467B681968CB
:1045A00046F21003C4F20203994200F082807B6855
:1045B000196846F21043C4F20203994274D07B6832
:1045C000196846F27003C4F20203994267D07B680F
:1045D000196846F27043C4F2020399425AD07B68CC
:1045E000196846F22803C4F2020399424FD07B684F
:1045F000196846F22843C4F20203994244D07B680A
:10460000196846F28803C4F20203994239D07B68E4
:10461000196846F28843C4F2020399422ED07B689F
:10462000196846F24003C4F20203994223D07B6822
:10463000196846F24043C4F20203994218D07B68DD
:10464000196846F2A003C4F2020399420DD07B68B8
:10465000196846F2A043C4F20203994202D14FF412
:10466000802301E04FF0807301E04FF4802301E0EC
:104670004FF4802301E04FF4802301E04FF4807376
:1046800001E04FF4807301E04FF4807301E04FF4D8
:10469000807303E04FF00403C0F2800303E04FF0A7
:1046A0000403C0F2800303E04FF00403C0F2800370
:1046B00003E04FF00403C0F280031340002B0CBF53
:1046C00000230123DBB240E17B681B681A4646F2F7
:1046D0005803C4F202039A4240F29C804FF4C04354
:1046E000C4F202035B681A467B68196846F210033D
:1046F000C4F20203994200F082807B68196846F296
:104700001043C4F20203994274D07B68196846F2E0
:104710007003C4F20203994267D07B68196846F2BD
:104720007043C4F2020399425AD07B68196846F27A
:104730002803C4F2020399424FD07B68196846F2FD
:104740002843C4F20203994244D07B68196846F2B8
:104750008803C4F20203994239D07B68196846F293
:104760008843C4F2020399422ED07B68196846F24E
:104770004003C4F20203994223D07B68196846F2D1
:104780004043C4F20203994218D07B68196846F28C
:10479000A003C4F2020399420DD07B68196846F267
:1047A000A043C4F20203994202D14FF4802301E0F6
:1047B0004FF0807301E04FF4802301E04FF4802339
:1047C00001E04FF4802301E04FF4807301E04FF4E7
:1047D000807301E04FF4807301E04FF4807303E0D5
:1047E0004FF00403C0F2800303E04FF00403C0F273
:1047F000800303E04FF00403C0F2800303E04FF0B6
:104800000403C0F280031340002B0CBF00230123DC
:10481000DBB29AE04FF4C043C4F202031B681A46AD
:104820007B68196846F21003C4F20203994200F053
:1048300082807B68196846F21043C4F202039942F1
:1048400074D07B68196846F27003C4F2020399427F
:1048500067D07B68196846F27043C4F2020399423C
:104860005AD07B68196846F22803C4F202039942C1
:104870004FD07B68196846F22843C4F2020399427C
:1048800044D07B68196846F28803C4F20203994257
:1048900039D07B68196846F28843C4F20203994212
:1048A0002ED07B68196846F24003C4F20203994295
:1048B00023D07B68196846F24043C4F20203994250
:1048C00018D07B68196846F2A003C4F2020399422B
:1048D0000DD07B68196846F2A043C4F202039942E6
:1048E00002D14FF4802301E04FF0807301E04FF4D8
:1048F000802301E04FF4802301E04FF4802301E0A6
:104900004FF4807301E04FF4807301E04FF4807343
:1049100001E04FF4807303E04FF00403C0F2800322
:1049200003E04FF00403C0F2800303E04FF0040300
:10493000C0F2800303E04FF00403C0F28003134091
:10494000002B0CBF00230123DBB2002B00F0B5824B
:104950007B681B681B6803F00203002B00F0AD822C
:104960007B681B687A681268126822F002021A607B
:104970007B681B681A4646F25843C4F202039A4207
:1049800040F29C804FF4C842C4F202024FF4C84384
:10499000C4F20203DB6819467B68186846F210030C
:1049A000C4F20203984200F082807B68186846F2E5
:1049B0001043C4F20203984274D07B68186846F230
:1049C0007003C4F20203984267D07B68186846F20D
:1049D0007043C4F2020398425AD07B68186846F2CA
:1049E0002803C4F2020398424FD07B68186846F24D
:1049F0002843C4F20203984244D07B68186846F208
:104A00008803C4F20203984239D07B68186846F2E2
:104A10008843C4F2020398422ED07B68186846F29D
:104A20004003C4F20203984223D07B68186846F220
:104A30004043C4F20203984218D07B68186846F2DB
:104A4000A003C4F2020398420DD07B68186846F2B6
:104A5000A043C4F20203984202D14FF4802301E044
:104A60004FF0807301E04FF4802301E04FF4802386
:104A700001E04FF4802301E04FF4807301E04FF434
:104A8000807301E04FF4807301E04FF4807303E022
:104A90004FF00403C0F2800303E04FF00403C0F2C0
:104AA000800303E04FF00403C0F2800303E04FF003
:104AB0000403C0F280030B43D360E6E17B681B680C
:104AC0001A4646F2B803C4F202039A4240F29C80AE
:104AD0004FF4C842C4F202024FF4C843C4F20203C6
:104AE0009B6819467B68186846F21003C4F20203FB
:104AF000984200F082807B68186846F21043C4F246
:104B00000203984274D07B68186846F27003C4F2BE
:104B10000203984267D07B68186846F27043C4F27B
:104B2000020398425AD07B68186846F22803C4F200
:104B3000020398424FD07B68186846F22843C4F2BB
:104B40000203984244D07B68186846F28803C4F296
:104B50000203984239D07B68186846F28843C4F251
:104B6000020398422ED07B68186846F24003C4F2D4
:104B70000203984223D07B68186846F24043C4F28F
:104B80000203984218D07B68186846F2A003C4F26A
:104B9000020398420DD07B68186846F2A043C4F225
:104BA0000203984202D14FF4802301E04FF080735A
:104BB00001E04FF4802301E04FF4802301E04FF443
:104BC000802301E04FF4807301E04FF4807301E033
:104BD0004FF4807301E04FF4807303E04FF004035F
:104BE000C0F2800303E04FF00403C0F2800303E04F
:104BF0004FF00403C0F2800303E04FF00403C0F25F
:104C000080030B43936040E17B681B681A4646F2C1
:104C10005803C4F202039A4240F29C804FF4C0420F
:104C2000C4F202024FF4C043C4F20203DB68194627
:104C30007B68186846F21003C4F20203984200F041
:104C400082807B68186846F21043C4F202039842DF
:104C500074D07B68186846F27003C4F2020398426D
:104C600067D07B68186846F27043C4F2020398422A
:104C70005AD07B68186846F22803C4F202039842AF
:104C80004FD07B68186846F22843C4F2020398426A
:104C900044D07B68186846F28803C4F20203984245
:104CA00039D07B68186846F28843C4F20203984200
:104CB0002ED07B68186846F24003C4F20203984283
:104CC00023D07B68186846F24043C4F2020398423E
:104CD00018D07B68186846F2A003C4F20203984219
:104CE0000DD07B68186846F2A043C4F202039842D4
:104CF00002D14FF4802301E04FF0807301E04FF4C4
:104D0000802301E04FF4802301E04FF4802301E091
:104D10004FF4807301E04FF4807301E04FF480732F
:104D200001E04FF4807303E04FF00403C0F280030E
:104D300003E04FF00403C0F2800303E04FF00403EC
:104D4000C0F2800303E04FF00403C0F280030B4382
:104D5000D3609AE04FF4C042C4F202024FF4C04361
:104D6000C4F202039B6819467B68186846F2100378
:104D7000C4F20203984200F082807B68186846F211
:104D80001043C4F20203984274D07B68186846F25C
:104D90007003C4F20203984267D07B68186846F239
:104DA0007043C4F2020398425AD07B68186846F2F6
:104DB0002803C4F2020398424FD07B68186846F279
:104DC0002843C4F20203984244D07B68186846F234
:104DD0008803C4F20203984239D07B68186846F20F
:104DE0008843C4F2020398422ED07B68186846F2CA
:104DF0004003C4F20203984223D07B68186846F24D
:104E00004043C4F20203984218D07B68186846F207
:104E1000A003C4F2020398420DD07B68186846F2E2
:104E2000A043C4F20203984202D14FF4802301E070
:104E30004FF0807301E04FF4802301E04FF48023B2
:104E400001E04FF4802301E04FF4807301E04FF460
:104E5000807301E04FF4807301E04FF4807303E04E
:104E60004FF00403C0F2800303E04FF00403C0F2EC
:104E7000800303E04FF00403C0F2800303E04FF02F
:104E80000403C0F280030B4393607B68DB6C43F048
:104E900004027B68DA647B684FF0040283F83520F3
:104EA0007B684FF0000283F834207B689B6C002BFA
:104EB00003D07B689B6C786898477B681B681A46B0
:104EC00046F25843C4F202039A4240F293804FF4F0
:104ED000C843C4F202035B681A467B68196846F24D
:104EE0001003C4F2020399427BD07B68196846F232
:104EF0001043C4F20203994270D07B68196846F2ED
:104F00007003C4F20203994265D07B68196846F2C7
:104F10007043C4F2020399425AD07B68196846F282
:104F20002803C4F2020399424FD07B68196846F205
:104F30002843C4F20203994244D07B68196846F2C0
:104F40008803C4F20203994239D07B68196846F29B
:104F50008843C4F2020399422ED07B68196846F256
:104F60004003C4F20203994223D07B68196846F2D9
:104F70004043C4F20203994218D07B68196846F294
:104F8000A003C4F2020399420DD07B68196846F26F
:104F9000A043C4F20203994202D14FF4801301E00E
:104FA0004FF0806301E04FF4801301E04FF4801371
:104FB00001E04FF4801301E04FF4806301E04FF40F
:104FC000806301E04FF4806301E04FF4806301E00F
:104FD0004FF0100301E04FF0100301E04FF0100319
:104FE00001E04FF010031340002B0CBF00230123FE
:104FF000DBB2CBE17B681B681A4646F2B803C4F209
:1050000002039A4240F293804FF4C843C4F2020371
:105010001B681A467B68196846F21003C4F2020343
:1050200099427BD07B68196846F21043C4F20203B0
:10503000994270D07B68196846F27003C4F202038B
:10504000994265D07B68196846F27043C4F2020346
:1050500099425AD07B68196846F22803C4F20203C9
:1050600099424FD07B68196846F22843C4F2020384
:10507000994244D07B68196846F28803C4F202035F
:10508000994239D07B68196846F28843C4F202031A
:1050900099422ED07B68196846F24003C4F202039D
:1050A000994223D07B68196846F24043C4F2020358
:1050B000994218D07B68196846F2A003C4F2020333
:1050C00099420DD07B68196846F2A043C4F20203EE
:1050D000994202D14FF4801301E04FF0806301E068
:1050E0004FF4801301E04FF4801301E04FF480137C
:1050F00001E04FF4806301E04FF4806301E04FF47E
:10510000806301E04FF4806301E04FF0100301E0A1
:105110004FF0100301E04FF0100301E04FF01003D7
:105120001340002B0CBF00230123DBB22EE17B6870
:105130001B681A4646F25803C4F202039A4240F230
:1051400093804FF4C043C4F202035B681A467B6845
:10515000196846F21003C4F2020399427BD07B68BF
:10516000196846F21043C4F20203994270D07B687A
:10517000196846F27003C4F20203994265D07B6855
:10518000196846F27043C4F2020399425AD07B6810
:10519000196846F22803C4F2020399424FD07B6893
:1051A000196846F22843C4F20203994244D07B684E
:1051B000196846F28803C4F20203994239D07B6829
:1051C000196846F28843C4F2020399422ED07B68E4
:1051D000196846F24003C4F20203994223D07B6867
:1051E000196846F24043C4F20203994218D07B6822
:1051F000196846F2A003C4F2020399420DD07B68FD
:10520000196846F2A043C4F20203994202D14FF456
:10521000801301E04FF0806301E04FF4801301E060
:105220004FF4801301E04FF4801301E04FF48063EA
:1052300001E04FF4806301E04FF4806301E04FF43C
:10524000806301E04FF0100301E04FF0100301E034
:105250004FF0100301E04FF010031340002B0CBF80
:1052600000230123DBB291E04FF4C043C4F20203F8
:105270001B681A467B68196846F21003C4F20203E1
:1052800099427BD07B68196846F21043C4F202034E
:10529000994270D07B68196846F27003C4F2020329
:1052A000994265D07B68196846F27043C4F20203E4
:1052B00099425AD07B68196846F22803C4F2020367
:1052C00099424FD07B68196846F22843C4F2020322
:1052D000994244D07B68196846F28803C4F20203FD
:1052E000994239D07B68196846F28843C4F20203B8
:1052F00099422ED07B68196846F24003C4F202033B
:10530000994223D07B68196846F24043C4F20203F5
:10531000994218D07B68196846F2A003C4F20203D0
:1053200099420DD07B68196846F2A043C4F202038B
:10533000994202D14FF4801301E04FF0806301E005
:105340004FF4801301E04FF4801301E04FF4801319
:1053500001E04FF4806301E04FF4806301E04FF41B
:10536000806301E04FF4806301E04FF0100301E03F
:105370004FF0100301E04FF0100301E04FF0100375
:105380001340002B0CBF00230123DBB2002B00F0E5
:1053900019857B681B681B6803F00803002B00F06D
:1053A00011857B681B681B6803F48023002B00F0C9
:1053B00084827B681B681A4646F25843C4F2020393
:1053C0009A4240F293804FF4C843C4F202034FF470
:1053D000C842C4F20202D26811467A68106846F2E6
:1053E0001002C4F2020290427BD07A68106846F242
:1053F0001042C4F20202904270D07A68106846F2FD
:105400007002C4F20202904265D07A68106846F2D7
:105410007042C4F2020290425AD07A68106846F292
:105420002802C4F2020290424FD07A68106846F215
:105430002842C4F20202904244D07A68106846F2D0
:105440008802C4F20202904239D07A68106846F2AB
:105450008842C4F2020290422ED07A68106846F266
:105460004002C4F20202904223D07A68106846F2E9
:105470004042C4F20202904218D07A68106846F2A4
:10548000A002C4F2020290420DD07A68106846F27F
:10549000A042C4F20202904202D14FF4801201E015
:1054A0004FF0806201E04FF4801201E04FF480126F
:1054B00001E04FF4801201E04FF4806201E04FF40C
:1054C000806201E04FF4806201E04FF4806201E00D
:1054D0004FF0100201E04FF0100201E04FF0100217
:1054E00001E04FF010020A43DA60CBE17B681B68F1
:1054F0001A4646F2B803C4F202039A4240F293807D
:105500004FF4C843C4F202034FF4C842C4F202028B
:10551000926811467A68106846F21002C4F20202DC
:1055200090427BD07A68106846F21042C4F20202C0
:10553000904270D07A68106846F27002C4F202029B
:10554000904265D07A68106846F27042C4F2020256
:1055500090425AD07A68106846F22802C4F20202D9
:1055600090424FD07A68106846F22842C4F2020294
:10557000904244D07A68106846F28802C4F202026F
:10558000904239D07A68106846F28842C4F202022A
:1055900090422ED07A68106846F24002C4F20202AD
:1055A000904223D07A68106846F24042C4F2020268
:1055B000904218D07A68106846F2A002C4F2020243
:1055C00090420DD07A68106846F2A042C4F20202FE
:1055D000904202D14FF4801201E04FF0806201E06E
:1055E0004FF4801201E04FF4801201E04FF480127A
:1055F00001E04FF4806201E04FF4806201E04FF47B
:10560000806201E04FF4806201E04FF0100201E09F
:105610004FF0100201E04FF0100201E04FF01002D5
:105620000A439A602EE17B681B681A4646F25803CB
:10563000C4F202039A4240F293804FF4C043C4F292
:1056400002034FF4C042C4F20202D26811467A68E3
:10565000106846F21002C4F2020290427BD07A68CF
:10566000106846F21042C4F20202904270D07A688A
:10567000106846F27002C4F20202904265D07A6865
:10568000106846F27042C4F2020290425AD07A6820
:10569000106846F22802C4F2020290424FD07A68A3
:1056A000106846F22842C4F20202904244D07A685E
:1056B000106846F28802C4F20202904239D07A6839
:1056C000106846F28842C4F2020290422ED07A68F4
:1056D000106846F24002C4F20202904223D07A6877
:1056E000106846F24042C4F20202904218D07A6832
:1056F000106846F2A002C4F2020290420DD07A680D
:10570000106846F2A042C4F20202904202D14FF465
:10571000801201E04FF0806201E04FF4801201E05E
:105720004FF4801201E04FF4801201E04FF48062E8
:1057300001E04FF4806201E04FF4806201E04FF439
:10574000806201E04FF0100201E04FF0100201E032
:105750004FF0100201E04FF010020A43DA6091E0CE
:105760004FF4C043C4F202034FF4C042C4F2020239
:10577000926811467A68106846F21002C4F202027A
:1057800090427BD07A68106846F21042C4F202025E
:10579000904270D07A68106846F27002C4F2020239
:1057A000904265D07A68106846F27042C4F20202F4
:1057B00090425AD07A68106846F22802C4F2020277
:1057C00090424FD07A68106846F22842C4F2020232
:1057D000904244D07A68106846F28802C4F202020D
:1057E000904239D07A68106846F28842C4F20202C8
:1057F00090422ED07A68106846F24002C4F202024B
:10580000904223D07A68106846F24042C4F2020205
:10581000904218D07A68106846F2A002C4F20202E0
:1058200090420DD07A68106846F2A042C4F202029B
:10583000904202D14FF4801201E04FF0806201E00B
:105840004FF4801201E04FF4801201E04FF4801217
:1058500001E04FF4806201E04FF4806201E04FF418
:10586000806201E04FF4806201E04FF0100201E03D
:105870004FF0100201E04FF0100201E04FF0100273
:105880000A439A607B681B681B6803F40023002BA3
:1058900005D17B684FF0310283F835208AE27B68BE
:1058A0001B681B6803F40023002B00F083827B68D5
:1058B0004FF0410283F835207CE27B681B681B684F
:1058C00003F48073002B07D17B681B687A68126829
:1058D000126822F008021A607B681B681A4646F2BA
:1058E0005843C4F202039A4240F293804FF4C843F3
:1058F000C4F202034FF4C842C4F20202D268114655
:105900007A68106846F21002C4F2020290427BD01C
:105910007A68106846F21042C4F20202904270D0D7
:105920007A68106846F27002C4F20202904265D0B2
:105930007A68106846F27042C4F2020290425AD06D
:105940007A68106846F22802C4F2020290424FD0F0
:105950007A68106846F22842C4F20202904244D0AB
:105960007A68106846F28802C4F20202904239D086
:105970007A68106846F28842C4F2020290422ED041
:105980007A68106846F24002C4F20202904223D0C4
:105990007A68106846F24042C4F20202904218D07F
:1059A0007A68106846F2A002C4F2020290420DD05A
:1059B0007A68106846F2A042C4F20202904202D114
:1059C0004FF4801201E04FF0806201E04FF480124A
:1059D00001E04FF4801201E04FF4801201E04FF437
:1059E000806201E04FF4806201E04FF4806201E0E8
:1059F0004FF4806201E04FF0100201E04FF010021E
:105A000001E04FF0100201E04FF010020A43DA60AB
:105A1000CBE17B681B681A4646F2B803C4F2020366
:105A20009A4240F293804FF4C843C4F202034FF409
:105A3000C842C4F20202926811467A68106846F2BF
:105A40001002C4F2020290427BD07A68106846F2DB
:105A50001042C4F20202904270D07A68106846F296
:105A60007002C4F20202904265D07A68106846F271
:105A70007042C4F2020290425AD07A68106846F22C
:105A80002802C4F2020290424FD07A68106846F2AF
:105A90002842C4F20202904244D07A68106846F26A
:105AA0008802C4F20202904239D07A68106846F245
:105AB0008842C4F2020290422ED07A68106846F200
:105AC0004002C4F20202904223D07A68106846F283
:105AD0004042C4F20202904218D07A68106846F23E
:105AE000A002C4F2020290420DD07A68106846F219
:105AF000A042C4F20202904202D14FF4801201E0AF
:105B00004FF0806201E04FF4801201E04FF4801208
:105B100001E04FF4801201E04FF4806201E04FF4A5
:105B2000806201E04FF4806201E04FF4806201E0A6
:105B30004FF0100201E04FF0100201E04FF01002B0
:105B400001E04FF010020A439A602EE17B681B6867
:105B50001A4646F25803C4F202039A4240F2938076
:105B60004FF4C043C4F202034FF4C042C4F2020235
:105B7000D26811467A68106846F21002C4F2020236
:105B800090427BD07A68106846F21042C4F202025A
:105B9000904270D07A68106846F27002C4F2020235
:105BA000904265D07A68106846F27042C4F20202F0
:105BB00090425AD07A68106846F22802C4F2020273
:105BC00090424FD07A68106846F22842C4F202022E
:105BD000904244D07A68106846F28802C4F2020209
:105BE000904239D07A68106846F28842C4F20202C4
:105BF00090422ED07A68106846F24002C4F2020247
:105C0000904223D07A68106846F24042C4F2020201
:105C1000904218D07A68106846F2A002C4F20202DC
:105C200090420DD07A68106846F2A042C4F2020297
:105C3000904202D14FF4801201E04FF0806201E007
:105C40004FF4801201E04FF4801201E04FF4801213
:105C500001E04FF4806201E04FF4806201E04FF414
:105C6000806201E04FF4806201E04FF0100201E039
:105C70004FF0100201E04FF0100201E04FF010026F
:105C80000A43DA6091E04FF4C043C4F202034FF4D8
:105C9000C042C4F20202926811467A68106846F265
:105CA0001002C4F2020290427BD07A68106846F279
:105CB0001042C4F20202904270D07A68106846F234
:105CC0007002C4F20202904265D07A68106846F20F
:105CD0007042C4F2020290425AD07A68106846F2CA
:105CE0002802C4F2020290424FD07A68106846F24D
:105CF0002842C4F20202904244D07A68106846F208
:105D00008802C4F20202904239D07A68106846F2E2
:105D10008842C4F2020290422ED07A68106846F29D
:105D20004002C4F20202904223D07A68106846F220
:105D30004042C4F20202904218D07A68106846F2DB
:105D4000A002C4F2020290420DD07A68106846F2B6
:105D5000A042C4F20202904202D14FF4801201E04C
:105D60004FF0806201E04FF4801201E04FF48012A6
:105D700001E04FF4801201E04FF4806201E04FF443
:105D8000806201E04FF4806201E04FF4806201E044
:105D90004FF0100201E04FF0100201E04FF010024E
:105DA00001E04FF010020A439A607B684FF0310225
:105DB00083F835207B681B6C002B03D07B681B6C41
:105DC000786898477B681B681A4646F25843C4F2C5
:105DD00002039A4240F293804FF4C843C4F2020394
:105DE0005B681A467B68196846F21003C4F2020326
:105DF00099427BD07B68196846F21043C4F20203D3
:105E0000994270D07B68196846F27003C4F20203AD
:105E1000994265D07B68196846F27043C4F2020368
:105E200099425AD07B68196846F22803C4F20203EB
:105E300099424FD07B68196846F22843C4F20203A6
:105E4000994244D07B68196846F28803C4F2020381
:105E5000994239D07B68196846F28843C4F202033C
:105E600099422ED07B68196846F24003C4F20203BF
:105E7000994223D07B68196846F24043C4F202037A
:105E8000994218D07B68196846F2A003C4F2020355
:105E900099420DD07B68196846F2A043C4F2020310
:105EA000994202D14FF4001301E04FF0006301E08A
:105EB0004FF4001301E04FF4001301E04FF400131E
:105EC00001E04FF4006301E04FF4006301E04FF4A0
:105ED000006301E04FF4006301E04FF0200301E0B4
:105EE0004FF0200301E04FF0200301E04FF02003CA
:105EF0001340002B0CBF00230123DBB2CBE17B68F6
:105F00001B681A4646F2B803C4F202039A4240F2F2
:105F100093804FF4C843C4F202031B681A467B689F
:105F2000196846F21003C4F2020399427BD07B68E1
:105F3000196846F21043C4F20203994270D07B689C
:105F4000196846F27003C4F20203994265D07B6877
:105F5000196846F27043C4F2020399425AD07B6832
:105F6000196846F22803C4F2020399424FD07B68B5
:105F7000196846F22843C4F20203994244D07B6870
:105F8000196846F28803C4F20203994239D07B684B
:105F9000196846F28843C4F2020399422ED07B6806
:105FA000196846F24003C4F20203994223D07B6889
:105FB000196846F24043C4F20203994218D07B6844
:105FC000196846F2A003C4F2020399420DD07B681F
:105FD000196846F2A043C4F20203994202D14FF479
:105FE000001301E04FF0006301E04FF4001301E003
:105FF0004FF4001301E04FF4001301E04FF400638D
:1060000001E04FF4006301E04FF4006301E04FF45E
:10601000006301E04FF0200301E04FF0200301E0B6
:106020004FF0200301E04FF020031340002B0CBF82
:1060300000230123DBB22EE17B681B681A4646F27F
:106040005803C4F202039A4240F293804FF4C043D3
:10605000C4F202035B681A467B68196846F21003B3
:10606000C4F2020399427BD07B68196846F2104360
:10607000C4F20203994270D07B68196846F270033B
:10608000C4F20203994265D07B68196846F27043F6
:10609000C4F2020399425AD07B68196846F2280379
:1060A000C4F2020399424FD07B68196846F2284334
:1060B000C4F20203994244D07B68196846F288030F
:1060C000C4F20203994239D07B68196846F28843CA
:1060D000C4F2020399422ED07B68196846F240034D
:1060E000C4F20203994223D07B68196846F2404308
:1060F000C4F20203994218D07B68196846F2A003E3
:10610000C4F2020399420DD07B68196846F2A0439D
:10611000C4F20203994202D14FF4001301E04FF0A0
:10612000006301E04FF4001301E04FF4001301E0BD
:106130004FF4001301E04FF4006301E04FF40063FB
:1061400001E04FF4006301E04FF4006301E04FF021
:10615000200301E04FF0200301E04FF0200301E0B5
:106160004FF020031340002B0CBF00230123DBB2B0
:1061700091E04FF4C043C4F202031B681A467B68E7
:10618000196846F21003C4F2020399427BD07B687F
:10619000196846F21043C4F20203994270D07B683A
:1061A000196846F27003C4F20203994265D07B6815
:1061B000196846F27043C4F2020399425AD07B68D0
:1061C000196846F22803C4F2020399424FD07B6853
:1061D000196846F22843C4F20203994244D07B680E
:1061E000196846F28803C4F20203994239D07B68E9
:1061F000196846F28843C4F2020399422ED07B68A4
:10620000196846F24003C4F20203994223D07B6826
:10621000196846F24043C4F20203994218D07B68E1
:10622000196846F2A003C4F2020399420DD07B68BC
:10623000196846F2A043C4F20203994202D14FF416
:10624000001301E04FF0006301E04FF4001301E0A0
:106250004FF4001301E04FF4001301E04FF400632A
:1062600001E04FF4006301E04FF4006301E04FF4FC
:10627000006301E04FF0200301E04FF0200301E054
:106280004FF0200301E04FF020031340002B0CBF20
:1062900000230123DBB2002B00F02B857B681B68F9
:1062A0001B6803F01003002B00F023857B681B683C
:1062B0001B6803F48023002B00F08C827B681B6832
:1062C0001A4646F25843C4F202039A4240F29380BF
:1062D0004FF4C843C4F202034FF4C842C4F20202AE
:1062E000D26811467A68106846F21002C4F20202BF
:1062F00090427BD07A68106846F21042C4F20202E3
:10630000904270D07A68106846F27002C4F20202BD
:10631000904265D07A68106846F27042C4F2020278
:1063200090425AD07A68106846F22802C4F20202FB
:1063300090424FD07A68106846F22842C4F20202B6
:10634000904244D07A68106846F28802C4F2020291
:10635000904239D07A68106846F28842C4F202024C
:1063600090422ED07A68106846F24002C4F20202CF
:10637000904223D07A68106846F24042C4F202028A
:10638000904218D07A68106846F2A002C4F2020265
:1063900090420DD07A68106846F2A042C4F2020220
:1063A000904202D14FF4001201E04FF0006201E090
:1063B0004FF4001201E04FF4001201E04FF400121C
:1063C00001E04FF4006201E04FF4006201E04FF49D
:1063D000006201E04FF4006201E04FF0200201E0B2
:1063E0004FF0200201E04FF0200201E04FF02002C8
:1063F0000A43DA60CBE17B681B681A4646F2B803B1
:10640000C4F202039A4240F293804FF4C843C4F2AC
:1064100002034FF4C842C4F20202926811467A683D
:10642000106846F21002C4F2020290427BD07A68F1
:10643000106846F21042C4F20202904270D07A68AC
:10644000106846F27002C4F20202904265D07A6887
:10645000106846F27042C4F2020290425AD07A6842
:10646000106846F22802C4F2020290424FD07A68C5
:10647000106846F22842C4F20202904244D07A6880
:10648000106846F28802C4F20202904239D07A685B
:10649000106846F28842C4F2020290422ED07A6816
:1064A000106846F24002C4F20202904223D07A6899
:1064B000106846F24042C4F20202904218D07A6854
:1064C000106846F2A002C4F2020290420DD07A682F
:1064D000106846F2A042C4F20202904202D14FF488
:1064E000001201E04FF0006201E04FF4001201E001
:1064F0004FF4001201E04FF4001201E04FF400628B
:1065000001E04FF4006201E04FF4006201E04FF45B
:10651000006201E04FF0200201E04FF0200201E0B4
:106520004FF0200201E04FF020020A439A602EE172
:106530007B681B681A4646F25803C4F202039A426B
:1065400040F293804FF4C043C4F202034FF4C042C0
:10655000C4F20202D26811467A68106846F210024C
:10656000C4F2020290427BD07A68106846F2104270
:10657000C4F20202904270D07A68106846F270024B
:10658000C4F20202904265D07A68106846F2704206
:10659000C4F2020290425AD07A68106846F2280289
:1065A000C4F2020290424FD07A68106846F2284244
:1065B000C4F20202904244D07A68106846F288021F
:1065C000C4F20202904239D07A68106846F28842DA
:1065D000C4F2020290422ED07A68106846F240025D
:1065E000C4F20202904223D07A68106846F2404218
:1065F000C4F20202904218D07A68106846F2A002F3
:10660000C4F2020290420DD07A68106846F2A042AD
:10661000C4F20202904202D14FF4001201E04FF0A6
:10662000006201E04FF4001201E04FF4001201E0BB
:106630004FF4001201E04FF4006201E04FF40062F9
:1066400001E04FF4006201E04FF4006201E04FF01E
:10665000200201E04FF0200201E04FF0200201E0B3
:106660004FF020020A43DA6091E04FF4C043C4F2D5
:1066700002034FF4C042C4F20202926811467A68E3
:10668000106846F21002C4F2020290427BD07A688F
:10669000106846F21042C4F20202904270D07A684A
:1066A000106846F27002C4F20202904265D07A6825
:1066B000106846F27042C4F2020290425AD07A68E0
:1066C000106846F22802C4F2020290424FD07A6863
:1066D000106846F22842C4F20202904244D07A681E
:1066E000106846F28802C4F20202904239D07A68F9
:1066F000106846F28842C4F2020290422ED07A68B4
:10670000106846F24002C4F20202904223D07A6836
:10671000106846F24042C4F20202904218D07A68F1
:10672000106846F2A002C4F2020290420DD07A68CC
:10673000106846F2A042C4F20202904202D14FF425
:10674000001201E04FF0006201E04FF4001201E09E
:106750004FF4001201E04FF4001201E04FF4006228
:1067600001E04FF4006201E04FF4006201E04FF4F9
:10677000006201E04FF0200201E04FF0200201E052
:106780004FF0200201E04FF020020A439A607B683C
:106790001B681B6803F40023002B09D17B685B6C2A
:1067A000002B00F0A6827B685B6C78689847A0E2BB
:1067B0007B681B681B6803F40023002B00F09982A0
:1067C0007B68DB6B002B00F094827B68DB6B786866
:1067D00098478EE27B681B681B6803F48073002B6C
:1067E00007D17B681B687A681268126822F0100271
:1067F0001A607B681B681A4646F25843C4F20203CB
:106800009A4240F293804FF4C843C4F202034FF41B
:10681000C842C4F20202D26811467A68106846F291
:106820001002C4F2020290427BD07A68106846F2ED
:106830001042C4F20202904270D07A68106846F2A8
:106840007002C4F20202904265D07A68106846F283
:106850007042C4F2020290425AD07A68106846F23E
:106860002802C4F2020290424FD07A68106846F2C1
:106870002842C4F20202904244D07A68106846F27C
:106880008802C4F20202904239D07A68106846F257
:106890008842C4F2020290422ED07A68106846F212
:1068A0004002C4F20202904223D07A68106846F295
:1068B0004042C4F20202904218D07A68106846F250
:1068C000A002C4F2020290420DD07A68106846F22B
:1068D000A042C4F20202904202D14FF4001201E041
:1068E0004FF0006201E04FF4001201E04FF400129B
:1068F00001E04FF4001201E04FF4006201E04FF4B8
:10690000006201E04FF4006201E04FF4006201E038
:106910004FF0200201E04FF0200201E04FF0200292
:1069200001E04FF020020A43DA60CBE17B681B688C
:106930001A4646F2B803C4F202039A4240F2938028
:106940004FF4C843C4F202034FF4C842C4F2020237
:10695000926811467A68106846F21002C4F2020288
:1069600090427BD07A68106846F21042C4F202026C
:10697000904270D07A68106846F27002C4F2020247
:10698000904265D07A68106846F27042C4F2020202
:1069900090425AD07A68106846F22802C4F2020285
:1069A00090424FD07A68106846F22842C4F2020240
:1069B000904244D07A68106846F28802C4F202021B
:1069C000904239D07A68106846F28842C4F20202D6
:1069D00090422ED07A68106846F24002C4F2020259
:1069E000904223D07A68106846F24042C4F2020214
:1069F000904218D07A68106846F2A002C4F20202EF
:106A000090420DD07A68106846F2A042C4F20202A9
:106A1000904202D14FF4001201E04FF0006201E019
:106A20004FF4001201E04FF4001201E04FF40012A5
:106A300001E04FF4006201E04FF4006201E04FF426
:106A4000006201E04FF4006201E04FF0200201E03B
:106A50004FF0200201E04FF0200201E04FF0200251
:106A60000A439A602EE17B681B681A4646F2580377
:106A7000C4F202039A4240F293804FF4C043C4F23E
:106A800002034FF4C042C4F20202D26811467A688F
:106A9000106846F21002C4F2020290427BD07A687B
:106AA000106846F21042C4F20202904270D07A6836
:106AB000106846F27002C4F20202904265D07A6811
:106AC000106846F27042C4F2020290425AD07A68CC
:106AD000106846F22802C4F2020290424FD07A684F
:106AE000106846F22842C4F20202904244D07A680A
:106AF000106846F28802C4F20202904239D07A68E5
:106B0000106846F28842C4F2020290422ED07A689F
:106B1000106846F24002C4F20202904223D07A6822
:106B2000106846F24042C4F20202904218D07A68DD
:106B3000106846F2A002C4F2020290420DD07A68B8
:106B4000106846F2A042C4F20202904202D14FF411
:106B5000001201E04FF0006201E04FF4001201E08A
:106B60004FF4001201E04FF4001201E04FF4006214
:106B700001E04FF4006201E04FF4006201E04FF4E5
:106B8000006201E04FF0200201E04FF0200201E03E
:106B90004FF0200201E04FF020020A43DA6091E05A
:106BA0004FF4C043C4F202034FF4C042C4F20202E5
:106BB000926811467A68106846F21002C4F2020226
:106BC00090427BD07A68106846F21042C4F202020A
:106BD000904270D07A68106846F27002C4F20202E5
:106BE000904265D07A68106846F27042C4F20202A0
:106BF00090425AD07A68106846F22802C4F2020223
:106C000090424FD07A68106846F22842C4F20202DD
:106C1000904244D07A68106846F28802C4F20202B8
:106C2000904239D07A68106846F28842C4F2020273
:106C300090422ED07A68106846F24002C4F20202F6
:106C4000904223D07A68106846F24042C4F20202B1
:106C5000904218D07A68106846F2A002C4F202028C
:106C600090420DD07A68106846F2A042C4F2020247
:106C7000904202D14FF4001201E04FF0006201E0B7
:106C80004FF4001201E04FF4001201E04FF4001243
:106C900001E04FF4006201E04FF4006201E04FF4C4
:106CA000006201E04FF4006201E04FF0200201E0D9
:106CB0004FF0200201E04FF0200201E04FF02002EF
:106CC0000A439A607B68DB6C1A467B68DA647B68EF
:106CD0004FF0110283F835207B684FF0000283F8F3
:106CE00034207B68DB6B002B03D07B68DB6B786820
:106CF000984707F10807BD4680BD00BF80B582B048
:106D000000AF78607B68002B02D14FF0010325E0D3
:106D10007B681A684FF4E843C4F200039A4207D034
:106D200046F2AC10C0F601004FF0E80101F0B4F8F3
:106D30007B681B79DBB2002B02D1786800F014F875
:106D40007B684FF002021A717B684FF000021A61F3
:106D50007B684FF001021A714FF00003184607F1EB
:106D60000807BD4680BD00BF80B483B000AF786027
:106D700007F10C07BD4680BC704700BF80B584B0EA
:106D800000AF786039604FF00003FB604FF0000304
:106D9000BB603B68002B0AD03B68102B07D046F243
:106DA000AC10C0F6010040F26B1101F075F87B6881
:106DB0005B79012B02D14FF0020358E07B684FF062
:106DC00001025A717B684FF002021A717B681B68DE
:106DD0007A681268126811463A684FF0010000FAAA
:106DE00002F20A431A603B68002B1AD17B681B68C9
:106DF0001B6803F00403FB607B681B681B6803F0DF
:106E00003803BB60FB68042B27D1BB68382B24D127
:106E10007B681B687A681268526842F001025A6007
:106E20001BE07B681B681B6803F48023FB607B68A6
:106E30001B681B6803F46013BB60FB68B3F5802F0D
:106E40000BD1BB68B3F5601F07D17B681B687A68FC
:106E50001268526842F002025A607B684FF00102E9
:106E60001A717B684FF000025A714FF00003184608
:106E700007F11007BD4680BD80B586B000AFF86051
:106E8000B9607A604FF000037B614FF000033B6113
:106E9000BB681B68002B27D0BB681B68242B23D042
:106EA000BB681B680C2B1FD0BB681B68142B1BD046
:106EB000BB681B681C2B17D0BB681B68042B13D046
:106EC000BB681B682C2B0FD0BB681B68342B0BD006
:106ED000BB681B683C2B07D046F2AC10C0F6010023
:106EE00040F2F32100F0D8FFBB685B68002B0BD0A9
:106EF000BB685B68022B07D046F2AC10C0F60100FD
:106F00004FF43D7100F0C8FFBB681B68002B27D011
:106F1000BB681B68242B23D0BB681B680C2B1FD0BD
:106F2000BB681B68142B1BD0BB681B681C2B17D0BD
:106F3000BB681B68042B13D0BB681B682C2B0FD0BD
:106F4000BB681B68342B0BD0BB681B683C2B07D07D
:106F500046F2AC10C0F6010040F2F52100F09CFFB3
:106F60007B68002B0AD07B68102B07D046F2AC1050
:106F7000C0F6010040F2F62100F08EFFFB685B795D
:106F8000012B02D14FF0020347E0FB684FF00102F2
:106F90005A71FB684FF002021A714FF4E843C4F2D1
:106FA00000031B687B617B6840F6FE7202FA03F304
:106FB0006FEA03037A6913407B61BB681A68BB6898
:106FC0005B6813433B617B683A6902FA03F37A69B1
:106FD00013437B614FF4E843C4F200037A691A60FB
:106FE0004FF4E843C4F200034FF4E842C4F2000255
:106FF000126811467A684FF0C00000FA02F26FEA98
:1070000002020A401A60FB684FF001021A71FB6825
:107010004FF000025A714FF00003184607F11807AD
:10702000BD4680BD80B586B000AFF860B9607A60BB
:107030003B604FF000037B61BB68002B0AD0BB684C
:10704000102B07D046F2AC10C0F601004FF44B7184
:1070500000F022FF7B68002B0DD07B68042B0AD048
:107060007B68082B07D046F2AC10C0F6010040F256
:107070002D3100F011FF3A684FF6F0739A4207D9AC
:1070800046F2AC10C0F6010040F22E3100F004FFD1
:10709000FB681B687B61BB68002B06D17A697B6843
:1070A000D31803F108037B6105E07A697B68D31884
:1070B00003F114037B617B693A681A604FF00003A7
:1070C000184607F11807BD4680BD00BF80B485B0E3
:1070D00000AF78607B6803F00703FB604FF46D43FB
:1070E000CEF20003DB68BB60BA684FF6FF031340C3
:1070F000BB60FB684FEA0322BB68134343F0BE63E7
:1071000043F42023BB604FF46D43CEF20003BA6812
:10711000DA6007F11407BD4680BC704780B400AF49
:107120004FF46D43CEF20003DB6803F4E0634FEAF3
:1071300013231846BD4680BC704700BF80B483B09F
:1071400000AF0346FB714FF46143CEF2000397F9A1
:1071500007204FEA5212F97901F01F014FF00100A8
:1071600000FA01F143F8221007F10C07BD4680BC7C
:10717000704700BF80B483B000AF03463960FB7135
:1071800097F90730002B10DA4FF46D43CEF200036D
:10719000FA7902F00F02A2F104013A68D2B24FEA82
:1071A0000212D2B25B181A760DE04FF46143CEF2B0
:1071B000000397F907103A68D2B24FEA0212D2B22E
:1071C0005B1883F8002307F10C07BD4680BC7047AD
:1071D00080B489B000AFF860B9607A60FB6803F0F2
:1071E0000703FB61FB69C3F10703042B28BF0423DA
:1071F000BB61FB6903F10403062B03D9FB69A3F10F
:10720000030301E04FF000037B61BB694FF0010213
:1072100002FA03F303F1FF331A46BB681A407B6995
:1072200002FA03F27B694FF0010101FA03F303F163
:10723000FF3319467B680B401343184607F12407B8
:10724000BD4680BC704700BF80B582B000AF78609B
:107250007B6803F1FF326FF07F439A4202D94FF00F
:1072600001031DE04EF21003CEF200037A6802F132
:10727000FF325A604FF0FF304FF00F01FFF77AFFF7
:107280004EF21003CEF200034FF000029A604EF26D
:107290001003CEF200034FF007021A604FF0000314
:1072A000184607F10807BD4680BD00BF80B582B013
:1072B00000AF78607B68072B13D07B68062B10D05B
:1072C0007B68052B0DD07B68042B0AD07B68032BD1
:1072D00007D046F2DC10C0F601004FF0BA0100F012
:1072E000DBFD7868FFF7F2FE07F10807BD4680BDB9
:1072F00080B586B000AF0346B9607A60FB734FF08B
:1073000000037B617B680F2B07D946F2DC10C0F6C7
:1073100001004FF0D20100F0BFFDBB680F2B07D971
:1073200046F2DC10C0F601004FF0D30100F0B4FDCE
:10733000FFF7F4FE03467B617869B9687A68FFF766
:1073400047FF034697F90F2010461946FFF712FF33
:1073500007F11807BD4680BD80B582B000AF034677
:10736000FB7197F907301846FFF7E8FE07F10807A9
:10737000BD4680BD80B582B000AF78607868FFF709
:1073800063FF0346184607F10807BD4680BD00BFEE
:1073900080B582B000AF78607B68002B02D14FF0DF
:1073A00001035DE17B681A684FF40053C4F20103E6
:1073B0009A4217D07B681A684FF40453C4F2010351
:1073C0009A420FD07B681A684FF40853C4F2010345
:1073D0009A4207D046F21020C0F601004FF0D701C4
:1073E00000F05AFD7B685B68002B16D07B685B68F9
:1073F000B3F5803F11D07B685B68B3F5003F0CD0DC
:107400007B685B68B3F5403F07D046F21020C0F6BA
:1074100001004FF0D80100F03FFD7B689B68002B16
:1074200016D07B689B68B3F1807F11D07B689B6826
:10743000B3F1007F0CD07B689B68B3F1407F07D02D
:1074400046F21020C0F601004FF0D90100F024FDF3
:107450007B681B69002B0BD07B681B69012B07D055
:1074600046F21020C0F601004FF0DA0100F014FDE2
:107470007B689B69002B0BD07B689B69012B07D035
:1074800046F21020C0F601004FF0DB0100F004FDD1
:107490007B68DB6A002B16D07B68DB6AB3F1805F08
:1074A00011D07B68DB6AB3F1005F0CD07B68DB6ACC
:1074B000B3F1405F07D046F21020C0F601004FF054
:1074C000DC0100F0E9FC7B681B6B002B52D07B6871
:1074D0001B6BB3F1807F4DD07B681B6BB3F1007FDA
:1074E00048D07B681B6BB3F1407F43D07B681B6B3C
:1074F000B3F1806F3ED07B681B6BB3F1A06F39D0C6
:107500007B681B6BB3F1C06F34D07B681B6BB3F12E
:10751000E06F2FD07B681B6BB3F1006F2AD07B68C4
:107520001B6BB3F1106F25D07B681B6BB3F1206F21
:1075300020D07B681B6BB3F1306F1BD07B681B6B5B
:10754000B3F1406F16D07B681B6BB3F1506F11D055
:107550007B681B6BB3F1606F0CD07B681B6BB3F166
:10756000706F07D046F21020C0F601004FF0DD0129
:1075700000F092FC7B68DB68002B0CD07B68DB683A
:10758000B3F5006F07D046F21020C0F601004FF0AF
:10759000DE0100F081FC7B681B6A002B03D07B6856
:1075A0001B6A102B07D946F21020C0F601004FF0DD
:1075B000DF0100F071FC7B68DB69002B0BD07B687E
:1075C000DB69012B07D046F21020C0F601004FF016
:1075D000E00100F061FC7B685B69012B0FD07B68E8
:1075E0005B69002B0BD07B685B69022B07D046F2EE
:1075F0001020C0F601004FF0E10100F04DFC7B6867
:107600005B6A002B0BD07B685B6A012B07D046F2CC
:107610001020C0F601004FF0E20100F03DFC7B6855
:1076200093F83D30DBB2002B02D1786800F01EF8F1
:107630007B684FF0020283F83D20786800F0DAFAA8
:107640007B684FF000021A647B684FF0010283F8F8
:107650003D207B684FF0000283F83C204FF0000390
:10766000184607F10807BD4680BD00BF80B483B04F
:1076700000AF786007F10C07BD4680BC704700BFC3
:1076800080B584B000AF78604FF00003FB817B6869
:107690009B69002B0BD07B689B69012B07D046F2BE
:1076A0001020C0F601004FF4B37100F0F5FB7B68C9
:1076B000DB6A002B16D07B68DB6AB3F1805F11D0E8
:1076C0007B68DB6AB3F1005F0CD07B68DB6AB3F1E7
:1076D000405F07D046F21020C0F6010040F267116B
:1076E00000F0DAFB7B6893F83C30012B02D14FF0BD
:1076F00002035FE07B684FF0010283F83C207B6867
:1077000093F83D30DBB2222B05D17B684FF032027B
:1077100083F83D2004E07B684FF0120283F83D209F
:107720007B681B689B6803F00103002B11D17B6809
:107730001B687A681268926842F001029A6004E05D
:1077400000BFFB8903F10103FB81FB89B3F5077FD0
:10775000F6D94FF40C53C4F201035B6803F01F0326
:10776000002B0CD17B68DB6A002B1CD17B681B686B
:107770007A681268926842F080429A6013E07B68EF
:107780001A684FF40053C4F201039A420BD17B688C
:10779000DB6A002B07D17B681B687A6812689268E5
:1077A00042F080429A607B684FF0000283F83C20F0
:1077B0004FF00003184607F11007BD4680BD00BF1B
:1077C00080B584B000AF7860396000F059FB0246A4
:1077D0003B68D318FB6016E03B68B3F1FF3F12D063
:1077E00000F04EFB0246FB689A420CD37B684FF0D8
:1077F000030283F83D207B684FF0000283F83C20B1
:107800004FF0030319E07B681B681B6803F0020359
:10781000002BE1D07B6893F83D30DBB2252B05D1FE
:107820007B684FF0350283F83D2004E07B684FF021
:10783000150283F83D204FF00003184607F11007AA
:10784000BD4680BD80B483B000AF78607B681B68A4
:10785000DB6C184607F10C07BD4680BC704700BFC3
:1078600090B583B000AF786039603B681B68002B2F
:107870004FD03B681B68012B4BD03B681B68022B29
:1078800047D03B681B68032B43D03B681B68042B25
:107890003FD03B681B68052B3BD03B681B68062B21
:1078A00037D03B681B68072B33D03B681B68082B1D
:1078B0002FD03B681B68092B2BD03B681B680A2B19
:1078C00027D03B681B680B2B23D03B681B680C2B15
:1078D0001FD03B681B680D2B1BD03B681B680E2B11
:1078E00017D03B681B680F2B13D03B681B68102B0D
:1078F0000FD03B681B68112B0BD03B681B68122B09
:1079000007D046F21020C0F6010040F2DE3100F050
:10791000C3FA3B685B68002B03D03B685B68102BA5
:1079200007D946F21020C0F6010040F2DF3100F026
:10793000B3FA3B689B68002B23D03B689B68012B04
:107940001FD03B689B68022B1BD03B689B68032BB6
:1079500017D03B689B68042B13D03B689B68052BB2
:107960000FD03B689B68062B0BD03B689B68072BAE
:1079700007D046F21020C0F601004FF4787100F0F5
:107980008BFA7B6893F83C30012B02D14FF0020355
:107990001CE17B684FF0010283F83C203B681B68C8
:1079A000092B2AD97B6819687B681B68DB68184635
:1079B0003B681A6813464FEA43039B18A3F11E0362
:1079C0004FF0070202FA03F36FEA03030340CB60B0
:1079D0007B6819687B681B68DB6818463B689C6895
:1079E0003B681A6813464FEA43039B18A3F11E0332
:1079F00004FA03F30343CB6025E07B6819687B68D6
:107A00001B681B6918463B681A6813464FEA430314
:107A10009B184FF0070202FA03F36FEA03030340D7
:107A20000B617B6819687B681B681B6918463B689B
:107A30009C683B681A6813464FEA43039B1804FA94
:107A400003F303430B613B685B68062B2AD87B6812
:107A500019687B681B685B6B18463B685A6813465D
:107A60004FEA83039B18A3F105034FF01F0202FAAC
:107A700003F36FEA030303404B637B6819687B6879
:107A80001B685B6B18463B681C683B685A6813466A
:107A90004FEA83039B18A3F1050304FA03F303439E
:107AA0004B6358E03B685B680C2B2AD87B681968ED
:107AB0007B681B681B6B18463B685A6813464FEA85
:107AC00083039B18A3F123034FF01F0202FA03F371
:107AD0006FEA030303400B637B6819687B681B68CC
:107AE0001B6B18463B681C683B685A6813464FEA94
:107AF00083039B18A3F1230304FA03F303430B63EB
:107B000029E07B6819687B681B68DB6A18463B685C
:107B10005A6813464FEA83039B18A3F141034FF0C1
:107B20001F0202FA03F36FEA03030340CB627B6890
:107B300019687B681B68DB6A18463B681C683B68F1
:107B40005A6813464FEA83039B18A3F1410304FAD2
:107B500003F30343CB627B681A684FF40053C4F20B
:107B600001039A420FD13B681B68122B0BD14FF4D3
:107B70000C53C4F201034FF40C52C4F201025268D8
:107B800042F480025A607B681A684FF40053C4F2D2
:107B900001039A4213D13B681B68102B03D03B684A
:107BA0001B68112B0BD14FF40C53C4F201034FF49B
:107BB0000C52C4F20102526842F400025A607B681F
:107BC0004FF0000283F83C204FF00003184607F105
:107BD0000C07BD4690BD00BF80B483B000AF786095
:107BE0007B6893F83D30DBB2184607F10C07BD46C1
:107BF00080BC704780B582B000AF78604FF40C5302
:107C0000C4F201034FF40C52C4F20102526822F490
:107C100040325A604FF40C53C4F201034FF40C523B
:107C2000C4F20102526811467A6852680A435A60E7
:107C30007B681B687A681268526822F480725A6006
:107C40007B681B687A681268526811467A68126904
:107C50004FEA02220A435A607B681B687A681268FE
:107C6000526822F040725A607B681B687A6812681A
:107C7000526811467A6892680A435A607B681B68AA
:107C80007A681268926822F400629A607B681B68C6
:107C90007A681268926811467A68D2680A439A60D4
:107CA0007B681B687A681268926822F070629A603A
:107CB0007B681B687A681268926811467A68126B52
:107CC0000A439A607B681B687A681268926822F09F
:107CD00040529A607B681B687A6812689268114605
:107CE0007A68D26A0A439A607B681B687A6812686D
:107CF000926822F002029A607B681B687A681268B8
:107D0000926811467A6892694FEA42020A439A6081
:107D10007B685B6A002B2ED07B689B6A002B03D0AC
:107D20007B689B6A082B07D946F21020C0F6010039
:107D30004FF4986100F0B0F87B681B687A681268AD
:107D4000526842F400625A607B681B687A68126865
:107D5000526822F460425A607B681B687A68126835
:107D6000526811467A68926A02F1FF324FEA423253
:107D70000A435A6007E07B681B687A681268526899
:107D800022F400625A607B681B687A681268D26AC3
:107D900022F47002DA627B681B687A681268D26A21
:107DA00011467A68126A02F1FF324FEA02520A4320
:107DB000DA627B681B687A681268926822F4007243
:107DC0009A607B681B687A681268926811467A68C4
:107DD000D2694FEA42220A439A607B681B687A683C
:107DE0001268926822F480629A607B681B687A68E5
:107DF0001268926811467A6852694FEA82220A43F1
:107E00009A6007F10807BD4680BD00BF80B500AF8E
:107E10004FF47053C4F202034FF47052C4F20202E2
:107E2000126842F400721A604FF47053C4F20203F5
:107E30004FF47052C4F20202126842F480621A6077
:107E40004FF47053C4F202034FF47052C4F20202B2
:107E5000126842F480721A604FF47A50FFF78AFA7F
:107E60004FF00300FFF722FA00F004F84FF0000390
:107E7000184680BD80B400AFBD4680BC704700BFCF
:107E800080B400AF40F6DC03C2F200031B68184662
:107E9000BD4680BC704700BF80B584B000AF78603D
:107EA000396046F28423C0F60103FB6000F062F8FB
:107EB00080B483B000AF786039607B684FF0010216
:107EC0001A603A6840F20403C2F20003136007F13B
:107ED0000C07BD4680BC704780B584B000AF7860A9
:107EE00040F6E403C2F200031B68002B08D140F601
:107EF000E403C2F2000344F6DC42C2F200021A605C
:107F000040F6E403C2F200031B68FB607B6803F1E8
:107F1000030323F003037B6040F6E403C2F2000393
:107F20001A687B68D2184FF60043C2F201039A42E6
:107F300008D90AF079FB03464FF00C021A604FF0A3
:107F4000FF330CE040F6E403C2F200031A687B68DA
:107F5000D21840F6E403C2F200031A60FB68184628
:107F600007F11007BD4680BD80B483B000AF7860D4
:107F7000FEE700BF80B582B000AF46F2B023C0F686
:107F800001037B604FF00100FFF7EEFF80B400AF0C
:107F90004FF46D43CEF200034FF46D42CEF2000277
:107FA000D2F8882042F47002C3F888204FF460535E
:107FB000C4F202034FF46052C4F20202126842F0AB
:107FC00001021A604FF46053C4F202034FF0000242
:107FD0009A604FF46053C4F202034FF46052C4F24B
:107FE0000202126822F0847222F480321A604FF486
:107FF0006053C4F2020343F21002C2F200425A601C
:108000004FF46053C4F202034FF46052C4F2020210
:10801000126822F480221A604FF46053C4F2020303
:108020004FF00002DA604FF46D43CEF200034FF0E0
:1080300000629A60BD4680BC704700BF80B400AF4C
:10804000BD4680BC704700BF80B400AFFEE700BFF4
:1080500080B400AFFEE700BF80B400AFFEE700BF12
:1080600080B400AFFEE700BF80B400AFBD4680BC67
:10807000704700BF80B400AFBD4680BC704700BFF2
:1080800080B400AFBD4680BC704700BF80B500AF74
:1080900040F63C70C2F20000F8F71CFE80BD00BF45
:1080A00080B500AF03F012FB80BD00BF80B500AF0C
:1080B00040F6D863C2F200031B6C1846FAF772FF51
:1080C00080BD00BF80B500AF40F6D863C2F20003A8
:1080D0005B6C1846FAF766FF80BD00BF80B500AF45
:1080E00040F6B850C2F20000F8F7FCF980BD00BFBE
:1080F00080B590B000AF40F6D860C2F20000F9F74A
:108100005FF94FF46053C4F202034FF46052C4F2BB
:108110000202526C42F480525A644AF67003C0F66E
:1081200001039B883B604FF00203FB604FF00203AA
:108130007B604FF005033B614FF00003BB604AF6E4
:108140007003C0F601031A683B4610461946FAF759
:10815000EBFA4AF66003C0F601039B883B604FF0E0
:108160000203FB604FF002037B604FF00003BB6033
:108170004FF005033B614AF66003C0F601031A683D
:108180003B4610461946FAF7CFFA4AF66803C0F69E
:1081900001039B883B604FF00203FB604FF000033C
:1081A0007B604FF00103BB604FF005033B614AF673
:1081B0006803C0F601031A683B4610461946FAF7F1
:1081C000B3FA4AF61003C0F601039B883B604FF0F8
:1081D0000203FB604FF001037B604FF00003BB60C4
:1081E0004FF000033B614AF61003C0F601031A6822
:1081F0003B4610461946FAF797FA4AF61003C0F6BE
:1082000001031A684AF61003C0F601039B88104662
:1082100019464FF00102FAF761FE40F6D863C2F248
:1082200000034FF44052C4F201021A6040F6D863D2
:10823000C2F200034FF000029A6040F6D863C2F227
:1082400000034FF482725A6040F6D863C2F2000312
:108250004FF00002DA6040F6D863C2F200034FF03C
:1082600002021A6140F6D863C2F200034FF0010225
:108270005A6140F6D863C2F200034FF400729A616B
:1082800040F6D863C2F200034FF00002DA6140F614
:10829000D863C2F200034FF000021A6240F6D863BE
:1082A000C2F200034FF000029A6240F6D863C2F2B5
:1082B00000034FF000025A6240F6D863C2F2000396
:1082C0004FF00702DA6240F6D860C2F20000F8F719
:1082D00035FF07F14007BD4680BD00BF84B080B5C3
:1082E00000AF07F1080C8CE80F003B6E1B884FEACB
:1082F00013239BB2DAB240F6E803C2F200031A700D
:108300003B6E1B88DAB240F6E803C2F200035A70F3
:1083100040F6D860C2F2000040F6E801C2F2000167
:108320004FF002024FF00103F9F754F8BD46BDE8E3
:10833000804004B0704700BF80B582B000AF87EDC9
:10834000010A3860D7ED017AF5EEC07AF1EE10FA45
:10835000D4BF00230123DBB2002B0BD097ED010A21
:1083600008F072FEF0EE407A3B68C3ED007A4FF001
:10837000000304E03B68054A1A604FF0FF035BB25C
:10838000184607F10807BD4680BD00BF0000000089
:1083900080B592B000AF4FF46053C4F202034FF4C3
:1083A0006052C4F20202126C42F080521A644FF41E
:1083B000E043C4F200034FF4E042C4F2000212684A
:1083C00042F440421A604FF001037B604FF001031A
:1083D000BB604FF00203FB614FF480033B624FF040
:1083E0000F037B624FF0D203BB624FF00203FB62CC
:1083F0004FF007033B6307F104031846F9F75AFAF5
:108400004FF00D037B634FF00203BB634FF000039B
:10841000FB634FF4A0533B644FF480537B6407F13C
:10842000340318464FF00501F9F7FCFD07F1480742
:10843000BD4680BD80B48DB000AFF860B9607A6091
:108440004FF064037B85BB68022B00F39B804FF0E9
:108450000003FB627CE0BB68012B27D0022B45D0D8
:10846000002B71D17A68FB68D318C3F50072FB6AE0
:108470009A4210DA7B68C3F50072FB6A9A420ADD01
:1084800040F6D873C2F20003FA6A4FEA82029B18E0
:108490003F4A1A6058E040F6D873C2F20003FA6A05
:1084A0004FEA82029B183B4A1A604DE0FA6A7B68E9
:1084B0009A4210DD7A68FB68D218FB6A9A420ADD9C
:1084C00040F6D873C2F20003FA6A4FEA82029B18A0
:1084D0002F4A1A6038E040F6D873C2F20003FA6AF5
:1084E0004FEA82029B182B4A1A602DE07A68FB68DB
:1084F000D318C3F50072FB6A9A4205DA7B68C3F5AC
:108500000072FB6A9A4209DCFA6A7B689A4210DDC3
:108510007A68FB68D218FB6A9A420ADD40F6D87383
:10852000C2F20003FA6A4FEA82029B18184A1A60E4
:1085300009E040F6D873C2F20003FA6A4FEA8202F9
:108540009B18144A1A6000BFFB6A03F10103FB6227
:10855000FA6A40F2FF139A427FF77DAF40F6D87374
:10856000C2F2000303F580630A4A1A6040F6D8732A
:10857000C2F2000303F5FE6303F10C03054A1A601F
:1085800000BF00E000BF07F13407BD4680BC704764
:108590000000803F0000000080B485B000AF78602C
:1085A00039604FF00003FB607DE0FB684FEA430257
:1085B000FB684FEAC3037968CB1893ED007AFB6838
:1085C0004FEA430140F6D873C2F200034FEA81013B
:1085D0005B18D3ED007A27EE277AFB684FEAC303D6
:1085E00003F104037968CB18D3ED006AFB684FEA06
:1085F000430303F1010140F6D873C2F200034FEACE
:1086000081015B18D3ED007A66EEA77A77EE677A80
:1086100044F29003C2F200034FEA82029B18C3EDBA
:10862000007AFB684FEA430303F10102FB684FEA5B
:10863000C30303F104037968CB1893ED007AFB6858
:108640004FEA430303F1010140F6D873C2F200037D
:108650004FEA81015B18D3ED007A27EE277AFB6899
:108660004FEAC3037968CB18D3ED006AFB684FEA81
:10867000430140F6D873C2F200034FEA81015B1850
:10868000D3ED007A66EEA77A77EE277A44F290036C
:10869000C2F200034FEA82029B18C3ED007AFB6826
:1086A00003F10103FB60FB68FF2B7FF77EAF4FF008
:1086B0000003FB6032E03B684FEA4302FB68D318DB
:1086C000BB60FB68002B06DAFB684FEA83037A681D
:1086D000D318174A1A60FA6840F2FF139A4206DD6F
:1086E000FB684FEA83037A68D318114A1A60FB6863
:1086F0004FEA83037A68D2183B684FEA4301FB686C
:10870000C91844F29003C2F200034FEA81015B18DA
:108710001B681360FB6803F10103FB60FA6840F219
:10872000FF139A42C7DD07F11407BD4680BC7047AE
:108730000000000080B400AF4FF46053C4F20203A5
:108740004FF46052C4F20202126B42F001021A634B
:108750004FF46053C4F202034FF46052C4F20202B9
:10876000126B42F002021A634FF46053C4F2020328
:108770004FF46052C4F20202126B42F004021A6318
:108780004FF46053C4F202034FF46052C4F2020289
:10879000126B42F008021A634FF46053C4F20203F2
:1087A0004FF46052C4F20202126B42F010021A63DC
:1087B0004FF46053C4F202034FF46052C4F2020259
:1087C000126B42F400121A634FF46053C4F20203B6
:1087D0004FF46052C4F20202126B42F480021A6338
:1087E000BD4680BC704700BF80B483B000AF7860E6
:1087F00007F10C07BD4680BC704700BF80B400AFD6
:1088000040F66453C2F200031B6803F1010240F614
:108810006453C2F200031A60BD4680BC704700BFBB
:1088200080B500AF40F6F003C2F20003D3E90001C7
:108830004FF001024FF00003801841EB030140F6B6
:10884000F003C2F20003C3E9000105F05FFA48F645
:10885000D503C0F60003984740F68063C2F20003D8
:108860001B68002B0BD040F68063C2F200031B682C
:1088700003F1FF3240F68063C2F200031A6080BD4C
:1088800080B400AF41F2D873C2F200034FF000028F
:108890001A6040F6D473C2F200034FF000021A606F
:1088A00042F60003C2F200034FF07F021A6041F269
:1088B000DC73C2F200034FF000021A6044F6B443C6
:1088C000C2F200034FF064021A601846BD4680BC35
:1088D000704700BF98B500AF40F61813C2F200030E
:1088E0001B78002B40F0F5804AF68003C0F60103A8
:1088F0001A684AF68003C0F601039B8810461946A1
:10890000FAF792FA03464FEA43044AF67803C0F6B0
:1089100001031A684AF67803C0F601039B881046E3
:108920001946FAF781FA0346E21840F6D473C2F208
:1089300000031A6040F6D473C2F200031A6841F2D1
:10894000D873C2F200031B689A4200F0B88041F26B
:10895000D873C2F200031B68002B06D140F6D47313
:10896000C2F200031B68012B29D041F2D873C2F276
:1089700000031B68012B06D140F6D473C2F200033A
:108980001B68032B1BD041F2D873C2F200031B6893
:10899000032B06D140F6D473C2F200031B68022BEE
:1089A0000DD041F2D873C2F200031B68022B09D12B
:1089B00040F6D473C2F200031B68002B02D14FF0C3
:1089C000010201E04FF0000244F20C03C2F2000386
:1089D0001A604AF68803C0F601031A684AF688034B
:1089E000C0F601039B8810461946FAF71DFA0346A4
:1089F000002B44D144F20C03C2F200031B68002B8D
:108A00000DD040F6FC03C2F200031B8803F1010302
:108A10009AB240F6FC03C2F200031A800CE040F662
:108A2000FC03C2F200031B8803F1FF339AB240F645
:108A3000FC03C2F200031A8040F6FC03C2F20003FA
:108A40001B884FEA53039AB240F6FA03C2F20003BE
:108A50001A8040F6FA03C2F200031A8840F220039B
:108A6000C2F200031B88B2FBF3F103FB01F3D31A3C
:108A70009AB240F6FA03C2F200031A801FE044F2F1
:108A80000C03C2F200031B68002B0CD044F6B84361
:108A9000C2F200031B6803F1010244F6B843C2F2BC
:108AA00000031A600BE044F6B843C2F200031B68EF
:108AB00003F1FF3244F6B843C2F200031A6040F6F5
:108AC000D473C2F200031A6841F2D873C2F20003F1
:108AD0001A6098BD80B400AF44F6B843C2F20003F8
:108AE0001B684FEAD372D3184FEA63031846BD469A
:108AF00080BC70470000000098B500AF40F63173AD
:108B0000C2F200031B78002B00F02A8740F63A736C
:108B1000C2F200031B88642B09D14FF00000C4F29D
:108B200002004FF480714FF00102FAF7D7F904F018
:108B30006BFF40F62C13C2F200031B68012B00F000
:108B40002282022B00F04284002B40F0688640F61F
:108B50001013C2F200031B68002B62D140F63A7377
:108B6000C2F200031B884FEA430440F62E73C2F2A0
:108B700000031B889BB21A4640F24403C2F2000372
:108B80001B68D31A184608F0DFFE02460B46104653
:108B900019460FF2C443D3E9002309F065F80246F1
:108BA0000B461046194609F0F7F9024643F20C034A
:108BB000C2F200034FEA84015B181A6040F63A7370
:108BC000C2F200031B884FEA430303F1010440F69D
:108BD0007C63C2F200031B889BB21A4640F240033A
:108BE000C2F200031B68D31A184608F0ADFE024615
:108BF0000B46104619460FF26043D3E9002309F0F3
:108C000033F802460B461046194609F0C5F90246EC
:108C100043F20C03C2F200034FEA84015B181A60AE
:108C20005FE040F63A73C2F200031B884FEA430448
:108C300040F6A053C2F200031B889BB21A4640F2D2
:108C40003C03C2F200031B68D31A184608F07CFEEE
:108C500002460B4610461946FFA3D3E9002309F04C
:108C600003F802460B461046194609F095F90246EC
:108C700043F20C03C2F200034FEA84015B181A604E
:108C800040F63A73C2F200031B884FEA430303F134
:108C9000010440F6A053C2F200031B889BB21A469F
:108CA00040F23C03C2F200031B68D31A184608F0D6
:108CB0004BFE02460B4610461946E7A3D3E90023B4
:108CC00008F0D2FF02460B461046194609F064F937
:108CD000024643F20C03C2F200034FEA84015B1820
:108CE0001A6040F6A053C2F200031B889AB240F605
:108CF000F803C2F200031B889A420AD940F6A05337
:108D0000C2F200031B889AB240F6F803C2F20003D5
:108D10001A8040F67C63C2F200031B889AB240F6C8
:108D2000F803C2F200031B889A420AD940F67C631A
:108D3000C2F200031B889AB240F6F803C2F20003A5
:108D40001A8040F63A73C2F200031B884FEA4302CE
:108D500041F2E073C2F200034FEA82029B1893EDE6
:108D6000007A40F60813C2F20003D3ED007AB4EEA5
:108D7000E77AF1EE10FAD4BF00230123DBB2002B17
:108D800013D040F63A73C2F200031B884FEA430245
:108D900041F2E073C2F200034FEA82029B181A68A4
:108DA00040F60813C2F200031A6040F63A73C2F2AA
:108DB00000031B884FEA430303F1010241F2E07311
:108DC000C2F200034FEA82029B1893ED007A40F64C
:108DD0000813C2F20003D3ED007AB4EEE77AF1EEA5
:108DE00010FAD4BF00230123DBB2002B15D040F6CC
:108DF0003A73C2F200031B884FEA430303F10102F6
:108E000041F2E073C2F200034FEA82029B181A6833
:108E100040F60813C2F200031A6040F63A73C2F239
:108E200000031B884FEA430241F2E073C2F20003E1
:108E30004FEA82029B1893ED007ADFED897A27EEE4
:108E4000277A40F21003C2F20003D3ED007A27EE36
:108E5000277ADFED847A77EE277AFCEEE77A17EE51
:108E6000903A9BB2184603F06DF940F63A73C2F29D
:108E700000031B884FEA430303F1010241F2E07350
:108E8000C2F200034FEA82029B1893ED007ADFEDF5
:108E9000747A27EE277A40F21003C2F20003D3ED72
:108EA000007A27EE277ADFED6F7A77EE277AFCEEED
:108EB000E77A17EE903A9BB2184603F05DF940F658
:108EC0003A73C2F200031B881A4640F21C03C2F236
:108ED00000031B88C3F1FF039A42C0F29B8440F653
:108EE0003A73C2F200031B881A4640F21C03C2F216
:108EF00000031B88A3F58073D3184FEA430140F6A3
:108F00003A73C2F200031B884FEA430243F20C0398
:108F1000C2F200034FEA82029B181A6844F69403D7
:108F2000C2F200034FEA81015B181A6040F63A73FF
:108F3000C2F200031B881A4640F21C03C2F200036F
:108F40001B88A3F58073D3184FEA430303F1010193
:108F500040F63A73C2F200031B884FEA430303F161
:108F6000010243F20C03C2F200034FEA82029B1893
:108F70001A6844F69403C2F200034FEA81015B18B9
:108F80001A6000F047BC40F61013C2F200031B68E1
:108F9000002B69D140F63A73C2F200031B884FEAF6
:108FA000430440F62E73C2F200031B889BB21A469C
:108FB00040F24403C2F200031B68D31A184608F0BB
:108FC000C3FC02460B461046194623A3D3E90023EF
:108FD00008F04AFE02460B461046194608F0DCFF30
:108FE000024641F2E073C2F200034FEA84015B18CB
:108FF0001A6040F63A73C2F200031B884FEA43033B
:1090000003F1010440F67C63C2F200031B889BB2AB
:109010001A4640F24003C2F200031B68D31A1846F6
:1090200008F092FC02460B46104619460AA3D3E903
:10903000002308F019FE02460B461046194608F0B8
:10904000ABFF024641F2E073C2F200034FEA840133
:109050005B181A6069E000BF000000000000B0402B
:10906000000080450000004540F63A73C2F200035C
:109070001B884FEA430440F6A053C2F200031B884A
:109080009BB21A4640F23C03C2F200031B68D31A9B
:10909000184608F059FC02460B46104619460FF2D6
:1090A0000043D3E9002308F0DFFD02460B461046DB
:1090B000194608F071FF024641F2E073C2F2000364
:1090C0004FEA84015B181A6040F63A73C2F200035B
:1090D0001B884FEA430303F1010440F6A053C2F298
:1090E00000031B889BB21A4640F23C03C2F2000305
:1090F0001B68D31A184608F027FC02460B46104698
:109100001946E7A3D3E9002308F0AEFD02460B465B
:109110001046194608F040FF024641F2E073C2F2E1
:1091200000034FEA84015B181A6040F6A053C2F2B4
:1091300000031B889AB240F6F803C2F200031B88B2
:109140009A420AD940F6A053C2F200031B889AB291
:1091500040F6F803C2F200031A8040F67C63C2F2C4
:1091600000031B889AB240F6F803C2F200031B8882
:109170009A420AD940F67C63C2F200031B889AB275
:1091800040F6F803C2F200031A8040F63A73C2F2C6
:1091900000031B884FEA430242F20003C2F20003BD
:1091A0004FEA82029B1893ED007A40F60813C2F250
:1091B0000003D3ED007AB4EEE77AF1EE10FAD4BFF3
:1091C00000230123DBB2002B13D040F63A73C2F226
:1091D00000031B884FEA430242F20003C2F200037D
:1091E0004FEA82029B181A6840F60813C2F2000385
:1091F0001A6040F63A73C2F200031B884FEA430339
:1092000003F1010242F20003C2F200034FEA8202BC
:109210009B1893ED007A40F60813C2F20003D3EDD9
:10922000007AB4EEE77AF1EE10FAD4BF00230123FE
:10923000DBB2002B15D040F63A73C2F200031B8854
:109240004FEA430303F1010242F20003C2F20003BA
:109250004FEA82029B181A6840F60813C2F2000314
:109260001A6040F63A73C2F200031B884FEA4302C9
:1092700042F20003C2F200034FEA82029B1893ED10
:10928000007ADFED897A27EE277A40F21003C2F2E6
:109290000003D3ED007A27EE277ADFED847A77EEAC
:1092A000277AFCEEE77A17EE903A9BB2184602F066
:1092B00049FF40F63A73C2F200031B884FEA4303AA
:1092C00003F1010242F20003C2F200034FEA8202FC
:1092D0009B1893ED007ADFED747A27EE277A40F23F
:1092E0001003C2F20003D3ED007A27EE277ADFEDF8
:1092F0006F7A77EE277AFCEEE77A17EE903A9BB218
:10930000184602F039FF40F63A73C2F200031B8898
:109310001A4640F21C03C2F200031B88C3F1FF038C
:109320009A42C0F2798240F63A73C2F200031B8877
:109330001A4640F21C03C2F200031B88A3F5807397
:10934000D3184FEA430140F63A73C2F200031B8878
:109350004FEA430241F2E073C2F200034FEA820295
:109360009B181A6844F69403C2F200034FEA810185
:109370005B181A6040F63A73C2F200031B881A4663
:1093800040F21C03C2F200031B88A3F58073D318BC
:109390004FEA430303F1010140F63A73C2F20003BE
:1093A0001B884FEA430303F1010241F2E073C2F26A
:1093B00000034FEA82029B181A6844F69403C2F233
:1093C00000034FEA81015B181A6025E240F6101392
:1093D000C2F200031B68002B6AD140F63A73C2F256
:1093E00000031B884FEA430440F62E73C2F20003C9
:1093F0001B889BB21A4640F24403C2F200031B686A
:10940000D31A184608F0A0FA02460B461046194631
:1094100023A3D3E9002308F027FC02460B4610469D
:10942000194608F0B9FD024642F20003C2F20003F9
:109430004FEA84015B181A6040F63A73C2F20003E7
:109440001B884FEA430303F1010440F67C63C2F238
:1094500000031B889BB21A4640F24003C2F200038D
:109460001B68D31A184608F06FFA02460B461046DE
:1094700019460BA3D3E9002308F0F6FB02460B467E
:109480001046194608F088FD024642F20003C2F277
:1094900000034FEA84015B181A606BE0AFF30080B1
:1094A000000000000000B0400000804500000045C2
:1094B00040F63A73C2F200031B884FEA430440F6B9
:1094C000A053C2F200031B889BB21A4640F23C0331
:1094D000C2F200031B68D31A184608F035FA024698
:1094E0000B46104619460FF29043D3E9002308F0CB
:1094F000BBFB02460B461046194608F04DFD0246DE
:1095000042F20003C2F200034FEA84015B181A60C2
:1095100040F63A73C2F200031B884FEA430303F19B
:10952000010440F6A053C2F200031B889BB21A4606
:1095300040F23C03C2F200031B68D31A184608F03D
:1095400003FA02460B46104619460FF22C43D3E9A4
:10955000002308F089FB02460B461046194608F026
:109560001BFD024642F20003C2F200034FEA8401EF
:109570005B181A6040F6A053C2F200031B889AB22F
:1095800040F6F803C2F200031B889A420AD940F65B
:10959000A053C2F200031B889AB240F6F803C2F24D
:1095A00000031A8040F67C63C2F200031B889AB263
:1095B00040F6F803C2F200031B889A420AD940F62B
:1095C0007C63C2F200031B889AB240F6F803C2F231
:1095D00000031A8040F63A73C2F200031B884FEA78
:1095E000430243F20C03C2F200034FEA82029B18CB
:1095F00093ED007A40F60813C2F20003D3ED007A2F
:10960000B4EEE77AF1EE10FAD4BF00230123DBB207
:10961000002B13D040F63A73C2F200031B884FEAC6
:10962000430243F20C03C2F200034FEA82029B188A
:109630001A6840F60813C2F200031A6040F63A7343
:10964000C2F200031B884FEA430303F1010243F215
:109650000C03C2F200034FEA82029B1893ED007ADA
:1096600040F60813C2F20003D3ED007AB4EEE77AB5
:10967000F1EE10FAD4BF00230123DBB2002B15D08A
:1096800040F63A73C2F200031B884FEA430303F12A
:10969000010243F20C03C2F200034FEA82029B185C
:1096A0001A6840F60813C2F200031A6040F63A73D3
:1096B000C2F200031B884FEA430243F20C03C2F2DA
:1096C00000034FEA82029B1893ED007ADFEDA87A3F
:1096D00027EE277A40F21003C2F20003D3ED007A9E
:1096E00027EE277ADFEDA37A77EE277AFCEEE77A8A
:1096F00017EE903A9BB2184602F024FD40F63A73FA
:10970000C2F200031B884FEA430303F1010243F254
:109710000C03C2F200034FEA82029B1893ED007A19
:10972000DFED937A27EE277A40F21003C2F20003AE
:10973000D3ED007A27EE277ADFED8E7A77EE277A5F
:10974000FCEEE77A17EE903A9BB2184602F014FD51
:1097500040F63A73C2F200031B881A4640F21C031B
:10976000C2F200031B88C3F1FF039A4256DB40F6A6
:109770003A73C2F200031B881A4640F21C03C2F27D
:1097800000031B88A3F58073D3184FEA430140F60A
:109790003A73C2F200031B884FEA430242F200030D
:1097A000C2F200034FEA82029B181A6844F694033F
:1097B000C2F200034FEA81015B181A6040F63A7367
:1097C000C2F200031B881A4640F21C03C2F20003D7
:1097D0001B88A3F58073D3184FEA430303F10101FB
:1097E00040F63A73C2F200031B884FEA430303F1C9
:1097F000010242F20003C2F200034FEA82029B1808
:109800001A6844F69403C2F200034FEA81015B1820
:109810001A6003E000BF02E000BF00E000BF40F6B6
:109820000813C2F200031B68184608F09FF80246AE
:109830000B46104619464CA3D3E9002308F0EAF87A
:1098400002460B461046194608F0A6FB024640F6B3
:109850000813C2F200031A6040F63A73C2F2000322
:109860001B8803F101039AB240F63A73C2F2000377
:109870001A8040F63A73C2F200031B88FF2B6DD9A1
:109880004FF00000C4F202004FF480714FF000026C
:10989000F9F724FB40F6D163C2F200034FF0010256
:1098A0001A7040F21C03C2F200031A8840F63A73A1
:1098B000C2F200031A8040F62C13C2F200031B68A8
:1098C000012B1BD0022B31D0002B47D140F61C13AB
:1098D000C2F200034FF001021A6040F62C13C2F2EC
:1098E00000034FF001021A6049F68113C0F600032D
:1098F00041F2E070C2F2000098472FE040F62013DA
:10990000C2F200034FF001021A6040F62C13C2F2BB
:1099100000034FF002021A6049F68113C0F60003FB
:1099200042F20000C2F20000984717E040F624130C
:10993000C2F200034FF001021A6040F62C13C2F28B
:1099400000034FF000021A6049F68113C0F60003CD
:1099500043F20C00C2F20000984700BF04F0B2F8D6
:1099600098BD00BFAFF300801EA7E8482EFFEF3F71
:109970000000804500000045000000000000B040ED
:1099800080B485B000AF78604FF00003FB8112E037
:10999000FB894FEA83037A68D218F98944F6940365
:1099A000C2F200034FEA81015B181B681360FB8958
:1099B00003F10103FB81FA8940F21C03C2F20003A8
:1099C0001B884FEA43039A42E2DB0AE0FB894FEA35
:1099D00083037A68D318084A1A60FB8903F10103EC
:1099E000FB81FA8940F2FF139A42EFD907F114077D
:1099F000BD4680BC704700BF0000000080B584B049
:109A000000AF02460B46FA71BB714AF63813C0F636
:109A100001031A684AF63813C0F601039B88104602
:109A200019464FF00002F9F759FA4AF63013C0F61A
:109A300001031A684AF63013C0F601039B881046EA
:109A400019464FF00002F9F749FA4AF62813C0F612
:109A500001031A684AF62813C0F601039B881046D2
:109A600019464FF00002F9F739FA4AF62813C0F602
:109A700001031A684AF62813C0F601039B881046B2
:109A800019464FF00102F9F729FA4FF00003FB7372
:109A90003CE04AF63013C0F6010319684AF6301369
:109AA000C0F601039A88F879FB7BC3F1070340FAFB
:109AB00003F3DBB203F00103DBB2084611461A469A
:109AC000F9F70CFA4AF62813C0F601031A684AF6A9
:109AD0002813C0F601039B88104619464FF0000278
:109AE000F9F7FCF94AF62813C0F601031A684AF69A
:109AF0002813C0F601039B88104619464FF0010257
:109B0000F9F7ECF9FB7B03F10103FB73FB7B072BFC
:109B1000BFD94AF63813C0F601031A684AF638135B
:109B2000C0F601039B88104619464FF00102F9F771
:109B3000D5F94AF63813C0F601031A684AF6381305
:109B4000C0F601039B88104619464FF00002F9F752
:109B5000C5F94AF63013C0F601031A684AF6301305
:109B6000C0F601039B88104619464FF00102F9F731
:109B7000B5F94AF62813C0F601031A684AF6281305
:109B8000C0F601039B88104619464FF00002F9F712
:109B9000A5F94AF62813C0F601031A684AF62813F5
:109BA000C0F601039B88104619464FF00102F9F7F1
:109BB00095F94FF00003FB733CE04AF63013C0F612
:109BC000010319684AF63013C0F601039A88B87980
:109BD000FB7BC3F1070340FA03F3DBB203F001039D
:109BE000DBB2084611461A46F9F778F94AF6281307
:109BF000C0F601031A684AF62813C0F601039B88D1
:109C0000104619464FF00002F9F768F94AF6281392
:109C1000C0F601031A684AF62813C0F601039B88B0
:109C2000104619464FF00102F9F758F9FB7B03F192
:109C30000103FB73FB7B072BBFD94AF63813C0F631
:109C400001031A684AF63813C0F601039B881046D0
:109C500019464FF00102F9F741F907F11007BD4627
:109C600080BD00BF80B500AFFEF738FA184680BD52
:109C700080B400AFBD4680BC704700BF80B58CB0DB
:109C800002AF78603960FEF7C1F8FEF781FB46F25B
:109C9000C423C0F601033B6146F2D823C0F601039A
:109CA000FB60FEF747FD02F099FAFEF721FA40F655
:109CB000D860C2F20000FEF797FD04F013F804F03C
:109CC0003DF84FF00000C4F202004FF480714FF0F5
:109CD0000102F9F703F940F22C03C2F200031B88DA
:109CE0001AB240F60413C2F200031B881BB2D11A49
:109CF00040F60613C2F200031B781A4640F604131E
:109D0000C2F200031B881BB2084611461A46FEF732
:109D100091FB4CF22503C0F600039847FEF7B0FD17
:109D200004F0FAF84FF0010004F05AFE4FF0000082
:109D300004F0E6FE4FF0030005F078FA4FF0010062
:109D400005F0A2FA4FF6FF704FF0000105F084FA1B
:109D50004FF000004FF078014FF0C80204F0FEFD14
:109D600003F0CAFB40F63173C2F200034FF0010268
:109D70001A7003F0A7FE4BF6B163C0F600039847D4
:109D80004FF000024FF00003C7E908234AF2A9731D
:109D9000C0F600034FF0010098474FF080004FF0ED
:109DA0008001FFF72BFEFFF763FF40F6B850C2F2C9
:109DB000000044F6B431C2F200014FF01002F6F791
:109DC0001FFB40F6B853C2F200039B6AFB6144F6E6
:109DD000B433C2F20003BB61FA69BB69D31A4FEA1C
:109DE000A3037B614AF2E913C0F6000398474AF2E5
:109DF000A973C0F600034FF0000098474BF2F1132F
:109E0000C0F6000398474AF2F903C0F600039847EA
:109E10004AF68813C0F601031A684AF68813C0F69A
:109E200001039B8810461946F8F7FEFF0346002BF6
:109E300002D14FF4784301E04FF01F0300934FF439
:109E40009B704FF000014FF003024FF0030304F04A
:109E500033FE4AF69013C0F601031A684AF69013CF
:109E6000C0F601039B8810461946F8F7DDFF03464C
:109E7000002B02D14FF4784301E04FF01F03009311
:109E80004FF49B704FF004014FF003024FF00303B7
:109E900004F012FE4AF67813C0F601031A684AF677
:109EA0007813C0F601039B8810461946F8F7BCFFEB
:109EB0000346002B02D04FF4784301E04FF01F031C
:109EC00000934FF49B704FF008014FF003024FF0E6
:109ED000030304F0F1FD4AF68013C0F601031A688B
:109EE0004AF68013C0F601039B8810461946F8F71E
:109EF0009BFF0346002B02D04FF4784301E04FF064
:109F00001F0300934FF49B704FF00C014FF00302BE
:109F10004FF0030304F0D0FD4AF67813C0F60103B6
:109F20001A684AF67813C0F601039B881046194652
:109F3000F8F77AFF0346002B6ED040F61013C2F2FA
:109F400000034FF001021A604AF64013C0F6010305
:109F50001A684AF64013C0F601039B88104619465A
:109F60004FF00102F8F7BAFF4AF6C803C0F6010342
:109F70001A684AF6C803C0F601039B8810461946C2
:109F80004FF00102F8F7AAFF4AF6D003C0F601032A
:109F90001A684AF6D003C0F601039B88104619469A
:109FA0004FF00002F8F79AFF4AF6D803C0F6010313
:109FB0001A684AF6D803C0F601039B881046194672
:109FC0004FF00102F8F78AFF4AF6E003C0F60103FA
:109FD0001A684AF6E003C0F601039B88104619464A
:109FE0004FF00002F8F77AFF4AF61813C0F60103A3
:109FF0001A684AF61813C0F601039B8810461946E2
:10A000004FF00002F8F76AFF40F61413C2F20003A3
:10A010004FF000021A60C8E640F61013C2F20003C7
:10A020004FF000021A604AF64013C0F601031A68A6
:10A030004AF64013C0F601039B88104619464FF0BC
:10A040000002F8F74BFF4AF6C803C0F601031A688E
:10A050004AF6C803C0F601039B88104619464FF024
:10A060000002F8F73BFF4AF6D003C0F601031A6876
:10A070004AF6D003C0F601039B88104619464FF0FC
:10A080000102F8F72BFF4AF6D803C0F601031A685D
:10A090004AF6D803C0F601039B88104619464FF0D4
:10A0A0000002F8F71BFF4AF6E003C0F601031A6846
:10A0B0004AF6E003C0F601039B88104619464FF0AC
:10A0C0000102F8F70BFF4AF61813C0F601031A68ED
:10A0D0004AF61813C0F601039B88104619464FF044
:10A0E0000102F8F7FBFE40F61413C2F200034FF032
:10A0F00000021A6059E600BF80B584B002AF40F696
:10A100003013C2F2000393ED007ADFED357A27EECB
:10A11000277AF7EE007A77EE277A17EE900A07F0A3
:10A1200025FC02460B4643EC102B06F007FF53ECD0
:10A13000102B1046194628A3D3E9002307F06AFC28
:10A1400002460B461046194607F0FEFE03467B60AA
:10A1500040F63413C2F200031B687A689A4219DD94
:10A1600040F63413C2F200031B6803F1960240F676
:10A170003413C2F200031B687968CB1A4FF478419C
:10A18000009110464FF09C011A464FF0030304F073
:10A1900093FC14E07B6803F1960240F63413C2F29C
:10A1A000000319687B68CB1A4FF00001009110463C
:10A1B0004FF09C011A464FF0030304F07DFC40F67B
:10A1C0003413C2F200037A681A6007F10807BD462B
:10A1D00080BD00BFAFF300800000000000002440FD
:10A1E00000247449AFF3008080B500AF40F6FA0355
:10A1F000C2F200031B880A2B00F2818201A050F8F2
:10A2000023F000BF31A200084FA200086DA2000891
:10A2100087A20008A1A20008BBA20008D5A20008DE
:10A22000EFA2000819A4000843A500080BA6000827
:10A2300040F22403C2F2000344F24022C0F20F02B3
:10A240001A604BF6C133C0F60003984760E240F253
:10A250002403C2F2000348F2A062C0F201021A60B5
:10A260004BF6C133C0F60003984751E240F2240395
:10A27000C2F2000342F210721A604BF6C133C0F60C
:10A280000003984744E240F22403C2F200034FF473
:10A290007A721A604BF6C133C0F60003984737E272
:10A2A00040F22403C2F200034FF064021A604BF63E
:10A2B000C133C0F6000398472AE240F22403C2F2F9
:10A2C00000034FF00A021A604BF6C133C0F60003D8
:10A2D00098471DE240F22403C2F200034FF001024E
:10A2E0001A604BF6C133C0F60003984710E2FEF740
:10A2F000F1FB024644F28C03C2F200031A6044F2FE
:10A300008C03C2F200031A6843F20803C2F200038E
:10A310001B689A4200F0F58143F20803C2F2000381
:10A320001B689AB244F28C03C2F200031B689BB212
:10A33000D31A9AB240F60413C2F200031B889BB2F0
:10A34000D3189BB29AB240F60413C2F200031A80EB
:10A3500040F60413C2F200031B881BB2002B06DC7C
:10A3600040F60413C2F200034FF000021A8040F6D8
:10A370000413C2F200031B881BB2C72B06DD40F694
:10A380000413C2F200034FF064021A8040F6041373
:10A39000C2F200031A8840F22C03C2F200031B88A9
:10A3A00012B21BB29A420EDB40F22C03C2F200033F
:10A3B0001B889BB203F1FF339BB29AB240F60413A1
:10A3C000C2F200031A8044F28C03C2F200031A683E
:10A3D00043F20803C2F200031A6040F22C03C2F2F7
:10A3E00000031B881AB240F60413C2F200031B8854
:10A3F0001BB2D11A40F60613C2F200031B781A46AC
:10A4000040F60413C2F200031B881BB20846114633
:10A410001A46FEF70FF874E1FEF75CFB024644F2C1
:10A420008C03C2F200031A6044F28C03C2F20003F0
:10A430001A6843F20803C2F200031B689A4200F054
:10A44000628143F20803C2F200031B689AB244F22D
:10A450008C03C2F200031B689BB2D31A9AB240F27B
:10A460002C03C2F200031B889BB2D3189BB29AB292
:10A4700040F22C03C2F200031A8040F22C03C2F215
:10A4800000031B881BB2002B06DC40F22C03C2F237
:10A4900000034FF000021A8040F22C03C2F20003C6
:10A4A0001B881BB2C72B06DD40F22C03C2F200034F
:10A4B0004FF064021A8040F22C03C2F200031A88A3
:10A4C00040F60413C2F200031B8812B21BB29A4278
:10A4D0000EDC40F60413C2F200031B889BB203F1AA
:10A4E00001039BB29AB240F22C03C2F200031A801D
:10A4F00044F28C03C2F200031A6843F20803C2F26A
:10A5000000031A6040F22C03C2F200031B881AB247
:10A5100040F60413C2F200031B881BB2D11A40F6A6
:10A520000613C2F200031B781A4640F60413C2F267
:10A5300000031B881BB2084611461A46FDF77AFF36
:10A54000E1E0FEF7C7FA024644F28C03C2F20003D0
:10A550001A6044F28C03C2F200031A6843F2080343
:10A56000C2F200031B689A4200F0CF8040F6061347
:10A57000C2F200031B781A4643F20803C2F200033A
:10A58000196844F28C03C2F200031B68CB1AD1187D
:10A5900045F25653C5F2555383FB01024FEAE1736E
:10A5A000D21A13464FEA43039B18CA1AD2B240F696
:10A5B0000613C2F200031A7040F22C03C2F2000329
:10A5C0001B881AB240F60413C2F200031B881BB2A8
:10A5D000D11A40F60613C2F200031B781A4640F661
:10A5E0000413C2F200031B881BB2084611461A4628
:10A5F000FDF720FF44F28C03C2F200031A6843F215
:10A600000803C2F200031A607FE0FEF763FA024615
:10A6100044F28C03C2F200031A6044F28C03C2F2CB
:10A6200000031A6843F20803C2F200031B689A424F
:10A630006DD043F20803C2F200031A6844F28C039F
:10A64000C2F200031B68D31A07EE903AB8EEE77A1D
:10A6500040F21403C2F20003D3ED007A27EE277A0A
:10A6600040F21003C2F20003D3ED007A77EE277AAE
:10A6700040F21003C2F20003C3ED007A40F210036F
:10A68000C2F2000393ED007A40F21803C2F2000315
:10A69000D3ED007AB4EEE77AF1EE10FAD4BF0023DE
:10A6A0000123DBB2002B09D040F21803C2F20003F1
:10A6B0001A6840F21003C2F200031A6040F210035D
:10A6C000C2F20003D3ED007AF5EEC07AF1EE10FA93
:10A6D0008CBF00230123DBB2002B05D040F2100316
:10A6E000C2F200030B4A1A6044F28C03C2F2000368
:10A6F0001A6843F20803C2F200031A6007E000BFC1
:10A7000006E000BF04E000BF02E000BF00E000BFC1
:10A7100080BD00BF0000000080B586B000AF78604B
:10A7200039601F4B3B614FF000037B6119E07B698F
:10A730004FEA83037A68D31893ED007A7B694FEA76
:10A7400083037A68D318D3ED007A67EE277A97ED02
:10A75000047A77EE277AC7ED047A7B6903F1010367
:10A760007B617A693B689A42E1DB3B6807EE103A0D
:10A77000F8EEC77A97ED047AC7EE277AC7ED047A28
:10A7800007F10C0397ED040A1846FDF7D5FDFB68A9
:10A7900007EE903AB0EE670A07F11807BD4680BD94
:10A7A000000000000000000090B589B004AF03462F
:10A7B000FB7140F61813C2F200034FF001021A7049
:10A7C000FB79002B74D04FF00C0300934FF6FF730E
:10A7D00001934FF096004FF05A0146F2FC22C0F66A
:10A7E00001024FF0280304F003FB4FF088030093AD
:10A7F0004FF0720301934FF6FF7302934FF07E0008
:10A800004FF077014FF088024FF07C0304F096F987
:10A810004FF00C0300934FF6FF7301934FF0960037
:10A820004FF0880148F23872C0F601024FF02F0352
:10A8300004F0DEFA4BF6AD44C0F600044FF02E00F3
:10A840004FF0AE014FF06C024FF6FF73A0474BF68E
:10A85000AD44C0F600044FF02E004FF0EE014FF073
:10A860006C024FF6FF73A0474FF00A0300934FF6B8
:10A87000FF7301934FF08E004FF0A20149F6CC32E6
:10A88000C0F601024FF09B0304F0B2FA4FF02E0322
:10A8900000934FF6FF73019340F211104FF0C00187
:10A8A00048F6A032C0F601024FF02D0304F0A0FAE2
:10A8B00040F22803C2F200031B6840F65450C2F273
:10A8C000000046F2EC21C0F601011A4607F0F4FE42
:10A8D00040F65453C2F200031A7840F24803C2F221
:10A8E00000031B7852B25BB29A421CD1FB79002B59
:10A8F00019D140F6FA03C2F200031A8840F21E038F
:10A90000C2F200031B889A4229D040F6FA03C2F231
:10A9100000031B88002B06D040F21E03C2F2000386
:10A920001B88002B1BD14BF6AD44C0F6000440F64B
:10A930005453C2F200031B785AB240F6FA03C2F233
:10A9400000031B88002B02D14FF4784301E04FF63F
:10A95000FF7310464FF08E014FF06C02A04740F697
:10A960005453C2F200035A7840F24803C2F2000383
:10A970005B7852B25BB29A4223D141F6E073C2F2E5
:10A9800000031B78002B1CD1FB79002B19D140F65A
:10A99000FA03C2F200031A8840F21E03C2F2000357
:10A9A0001B889A4229D040F6FA03C2F200031B88A2
:10A9B000002B06D040F21E03C2F200031B88002BBE
:10A9C0001BD14BF6AD44C0F6000440F65453C2F21E
:10A9D00000035B785AB240F6FA03C2F200031B8808
:10A9E000002B02D14FF4784301E04FF6FF7310467D
:10A9F0004FF09E014FF06C02A04740F65453C2F254
:10AA000000039A7840F24803C2F200039B7852B2E6
:10AA10005BB29A421CD1FB79002B19D140F6FA03A4
:10AA2000C2F200031A8840F21E03C2F200031B8820
:10AA30009A4229D040F6FA03C2F200031B88012B88
:10AA400006D040F21E03C2F200031B88012B1BD16B
:10AA50004BF6AD44C0F6000440F65453C2F2000376
:10AA60009B785AB240F6FA03C2F200031B88012B0E
:10AA700002D14FF4784301E04FF6FF7310464FF0D8
:10AA8000BE014FF06C02A04740F65453C2F20003DF
:10AA9000DA7840F24803C2F20003DB7852B25BB2CC
:10AAA0009A421CD1FB79002B19D140F6FA03C2F26D
:10AAB00000031A8840F21E03C2F200031B889A4268
:10AAC00029D040F6FA03C2F200031B88022B06D0FD
:10AAD00040F21E03C2F200031B88022B1BD14BF66F
:10AAE000AD44C0F6000440F65453C2F20003DB78D4
:10AAF0005AB240F6FA03C2F200031B88022B02D1BD
:10AB00004FF4784301E04FF6FF7310464FF0CE014B
:10AB10004FF06C02A04740F65453C2F200031A797A
:10AB200040F24803C2F200031B7952B25BB29A4270
:10AB30001CD1FB79002B19D140F6FA03C2F20003B5
:10AB40001A8840F21E03C2F200031B889A4229D0E1
:10AB500040F6FA03C2F200031B88032B06D040F232
:10AB60001E03C2F200031B88032B1BD14BF6AD441E
:10AB7000C0F6000440F65453C2F200031B795AB2E7
:10AB800040F6FA03C2F200031B88032B02D14FF4F4
:10AB9000784301E04FF6FF7310464FF0DE014FF0AF
:10ABA0006C02A04740F65453C2F200035A7940F2B7
:10ABB0004803C2F200035B7952B25BB29A421CD1E5
:10ABC000FB79002B19D140F6FA03C2F200031A8870
:10ABD00040F21E03C2F200031B889A4229D040F6BD
:10ABE000FA03C2F200031B88042B06D040F21E03B6
:10ABF000C2F200031B88042B1BD14BF6AD44C0F6F8
:10AC0000000440F65453C2F200035B795AB240F696
:10AC1000FA03C2F200031B88042B02D14FF47843DD
:10AC200001E04FF6FF7310464FF0FE014FF06C024B
:10AC3000A04740F65453C2F200039A7940F2480309
:10AC4000C2F200039B7952B25BB29A421CD1FB79EB
:10AC5000002B19D140F6FA03C2F200031A8840F221
:10AC60001E03C2F200031B889A4229D040F6FA0361
:10AC7000C2F200031B88052B06D040F21E03C2F26D
:10AC800000031B88052B1BD14BF6AD44C0F6000416
:10AC900040F65453C2F200039B795AB240F6FA03CD
:10ACA000C2F200031B88052B02D14FF4784301E068
:10ACB0004FF6FF7310464FF487714FF06C02A047B8
:10ACC00040F65453C2F20003DA7940F24803C2F26C
:10ACD0000003DB7952B25BB29A421CD1FB79002BA4
:10ACE00019D140F6FA03C2F200031A8840F21E039B
:10ACF000C2F200031B889A4229D040F6FA03C2F23E
:10AD000000031B88062B06D040F21E03C2F200038C
:10AD10001B88062B1BD14BF6AD44C0F6000440F651
:10AD20005453C2F20003DB795AB240F6FA03C2F27E
:10AD300000031B88062B02D14FF4784301E04FF645
:10AD4000FF7310464FF48F714FF06C02A04740F232
:10AD50002803C2F200031A6840F60013C2F200038F
:10AD60001A6040F24800C2F2000040F65451C2F2AC
:10AD7000000107F0C9FC40F60413C2F200031A8870
:10AD800040F23003C2F200031B8812B21BB29A4297
:10AD90001ED1FB79002B1BD140F6FA03C2F200034F
:10ADA0001A8840F21E03C2F200031B889A4200F088
:10ADB000998040F6FA03C2F200031B88072B07D0E4
:10ADC00040F21E03C2F200031B88072B40F08A806A
:10ADD00040F60413C2F200031B881AB213464FEA6E
:10ADE00083039B184FEAC30340F65450C2F200009D
:10ADF00046F2F021C0F601011A4607F05DFC4FF063
:10AE0000020004F013FA40F6FA03C2F200031B88B2
:10AE1000072B02D14FF4784301E04FF6FF73184639
:10AE20004FF0000104F018FA4FF0C8004FF087010E
:10AE300004F0E4F94FF00003FB600EE040F65453D9
:10AE4000C2F20003FA689B181B78DBB2184604F0C4
:10AE500059F8FB6803F10103FB60FB68032BEDDD90
:10AE60004FF0000300934FF079004FF078014FF05E
:10AE700003024FF0640303F01FFE40F60413C2F216
:10AE800000031B881BB24FEAD372D3184FEA630347
:10AE90009BB21BB203F1780240F22C03C2F2000312
:10AEA0001B8819B240F60413C2F200031B881BB2C0
:10AEB000CB1A4FEAD371CB184FEA63034FF6FF71F9
:10AEC00000914FF0790011464FF0030203F0F4FDBA
:10AED00040F60413C2F200031A8840F23003C2F2B3
:10AEE00000031A8040F22C03C2F200031A8840F2D9
:10AEF0002E03C2F200031B8812B21BB29A421ED16B
:10AF0000FB79002B1BD140F6FA03C2F200031A882A
:10AF100040F21E03C2F200031B889A4200F099809F
:10AF200040F6FA03C2F200031B88082B07D040F258
:10AF30001E03C2F200031B88082B40F08A8040F2F7
:10AF40002C03C2F200031B881AB213464FEA830394
:10AF50009B184FEAC30340F65450C2F2000046F279
:10AF6000F421C0F601011A4607F0A6FB4FF00200DB
:10AF700004F05CF940F6FA03C2F200031B88082BC8
:10AF800002D14FF4784301E04FF6FF7318464FF0BB
:10AF9000000104F061F940F209104FF0870104F05C
:10AFA0002DF94FF00003BB600EE040F65453C2F29F
:10AFB0000003BA689B181B78DBB2184603F0A2FFA7
:10AFC000BB6803F10103BB60BB68032BEDDD4FF0F1
:10AFD000000300934FF079004FF078014FF0030227
:10AFE0004FF0640303F068FD40F60413C2F200035F
:10AFF0001B881BB24FEAD372D3184FEA63039BB28C
:10B000001BB203F1780240F22C03C2F200031B884A
:10B0100019B240F60413C2F200031B881BB2CB1A0C
:10B020004FEAD371CB184FEA63034FF6FF710091DB
:10B030004FF0790011464FF0030203F03DFD40F25E
:10B040002C03C2F200031A8840F22E03C2F200035E
:10B050001A8040F60613C2F200031A7840F2320357
:10B06000C2F200031B789A421CD1FB79002B19D144
:10B0700040F6FA03C2F200031A8840F21E03C2F23D
:10B0800000031B889A4279D040F6FA03C2F200030B
:10B090001B88092B06D040F21E03C2F200031B8856
:10B0A000092B6BD140F60613C2F200031B78012B6B
:10B0B00020D0022B3BD0002B56D140F6FA03C2F22F
:10B0C00000031B88092B02D14FF4784301E04FF6AF
:10B0D000FF734FF00902009201934FF0C4004FF04C
:10B0E0005B0146F2BC62C0F601024FF01C0303F0A4
:10B0F0007FFE39E040F6FA03C2F200031B88092BF9
:10B1000002D14FF4784301E04FF6FF734FF009028C
:10B11000009201934FF0C4004FF05B0146F6B40279
:10B12000C0F601024FF01C0303F062FE1CE040F683
:10B13000FA03C2F200031B88092B02D14FF47843B3
:10B1400001E04FF6FF734FF00902009201934FF0B8
:10B15000C4004FF05B0146F6AC22C0F601024FF08E
:10B160001C0303F045FE00BF40F60613C2F20003C5
:10B170001A7840F23203C2F200031A7040F2100350
:10B18000C2F200031B68184606F0F0FB02460B46AD
:10B190001046194612A3D3E9002306F03BFC0246F1
:10B1A0000B461046194610A3D3E9002306F09AFE79
:10B1B0000346002B09D140F6FA03C2F200031A88B5
:10B1C00040F21E03C2F200031A8040F61813C2F2C6
:10B1D00000034FF000021A7007F11407BD4690BD3E
:10B1E000AE47E17A14AEEF3F00000000000000001F
:10B1F000B0B586B000AF40F61013C2F200031B6872
:10B20000002B05D048F23853C0F601037B6104E0FF
:10B2100048F23863C0F601037B6142F60800C2F2CF
:10B22000000040F64411C2F200014FF4807205F0B4
:10B23000A3FDDFF83C343B61DFF83834FB604FF0AE
:10B240000103FB722DE0FA7A40F64413C2F20003C8
:10B250004FEA82029B181B687B6097ED017AD7ED5D
:10B26000047AB4EEE77AF1EE10FAD4BF002301239A
:10B27000DBB2002B01D07B683B6197ED017AD7ED03
:10B28000037AB4EEE77AF1EE10FA54BF00230123FB
:10B29000DBB2002B01D07B68FB60FB7A03F101037A
:10B2A000FB72FB7AFF2BCED140F64453C2F200036F
:10B2B000D3ED007A97ED047AB4EEE77AF1EE10FA66
:10B2C000D4BF00230123DBB2002B27D040F6445328
:10B2D000C2F200031B68184606F048FB04460D4600
:10B2E000386906F043FB02460B4610461946D8A3C0
:10B2F000D3E9002306F08EFB02460B462046294682
:10B3000006F0D6F902460B461046194606F044FEF2
:10B31000024640F64453C2F200031A6040F644531A
:10B32000C2F200031B68184606F020FB02460B46DB
:10B3300043EC102B05F002FE53EC102B104619467F
:10B34000C5A3D3E9002306F08FFC02460B46104646
:10B35000194606F021FE024640F64853C2F20003A9
:10B360001A6040F64453C2F200031B68184606F008
:10B37000FDFA02460B4610461946B9A3D3E900234D
:10B3800006F048FB02460B461046194606F004FE3E
:10B39000024640F64453C2F200031A6040F644539A
:10B3A000C2F2000393ED007A40F23403C2F20003CC
:10B3B000D3ED007AB4EEE77AF1EE10FAD4BF0023B1
:10B3C0000123DBB2002B09D040F23403C2F20003A8
:10B3D0001A6840F64453C2F200031A6040F6445320
:10B3E000C2F2000393ED007A40F23803C2F2000388
:10B3F000D3ED007AB4EEE77AF1EE10FA54BF0023F1
:10B400000123DBB2002B09D040F23803C2F2000363
:10B410001A6840F64453C2F200031A6040F64C53D7
:10B42000C2F200031B781A4640F64C53C2F20003E6
:10B430001B7810464FF000011A464FF0780302F0D7
:10B4400017FF4FF07803FB725EE0FA7A40F6441380
:10B45000C2F200034FEA82029B1893ED007AF7EEE6
:10B46000007A77EE277A17EE900A06F07FFA024606
:10B470000B4643EC102B05F061FD53EC102B1046EE
:10B48000194675A3D3E9002306F0EEFB02460B46EE
:10B4900014461D4640F64453C2F200031B6818468A
:10B4A00006F064FA02460B462046294606F0DCFB0D
:10B4B00002460B46104619466BA3D3E9002306F05B
:10B4C000A9FA02460B461046194606F065FD0246EB
:10B4D00040F65053C2F200031A6040F65053C2F2D5
:10B4E0000003D3ED007AFCEEE77A17EE903ADBB278
:10B4F0004FEA43037A69D3181B88184602F000FF0D
:10B50000FB7A03F1FF33FB72FB7A002B9DD140F6EF
:10B510004C53C2F200031B781A4640F64C53C2F259
:10B5200000031B7810464FF078011A464FF0EF03E6
:10B5300002F09EFE4FF0FF03FB725EE0FA7A40F6E7
:10B540004413C2F200034FEA82029B1893ED007A83
:10B55000F7EE007A77EE277A17EE900A06F006FAF1
:10B5600002460B4643EC102B05F0E8FC53EC102B85
:10B570001046194638A3D3E9002306F075FB0246AE
:10B580000B4614461D4640F64453C2F200031B68A6
:10B59000184606F0EBF902460B462046294606F00F
:10B5A00063FB02460B46104619462FA3D3E900233E
:10B5B00006F030FA02460B461046194606F0ECFC3F
:10B5C000024640F65053C2F200031A6040F6505350
:10B5D000C2F20003D3ED007AFCEEE77A17EE903A60
:10B5E000DBB24FEA43037A69D3181B88184602F08E
:10B5F00087FEFB7A03F1FF33FB72FB7A872B9DD822
:10B6000040F64C53C2F200031B7803F10103DAB297
:10B6100040F64C53C2F200031A7040F64C53C2F28B
:10B6200000031B78772B06D940F64C53C2F2000377
:10B630004FF000021A7040F64C53C2F200031B7820
:10B64000184603F071F907F11807BD46B0BD00BFF9
:10B650009A9999999999B93FEF39FAFE422EE63FA6
:10B66000AE47E17A14AEEF3F000000000000594001
:10B67000000000000000C84280B485B000AF7860D0
:10B6800039604FF00003FB600AE0FB684FEA830378
:10B690003A68D3180B4A1A60FB6803F10103FB6098
:10B6A000FA6840F2FF139A42EFDD7B684FEA8303AA
:10B6B0003A68D318044A1A6007F11407BD4680BCE3
:10B6C000704700BF000000000000803F80B588B0D8
:10B6D00000AF40F6D163C2F200031B78DBB2002B4F
:10B6E00000F0648240F61C13C2F200031B68012BB9
:10B6F00040F0FE8040F61413C2F200031B68002BDA
:10B7000078D13B4618464FF480714FF000024FF05D
:10B71000010303F0C9FD3B46184643F20C01C2F297
:10B72000000105F0BDF940F61013C2F200031B68DA
:10B73000002B25D140F62813C2F200031B78012B01
:10B740001ED04FF00003FB8315E0F98BFA8B43F218
:10B750000C03C2F200034FEA82029B181A6842F6F9
:10B760000803C2F200034FEA81015B181A60FB8BE9
:10B7700003F10103FB83FA8B40F2FF139A42E4D9F1
:10B7800040F60C13C2F200031B6843F20C00C2F235
:10B7900000001946FCF700FF40F61013C2F2000348
:10B7A0001B68012B32D140F62813C2F200031B782C
:10B7B000012B2BD04FF00003BB8315E0B98BBA8B64
:10B7C00043F20C03C2F200034FEA82029B181A688C
:10B7D00042F60803C2F200034FEA81015B181A60C7
:10B7E000BB8B03F10103BB83BA8B40F2FF139A4278
:10B7F000E4D90BE040F61413C2F200031B681846AC
:10B8000043F20C01C2F20001FFF736FF3B46184637
:10B810004FF480714FF001024FF0010303F044FD3B
:10B820003B46184643F20C01C2F2000105F038F91C
:10B8300040F60613C2F200031B78022B40D143F2FC
:10B840000C00C2F2000043F60C01C2F200014FF4FA
:10B85000807205F091FA4FF000037B832DE07B8B23
:10B860004FEA43017A8B43F60C03C2F200034FEA1E
:10B8700082029B181A6843F20C03C2F200034FEADB
:10B8800081015B181A607B8B4FEA430303F10101CE
:10B890007A8B43F60C03C2F200034FEA82029B1834
:10B8A0001A6843F20C03C2F200034FEA81015B18ED
:10B8B0001A607B8B03F101037B837B8BFF2BCED93B
:10B8C00043F20C00C2F200004FF40071FEF724FFB7
:10B8D000F0EE407A40F63013C2F20003C3ED007A76
:10B8E00040F61C13C2F200034FF000021A6056E14A
:10B8F00040F62013C2F200031B68012B40F0A48025
:10B9000040F61413C2F200031B68002B1ED13B4605
:10B9100018464FF480714FF000024FF0010303F01E
:10B92000C3FC3B46184641F2E071C2F2000105F04B
:10B93000B7F840F60C13C2F200031B6841F2E07046
:10B94000C2F200001946FCF727FE0BE040F6141384
:10B95000C2F200031B68184641F2E071C2F2000116
:10B96000FFF78AFE3B4618464FF480714FF0010204
:10B970004FF0010303F098FC3B46184641F2E0719A
:10B98000C2F2000105F08CF840F60613C2F2000383
:10B990001B78022B40D141F2E070C2F2000043F666
:10B9A0000C01C2F200014FF4807205F0E5F94FF08E
:10B9B00000033B832DE03B8B4FEA43013A8B43F678
:10B9C0000C03C2F200034FEA82029B181A6841F28C
:10B9D000E073C2F200034FEA81015B181A603B8BEF
:10B9E0004FEA430303F101013A8B43F60C03C2F221
:10B9F00000034FEA82029B181A6841F2E073C2F218
:10BA000000034FEA81015B181A603B8B03F10103CD
:10BA10003B833B8BFF2BCED941F2E070C2F200009A
:10BA20004FF40071FEF778FEF0EE407A40F63013E6
:10BA3000C2F20003C3ED007A40F62013C2F2000305
:10BA40004FF000021A60AAE040F62413C2F200038D
:10BA50001B68012B40F0A38040F61413C2F20003D0
:10BA60001B68002B1ED13B4618464FF480714FF0E7
:10BA700000024FF0010303F017FC3B46184642F268
:10BA80000001C2F2000105F00BF840F60C13C2F2FF
:10BA900000031B6842F20000C2F200001946FCF7E6
:10BAA0007BFD0BE040F61413C2F200031B6818463E
:10BAB00042F20001C2F20001FFF7DEFD3B461846EC
:10BAC0004FF480714FF001024FF0010303F0ECFBE3
:10BAD0003B46184642F20001C2F2000104F0E0FFCA
:10BAE00040F60613C2F200031B78022B40D142F24B
:10BAF0000000C2F2000043F60C01C2F200014FF454
:10BB0000807205F039F94FF00003FB822DE0FB8ACB
:10BB10004FEA4301FA8A43F60C03C2F200034FEAEC
:10BB200082029B181A6842F20003C2F200034FEA35
:10BB300081015B181A60FB8A4FEA430303F101019C
:10BB4000FA8A43F60C03C2F200034FEA82029B1802
:10BB50001A6842F20003C2F200034FEA81015B1847
:10BB60001A60FB8A03F10103FB82FB8AFF2BCED90B
:10BB700042F20000C2F200004FF40071FEF7CCFD6B
:10BB8000F0EE407A40F63013C2F20003C3ED007AC3
:10BB900040F62413C2F200034FF000021A6040F690
:10BBA000D163C2F200034FF000021A7040F68460C5
:10BBB000C2F20000F5F7B8F907F12007BD4680BDD5
:10BBC00080B500AFFCF786FF024644F28C03C2F258
:10BBD00000031A6044F28C03C2F200031A6843F2B5
:10BBE0000803C2F200031B689A424AD043F20803DA
:10BBF000C2F200031A6844F28C03C2F200031B680D
:10BC0000D31A1A4640F22403C2F200031B6803FB56
:10BC100002F240F22803C2F200031B68D3181A464E
:10BC200040F22803C2F200031A6040F22803C2F275
:10BC300000031B68002B06DC40F22803C2F200035D
:10BC40004FF001021A6040F22803C2F200031A68A2
:10BC500043F26043C0F23C239A4208DD40F22803DD
:10BC6000C2F2000343F26042C0F23C221A6044F286
:10BC70008C03C2F200031A6843F20803C2F2000305
:10BC80001A6040F22803C2F200031A6840F600135B
:10BC9000C2F200031B689A4207D040F22803C2F2A6
:10BCA00000031B68184601F07FFB80BD80B584B09F
:10BCB00002AFF871B9807A803B8097F90730A3F121
:10BCC0002E030B2B00F2E28001A252F823F000BFFA
:10BCD00001BD00088DBE000869BE000825BD000832
:10BCE00049BD00086DBD000891BD0008B5BD000844
:10BCF000D9BD0008FDBD000821BE000845BE0008F2
:10BD0000BA887B8839884FF0130000900191104663
:10BD1000194646F6A442C0F601024FF00F0303F0A5
:10BD200067F8C0E0BA887B8839884FF0130000902C
:10BD300001911046194646F6E062C0F601024FF046
:10BD40000F0303F055F8AEE0BA887B8839884FF0CE
:10BD50001300009001911046194647F21C12C0F6DC
:10BD600001024FF00F0303F043F89CE0BA887B8890
:10BD700039884FF01300009001911046194647F2A0
:10BD80005832C0F601024FF00F0303F031F88AE099
:10BD9000BA887B8839884FF01300009001911046D3
:10BDA000194647F29452C0F601024FF00F0303F018
:10BDB0001FF878E0BA887B8839884FF0130000902C
:10BDC00001911046194647F2D072C0F601024FF0B9
:10BDD0000F0303F00DF866E0BA887B8839884FF0CE
:10BDE0001300009001911046194647F60C22C0F648
:10BDF00001024FF00F0302F0FBFF54E0BA887B888A
:10BE000039884FF01300009001911046194647F60B
:10BE10004842C0F601024FF00F0302F0E9FF42E092
:10BE2000BA887B8839884FF0130000900191104642
:10BE3000194647F68462C0F601024FF00F0302F084
:10BE4000D7FF30E0BA887B8839884FF01300009024
:10BE500001911046194648F2C002C0F601024FF0A7
:10BE60000F0302F0C5FF1EE0BA887B8839884FF0C7
:10BE70001300009001911046194648F2FC22C0F6CA
:10BE800001024FF00F0302F0B3FF0CE0BA887B8889
:10BE90004FF000010091104619464FF00F024FF08D
:10BEA000130302F009FE07F10807BD4680BD00BF7D
:10BEB00080B500AF40F20C03C2F200031A684DF6E1
:10BEC0002913C6F24263A3FB02134FEA136303F183
:10BED000FF3240F63813C2F200031A604FF4605389
:10BEE000C4F202034FF46052C4F20202126C42F038
:10BEF00002021A6440F63C73C2F200034FF48062FF
:10BF0000C4F200021A6040F63C73C2F200034FF024
:10BF100000029A6040F63C73C2F2000340F21A42FB
:10BF2000DA6040F63813C2F200031A6840F63C7338
:10BF3000C2F200035A6040F63C73C2F200034FF0B5
:10BF400000021A6140F63C70C2F20000F4F754FDA2
:10BF500040F63C70C2F20000F4F72CFE4FF01D00DA
:10BF60004FF000014FF00102FBF7C2F94FF01D0046
:10BF7000FBF7F2F94FF46053C4F202034FF460523E
:10BF8000C4F20202126C42F004021A6440F68463A6
:10BF9000C2F200034FF40062C4F200021A6040F6DD
:10BFA0008463C2F200034FF000029A6040F684639B
:10BFB000C2F2000340F21A42DA6040F63813C2F2CD
:10BFC00000031A6840F68463C2F200035A6040F628
:10BFD0008463C2F200034FF000021A6140F68460ED
:10BFE000C2F20000F4F708FD40F68460C2F20000DF
:10BFF000F4F7E0FD4FF01E004FF002014FF0040295
:10C00000FBF776F94FF01E00FBF7A6F980BD00BFE5
:10C0100080B582B000AF7860FCF76EFD07F10807CD
:10C02000BD4680BD80B500AF4FF46053C4F202033B
:10C030004FF46052C4F20202126C42F000521A64D1
:10C0400044F26403C2F200034FF4E842C4F2000277
:10C050001A6044F26400C2F20000FAF74FFE034691
:10C06000002B01D0FCF7CAFB40F63C13C2F20003E0
:10C070004FF000021A6040F63C13C2F200034FF08A
:10C0800000025A6044F26400C2F2000040F63C1123
:10C09000C2F200014FF00002FAF7EEFE0346002B59
:10C0A00001D0FCF7ABFB44F26400C2F2000040F6A2
:10C0B0003C11C2F200014FF01002FAF7DDFE034618
:10C0C000002B01D0FCF79AFB44F26400C2F200009E
:10C0D0004FF000014FF000024FF08803FAF7A2FF83
:10C0E0000346002B01D0FCF789FB44F26400C2F246
:10C0F00000004FF010014FF000024FF08803FAF7F4
:10C1000091FF0346002B01D0FCF778FB44F264005A
:10C11000C2F200004FF00001FAF730FE0346002B98
:10C1200001D0FCF76BFB44F26400C2F200004FF058
:10C130001001FAF723FE0346002B01D0FCF75EFB4B
:10C1400080BD00BF80B582B000AF0346FB80FB8896
:10C150004FEA03534FEA1353FB80FB8844F2640019
:10C16000C2F200004FF000014FF00002FAF75AFF50
:10C1700007F10807BD4680BD80B582B000AF034619
:10C18000FB80FB884FEA03534FEA1353FB80FB8885
:10C1900044F26400C2F200004FF010014FF00002C0
:10C1A000FAF740FF07F10807BD4680BD80B483B0B1
:10C1B00000AF786040F68063C2F200037A681A60CC
:10C1C00000BF40F68063C2F200031B68002BF8D169
:10C1D00007F10C07BD4680BC704700BF80B586B034
:10C1E00000AF4AF2E873C0F601039B887B604FF012
:10C1F00002033B614FF00203BB604FF00203FB60A0
:10C200004FF001037B614AF2E873C0F601031A683C
:10C2100007F1040310461946F6F786FA4AF2F0735E
:10C22000C0F601039B887B604FF002033B614FF037
:10C230000203BB604FF00203FB604FF001037B6120
:10C240004AF2F073C0F601031A6807F104031046BE
:10C250001946F6F769FA4AF60003C0F601039B880F
:10C260007B604FF002033B614FF00103BB604FF076
:10C2700000037B614FF00003FB604AF60003C0F649
:10C2800001031A6807F1040310461946F6F74CFA41
:10C290004AF60803C0F601039B887B604FF0020357
:10C2A0003B614FF00103BB604FF000037B614FF037
:10C2B0000003FB604AF60803C0F601031A6807F1A1
:10C2C000040310461946F6F72FFA4AF61803C0F68B
:10C2D00001039B887B604FF000033B614FF011032B
:10C2E000BB604FF000037B614FF00003FB604AF638
:10C2F0001803C0F601031A6807F104031046194633
:10C30000F6F712FA4AF61803C0F601031A684AF65D
:10C310001803C0F601039B88104619464FF000022F
:10C32000F6F7DCFD4AF2F873C0F601039B887B60E8
:10C330004FF002033B614FF00303BB604FF000037B
:10C34000FB604FF000037B614AF2F873C0F6010313
:10C350001A6807F1040310461946F6F7E5F94AF69C
:10C360007803C0F601039B887B604FF002033B61BA
:10C370004FF00003BB604FF00103FB604FF0000380
:10C380007B614AF67803C0F601031A6807F10403DB
:10C3900010461946F6F7C8F94AF68003C0F60103BD
:10C3A0009B887B604FF002033B614FF00003BB6052
:10C3B0004FF00103FB604FF000037B614AF68003FE
:10C3C000C0F601031A6807F1040310461946F6F790
:10C3D000ABF94AF68803C0F601039B887B604FF0F7
:10C3E00002033B614FF00003BB604FF00103FB60B1
:10C3F0004FF000037B614AF68803C0F601031A6818
:10C4000007F1040310461946F6F78EF94AF6900331
:10C41000C0F601039B887B604FF002033B614FF045
:10C420000303BB604FF00003FB604FF000037B6130
:10C430004AF69003C0F601031A6807F10403104698
:10C440001946F6F771F94AF69803C0F601039B887E
:10C450007B604FF002033B614FF00303BB604FF082
:10C460000003FB604FF000037B614AF69803C0F6BF
:10C4700001031A6807F1040310461946F6F754F948
:10C480004AF62003C0F601039B887B604FF001034E
:10C49000BB604FF002033B614FF00103FB604AF6C3
:10C4A0002003C0F601031A6807F104031046194679
:10C4B000F6F73AF94AF62003C0F601031A684AF67D
:10C4C0002003C0F601039B88104619464FF0000276
:10C4D000F6F704FD4AF62803C0F601039B887B604B
:10C4E0004FF00103BB604FF002033B614FF00103CB
:10C4F000FB604AF62803C0F601031A6807F104033B
:10C5000010461946F6F710F94AF62803C0F601035B
:10C510001A684AF62803C0F601039B88104619469C
:10C520004FF00002F6F7DAFC4AF63003C0F60103DA
:10C530009B887B604FF00103BB604FF002033B61BF
:10C540004FF00103FB604AF63003C0F601031A689E
:10C5500007F1040310461946F6F7E6F84AF63003E9
:10C56000C0F601031A684AF63003C0F601039B883F
:10C57000104619464FF00002F6F7B0FC4AF64003A9
:10C58000C0F601039B887B604FF00103BB604FF056
:10C5900002033B614FF00103FB604AF64003C0F623
:10C5A00001031A6807F1040310461946F6F7BCF8B0
:10C5B0004AF64003C0F601031A684AF64003C0F683
:10C5C00001039B88104619464FF00102F6F786FCDE
:10C5D0004AF63803C0F601039B887B604FF00103E5
:10C5E000BB604FF002033B614FF00103FB604AF672
:10C5F0003803C0F601031A6807F104031046194610
:10C60000F6F792F84AF63803C0F601031A684AF6BC
:10C610003803C0F601039B88104619464FF001020B
:10C62000F6F75CFC4AF64803C0F601039B887B6082
:10C630004FF00103BB604FF002033B614FF0010379
:10C64000FB604AF64803C0F601031A6807F10403C9
:10C6500010461946F6F768F84AF64803C0F6010393
:10C660001A684AF64803C0F601039B88104619462B
:10C670004FF00002F6F732FC4AF65803C0F6010309
:10C680009B887B604FF00103BB604FF002033B616E
:10C690004FF00103FB604AF65803C0F601031A6825
:10C6A00007F1040310461946F6F73EF84AF6580318
:10C6B000C0F601031A684AF65803C0F601039B88C6
:10C6C000104619464FF00102F6F708FC4AF65003EF
:10C6D000C0F601039B887B604FF00103BB604FF005
:10C6E00002033B614FF00103FB604AF65003C0F6C2
:10C6F00001031A6807F1040310461946F6F714F807
:10C700004AF65003C0F601031A684AF65003C0F611
:10C7100001039B88104619464FF00102F6F7DEFB35
:10C720004AF6A003C0F601039A884AF6A803C0F6A9
:10C7300001039B8813439BB27B604FF00303BB60F4
:10C740004FF00003FB604AF6A003C0F601031A682D
:10C7500007F1040310461946F5F7E6FF4AF6B00361
:10C76000C0F601039B887B604FF00103BB604FF074
:10C7700000033B614FF00003FB604AF6B003C0F6D4
:10C7800001031A6807F1040310461946F5F7CCFFB8
:10C790004AF6B003C0F601031A684AF6B003C0F6C1
:10C7A00001039B88104619464FF00102F6F796FBED
:10C7B0004AF6B803C0F601039B887B604FF0010383
:10C7C000BB604FF000033B614FF00003FB604AF693
:10C7D000B803C0F601031A6807F1040310461946AE
:10C7E000F5F7A2FF4AF6B803C0F601031A684AF645
:10C7F000B803C0F601039B88104619464FF00002AB
:10C80000F6F76CFB4AF6C003C0F601039B887B6019
:10C810004FF00103BB604FF000033B614FF000039A
:10C82000FB604AF6C003C0F601031A6807F104036F
:10C8300010461946F5F778FF4AF6C003C0F6010323
:10C840001A684AF6C003C0F601039B8810461946D1
:10C850004FF00002F6F742FB4AF6C803C0F60103A8
:10C860009B887B604FF00103BB604FF000033B618E
:10C870004FF00003FB604AF6C803C0F601031A68D4
:10C8800007F1040310461946F5F74EFF4AF6C803B0
:10C89000C0F601031A684AF6C803C0F601039B8874
:10C8A000104619464FF00102F6F718FB4AF6D0037E
:10C8B000C0F601039B887B604FF00103BB604FF023
:10C8C00000033B614FF00003FB604AF6D003C0F663
:10C8D00001031A6807F1040310461946F5F724FF0F
:10C8E0004AF6D003C0F601031A684AF6D003C0F630
:10C8F00001039B88104619464FF00002F6F7EEFA46
:10C900004AF60813C0F601039B887B604FF00103D1
:10C91000BB604FF000033B614FF00003FB604AF641
:10C920000813C0F601031A6807F1040310461946FC
:10C93000F5F7FAFE4AF60813C0F601031A684AF63C
:10C940000813C0F601039B88104619464FF00102F8
:10C95000F6F7C4FA4AF61013C0F601039B887B6011
:10C960004FF00103BB604FF000033B614FF0000349
:10C97000FB604AF61013C0F601031A6807F10403BE
:10C9800010461946F5F7D0FE4AF61013C0F601031B
:10C990001A684AF61013C0F601039B881046194620
:10C9A0004FF00002F6F79AFA4AF6F803C0F60103D0
:10C9B0009B887B604FF00103BB604FF000033B613D
:10C9C0004FF00003FB604AF6F803C0F601031A6853
:10C9D00007F1040310461946F5F7A6FE4AF6F803D8
:10C9E000C0F601031A684AF6F803C0F601039B88F3
:10C9F000104619464FF00002F6F770FA4AF6001397
:10CA0000C0F601039B887B604FF00103BB604FF0D1
:10CA100000033B614FF00003FB604AF60013C0F6D1
:10CA200001031A6807F1040310461946F5F77CFE66
:10CA30004AF60013C0F601031A684AF60013C0F65E
:10CA400001039B88104619464FF00102F6F746FA9B
:10CA50004AF6E803C0F601039B887B604FF00103B0
:10CA6000BB604FF000033B614FF00003FB604AF6F0
:10CA7000E803C0F601031A6807F1040310461946DB
:10CA8000F5F752FE4AF6E803C0F601031A684AF6C3
:10CA9000E803C0F601039B88104619464FF00002D8
:10CAA000F6F71CFA4AF6F003C0F601039B887B6098
:10CAB0004FF00103BB604FF000033B614FF00003F8
:10CAC000FB604AF6F003C0F601031A6807F104039D
:10CAD00010461946F5F728FE4AF6F003C0F60103A2
:10CAE0001A684AF6F003C0F601039B8810461946FF
:10CAF0004FF00102F6F7F2F94AF6D803C0F6010347
:10CB00009B887B604FF00103BB604FF000033B61EB
:10CB10004FF00003FB604AF6D803C0F601031A6821
:10CB200007F1040310461946F5F7FEFD4AF6D8034F
:10CB3000C0F601031A684AF6D803C0F601039B88C1
:10CB4000104619464FF00002F6F7C8F94AF6E0031E
:10CB5000C0F601039B887B604FF00103BB604FF080
:10CB600000033B614FF00003FB604AF6E003C0F6B0
:10CB700001031A6807F1040310461946F5F7D4FDBE
:10CB80004AF6E003C0F601031A684AF6E003C0F66D
:10CB900001039B88104619464FF00102F6F79EF9F3
:10CBA0004AF62013C0F601039B887B604FF0110307
:10CBB000BB604FF000033B614FF00103FB604AF69E
:10CBC0002013C0F601031A6807F104031046194642
:10CBD000F5F7AAFD4AF62013C0F601031A684AF6D3
:10CBE0002013C0F601039B88104619464FF001023E
:10CBF000F6F774F94AF61813C0F601039B887B60B8
:10CC00004FF01103BB604FF000033B614FF0010395
:10CC1000FB604AF61813C0F601031A6807F1040313
:10CC200010461946F5F780FD4AF61813C0F60103C1
:10CC30001A684AF61813C0F601039B881046194675
:10CC40004FF00102F6F74AF94AF63013C0F6010335
:10CC50009B887B604FF00103BB604FF000033B619A
:10CC60004FF00003FB604AF63013C0F601031A6868
:10CC700007F1040310461946F5F756FD4AF630133E
:10CC8000C0F601031A684AF63013C0F601039B8808
:10CC9000104619464FF00102F6F720F94AF628131C
:10CCA000C0F601039B887B604FF00103BB604FF02F
:10CCB00000033B614FF00003FB604AF62813C0F607
:10CCC00001031A6807F1040310461946F5F72CFD15
:10CCD0004AF62813C0F601031A684AF62813C0F66C
:10CCE00001039B88104619464FF00102F6F7F6F84B
:10CCF0004AF63813C0F601039B887B604FF00103AE
:10CD0000BB604FF000033B614FF00003FB604AF64D
:10CD10003813C0F601031A6807F1040310461946D8
:10CD2000F5F702FD4AF63813C0F601031A684AF611
:10CD30003813C0F601039B88104619464FF00102D4
:10CD4000F6F7CCF84AF64013C0F601039B887B60E7
:10CD50004FF00103BB604FF000033B614FF0000355
:10CD6000FB604AF64013C0F601031A6807F104039A
:10CD700010461946F5F7D8FC4AF64013C0F60103F1
:10CD80001A684AF64013C0F601039B8810461946FC
:10CD90004FF00102F6F7A2F84AF65013C0F601036D
:10CDA0009B887B604FF00103BB604FF000033B6149
:10CDB0004FF00003FB604AF65013C0F601031A68F7
:10CDC00007F1040310461946F5F7AEFC4AF6501376
:10CDD000C0F601031A684AF65013C0F601039B8897
:10CDE000104619464FF00102F6F778F84AF6481354
:10CDF000C0F601039B887B604FF00103BB604FF0DE
:10CE000000033B614FF00003FB604AF64813C0F695
:10CE100001031A6807F1040310461946F5F784FC6C
:10CE20004AF64813C0F601031A684AF64813C0F6DA
:10CE300001039B88104619464FF00102F6F74EF8A1
:10CE40004AF65813C0F601039B887B604FF003033A
:10CE5000BB604FF000033B614FF00003FB604AF6FC
:10CE60005813C0F601031A6807F104031046194667
:10CE7000F5F75AFC4AF65813C0F601031A684AF649
:10CE80005813C0F601039B88104619464FF0000264
:10CE9000F6F724F84AF66013C0F601039B887B601E
:10CEA0004FF00303BB604FF000033B614FF0000302
:10CEB000FB604AF66013C0F601031A6807F1040329
:10CEC00010461946F5F730FC4AF66813C0F6010320
:10CED0009B887B604FF00103BB604FF000033B6118
:10CEE0004FF00003FB604AF66813C0F601031A68AE
:10CEF00007F1040310461946F5F716FC4AF66813C5
:10CF0000C0F601031A684AF66813C0F601039B884D
:10CF1000104619464FF00102F5F7E0FF4AF670138C
:10CF2000C0F601039B887B604FF00103BB604FF0AC
:10CF300000033B614FF00003FB604AF67013C0F63C
:10CF400001031A6807F1040310461946F5F7ECFBD4
:10CF50004AF67013C0F601031A684AF67013C0F659
:10CF600001039B88104619464FF00102F5F7B6FF02
:10CF70004AF68813C0F601039B887B604FF00003DC
:10CF8000BB604FF000033B614FF00103FB604AF6CA
:10CF90008813C0F601031A6807F104031046194606
:10CFA000F5F7C2FB4AF69013C0F601039B887B603D
:10CFB0004FF00003BB604FF000033B614FF00103F3
:10CFC000FB604AF69013C0F601031A6807F10403E8
:10CFD00010461946F5F7A8FB4AF67813C0F6010388
:10CFE0009B887B604FF00003BB604FF000033B6108
:10CFF0004FF00003FB604AF67813C0F601031A688D
:10D0000007F1040310461946F5F78EFB4AF6801324
:10D01000C0F601039B887B604FF00003BB604FF0BC
:10D0200000033B614FF00003FB604AF68013C0F63B
:10D0300001031A6807F1040310461946F5F774FB5B
:10D040004AF6B013C0F601039B887B604FF00003E3
:10D050003B614FF00103BB604FF00103FB604AF6F8
:10D06000B013C0F601031A6807F10403104619460D
:10D07000F5F75AFB4AF6B013C0F601031A684AF6F0
:10D08000B013C0F601039B88104619464FF000020A
:10D09000F5F724FF4AF69813C0F601039B887B60DE
:10D0A0004FF000033B614FF00103BB604FF0000302
:10D0B000FB604AF69813C0F601031A6807F10403EF
:10D0C00010461946F5F730FB4AF69813C0F60103EF
:10D0D0001A684AF69813C0F601039B881046194651
:10D0E0004FF00102F5F7FAFE4AF6A013C0F601036D
:10D0F0009B887B604FF000033B614FF00003BB60F7
:10D100004FF00003FB604AF6A013C0F601031A6853
:10D1100007F1040310461946F5F706FB4AF6A81373
:10D12000C0F601039B887B604FF000033B614FF02A
:10D130000003BB604FF00003FB604AF6A813C0F683
:10D1400001031A6807F1040310461946F5F7ECFAD3
:10D1500007F11807BD4680BD80B500AF4AF6400311
:10D16000C0F601031A684AF64003C0F601039B8823
:10D17000104619464FF00102F5F7B0FE4AF6580383
:10D18000C0F601031A684AF65803C0F601039B88EB
:10D19000104619464FF00102F5F7A0FE4AF6380393
:10D1A000C0F601031A684AF63803C0F601039B88EB
:10D1B000104619464FF00002F5F790FE4AF650036C
:10D1C000C0F601031A684AF65003C0F601039B88B3
:10D1D000104619464FF00002F5F780FE80BD00BFF3
:10D1E00080B584B000AF02460B46FA80BB804FF09A
:10D1F0000003FB6075E04AF63003C0F601031968CE
:10D200004AF63003C0F601039A88F888FB68C3F138
:10D210000F0340FA03F3DBB203F00103DBB208466D
:10D2200011461A46F5F75AFE4AF64803C0F60103BE
:10D2300019684AF64803C0F601039A88B888FB6863
:10D24000C3F10F0340FA03F3DBB203F00103DBB2D7
:10D25000084611461A46F5F741FE4AF64003C0F665
:10D2600001031A684AF64003C0F601039B88104682
:10D2700019464FF00002F5F731FE4AF65803C0F6A2
:10D2800001031A684AF65803C0F601039B8810464A
:10D2900019464FF00002F5F721FE4AF64003C0F6AA
:10D2A00001031A684AF64003C0F601039B88104642
:10D2B00019464FF00102F5F711FE4AF65803C0F681
:10D2C00001031A684AF65803C0F601039B8810460A
:10D2D00019464FF00102F5F701FEFB6803F1010367
:10D2E000FB60FB680F2B86DD07F11007BD4680BD94
:10D2F00080B500AF4AF63803C0F601031A684AF653
:10D300003803C0F601039B88104619464FF001020E
:10D31000F5F7E4FD4AF65003C0F601031A684AF631
:10D320005003C0F601039B88104619464FF00102D6
:10D33000F5F7D4FD80BD00BF80B588B000AFC7E968
:10D34000000117A3D3E90023C7E906234FF0805259
:10D350004FF00003C7E904237B683A6902FB03F23C
:10D360007B69396801FB03F3D1183A683B69A2FB7A
:10D370000323C9180B46C7E90223C7E90223D7E9EB
:10D380000201D7E9062304F057FE02460B46104679
:10D39000194607F12007BD4680BD00BFAFF30080EE
:10D3A000C0687804000000002DE9B04384B000AFED
:10D3B000786079680A464FEAE27310461946FFF72B
:10D3C000BBFF02460B46C7E902234AF62003C0F61C
:10D3D00001031A684AF62003C0F601039B88104631
:10D3E00019464FF00102F5F779FDFFF7B5FE4FF44E
:10D3F00008504FF40851FFF7F3FEFFF779FF4AF6A4
:10D400002003C0F601031A684AF62003C0F60103A0
:10D410009B88104619464FF00102F5F75FFDFFF7B4
:10D420009BFE3B894FEA83434FEA93439BB243F40D
:10D4300080439BB29AB23B894FEA83434FEA9343BE
:10D440009BB243F480439BB29BB210461946FFF750
:10D45000C7FEFFF74DFFFFF77FFEFB684FEA8343F0
:10D46000BA684FEA923843EA0808FB684FEAA339E2
:10D470001FFA88F34FEA83434FEA93439BB243F486
:10D4800080439BB29AB2FB684FEA8343B9684FEA84
:10D4900091341C43FB684FEAA335A3B24FEA8343A0
:10D4A0004FEA93439BB243F480439BB29BB2104636
:10D4B0001946FFF795FEFFF71BFFFFF74DFE4FF4F0
:10D4C00040404FF44C41FFF78BFEFFF711FF4AF647
:10D4D0002003C0F601031A684AF62003C0F60103D0
:10D4E0009B88104619464FF00002F5F7F7FC07F14C
:10D4F0001007BD46BDE8B08380B500AF40F6A0532D
:10D50000C2F200034FF000021A8040F67C63C2F2C0
:10D5100000034FF000021A8040F63173C2F200039C
:10D520004FF000021A7040F63A73C2F200034FF057
:10D5300064021A8040F6D163C2F200034FF0000289
:10D540001A7040F6D063C2F200034FF000021A7066
:10D550004FF46053C4F202034FF46052C4F202026B
:10D56000526C42F480725A644FF46053C4F2020366
:10D570004FF46052C4F20202526C42F400725A64D8
:10D580004FF46053C4F202034FF46052C4F202023B
:10D59000526C42F480625A644FF46053C4F2020346
:10D5A0004FF46052C4F20202126B42F001021A639D
:10D5B0004FF46053C4F202034FF46052C4F202020B
:10D5C000126B42F002021A634FF46053C4F202037A
:10D5D0004FF46052C4F20202126B42F004021A636A
:10D5E0004FF46053C4F202034FF46052C4F20202DB
:10D5F000526A42F480725A624FF46053C4F20203DA
:10D600004FF46052C4F20202526A22F480725A62EB
:10D6100040F6F453C2F200034FF40052C4F2010288
:10D620001A6040F6F453C2F200034FF000025A6051
:10D6300040F6F453C2F200034FF000029A6040F645
:10D64000F453C2F200034FF000021A6140F6F453A3
:10D65000C2F200034FF001029A6140F6F453C2F2A5
:10D6600000034FF000025A6240F6F453C2F2000386
:10D670004FF000029A6240F6F453C2F200034FF0FA
:10D680000002DA6240F6F453C2F200034FF00002E7
:10D690001A6340F6F453C2F200034FF00002DA605E
:10D6A00040F6F453C2F200034FF001021A6240F652
:10D6B000F453C2F200034FF00002DA6140F6F45373
:10D6C000C2F200034FF000025A6140F6F450C2F279
:10D6D0000000F9F75DFE0346002B0CD040F6D06346
:10D6E000C2F200031B7803F10103DAB240F6D06303
:10D6F000C2F200031A7040F63863C2F200034FF41E
:10D700000452C4F201021A6040F63863C2F2000308
:10D710004FF000025A6040F63863C2F200034FF047
:10D7200000029A6040F63863C2F200034FF0000234
:10D730001A6140F63863C2F200034FF001029A61A9
:10D7400040F63863C2F200034FF000025A6240F61E
:10D750003863C2F200034FF000029A6240F6386369
:10D76000C2F200034FF00002DA6240F63863C2F200
:10D7700000034FF000021A6340F63863C2F2000360
:10D780004FF00002DA6040F63863C2F200034FF057
:10D7900001021A6240F63863C2F200034FF0000241
:10D7A000DA6140F63863C2F200034FF000025A61BA
:10D7B00040F63860C2F20000F9F7EAFD0346002B9C
:10D7C0000CD040F6D063C2F200031B7803F10103D2
:10D7D000DAB240F6D063C2F200031A7040F67873F2
:10D7E000C2F200034FF40852C4F201021A6040F67C
:10D7F0007873C2F200034FF000025A6040F678736B
:10D80000C2F200034FF000029A6040F67873C2F251
:10D8100000034FF000021A6140F67873C2F2000371
:10D820004FF001029A6140F67873C2F200034FF0A4
:10D8300000025A6240F67873C2F200034FF0000211
:10D840009A6240F67873C2F200034FF00002DA6287
:10D8500040F67873C2F200034FF000021A6340F6FC
:10D860007873C2F200034FF00002DA6040F678737A
:10D87000C2F200034FF001021A6240F67873C2F25E
:10D8800000034FF00002DA6140F67873C2F2000341
:10D890004FF000025A6140F67870C2F20000F9F7CA
:10D8A00077FD0346002B0CD040F6D063C2F2000394
:10D8B0001B7803F10103DAB240F6D063C2F2000331
:10D8C0001A7040F6A453C2F200034FF009021A6026
:10D8D00040F6A453C2F200034FF001025A6040F632
:10D8E000A453C2F200034FF000029A6040F6A45322
:10D8F000C2F200034FF00002DA6040F6BC73C2F2DD
:10D9000000034FF006021A6040F6BC73C2F2000337
:10D910004FF001025A6040F6BC73C2F200034FF0B0
:10D9200000029A6040F6BC73C2F200034FF000029E
:10D93000DA6040F6C063C2F200034FF003021A60DF
:10D9400040F6C063C2F200034FF001025A6040F695
:10D95000C063C2F200034FF000029A6040F6C06359
:10D96000C2F200034FF00002DA6040F6F450C2F257
:10D97000000040F6A451C2F20001F9F771FF03461E
:10D98000002B0CD040F6D063C2F200031B7803F1E9
:10D990000103DAB240F6D063C2F200031A7040F617
:10D9A0003860C2F2000040F6BC71C2F20001F9F723
:10D9B00057FF0346002B0CD040F6D063C2F20003A1
:10D9C0001B7803F10103DAB240F6D063C2F2000320
:10D9D0001A7040F67870C2F2000040F6C061C2F2E0
:10D9E0000001F9F73DFF0346002B0CD040F6D06351
:10D9F000C2F200031B7803F10103DAB240F6D063F0
:10DA0000C2F200031A7080BD80B500AF40F6F4503A
:10DA1000C2F200004FF00A01F9F7D2FE40F638607A
:10DA2000C2F200004FF00A01F9F7CAFE40F6787022
:10DA3000C2F200004FF00A01F9F7C2FE40F6F450BE
:10DA4000C2F20000FAF7C8F80346152B38D140F6A9
:10DA50003860C2F20000FAF7BFF80346152B2FD149
:10DA600040F67870C2F20000FAF7B6F80346152BBC
:10DA700026D140F6F450C2F20000F9F7E3FE034667
:10DA80009AB240F6A053C2F200031A8040F6386002
:10DA9000C2F20000F9F7D6FE03469AB240F67C6364
:10DAA000C2F200031A8040F67870C2F20000F9F763
:10DAB000C9FE03469AB240F62E73C2F200031A80E2
:10DAC00080BD00BF80B500AF40F6F450C2F2000048
:10DAD000F9F7D6FD0346002B0CD040F6D063C2F216
:10DAE00000031B7803F10103DAB240F6D063C2F2FF
:10DAF00000031A7040F63860C2F20000F9F7C0FD6A
:10DB00000346002B0CD040F6D063C2F200031B7812
:10DB100003F10103DAB240F6D063C2F200031A70D7
:10DB200040F67870C2F20000F9F7AAFD0346002B18
:10DB30000CD040F6D063C2F200031B7803F101035E
:10DB4000DAB240F6D063C2F200031A7080BD00BFA3
:10DB500080B500AFFAF71AFA4FF46D43CEF2000326
:10DB60004FF46D42CEF20002D2F8882042F47002E7
:10DB7000C3F88820FAF74AF900F002F880BD00BF28
:10DB800080B592B000AF4FF46053C4F202034FF47B
:10DB90006052C4F20202126C42F080521A644FF4D6
:10DBA000E043C4F200034FF4E042C4F20002126802
:10DBB00042F440421A604FF001037B604FF00103D2
:10DBC000BB604FF00203FB614FF480033B624FF0F8
:10DBD00018037B624FF4A873BB624FF00203FB6231
:10DBE0004FF007033B6307F104031846F3F762FEA7
:10DBF0004FF00F037B634FF00203BB634FF0000352
:10DC0000FB634FF4A0533B644FF480537B6407F1F4
:10DC1000340318464FF00501F4F704FA07F14807FA
:10DC2000BD4680BD80B483B000AF03463960FB7150
:10DC300097F90730002B10DA4FF46D43CEF2000352
:10DC4000FA7902F00F02A2F104013A68D2B24FEA67
:10DC50000212D2B25B181A760DE04FF46143CEF295
:10DC6000000397F907103A68D2B24FEA0212D2B213
:10DC70005B1883F8002307F10C07BD4680BC704792
:10DC800080B582B000AF78607B6803F1FF326FF03F
:10DC90007F439A4202D94FF001031DE04EF2100378
:10DCA000CEF200037A6802F1FF325A604FF0FF3083
:10DCB0004FF00F01FFF7B6FF4EF21003CEF2000354
:10DCC0004FF000029A604EF21003CEF200034FF0C4
:10DCD00007021A604FF00003184607F10807BD4617
:10DCE00080BD00BF80B500AF40F20C03C2F200035C
:10DCF0001A6844F6D353C1F26203A3FB02134FEA3E
:10DD000093131846FFF7BCFF80BD00BF80B400AF7F
:10DD100044F6BC43C2F200031B68002B0BD044F650
:10DD2000BC43C2F200031B6803F1FF3244F6BC435C
:10DD3000C2F200031A60BD4680BC704780B586B051
:10DD400000AF4FF46053C4F202034FF46052C4F2C8
:10DD50000202126B42F001021A634FF480737B607F
:10DD60004FF00103BB604FF002033B614FF0010332
:10DD7000FB6007F104034FF00000C4F202001946F3
:10DD8000F4F7D2FC4FF00000C4F202004FF48071AF
:10DD90004FF00002F5F7A2F807F11807BD4680BD65
:10DDA00080B582B000AF0346FB804AF60003C0F6A0
:10DDB00001031A684AF60003C0F601039B88104667
:10DDC00019464FF00002F5F789F84AF67003C0F6DD
:10DDD00001031A684AF67003C0F601039B881046D7
:10DDE00019464FF00002F5F779F84AF61003C0F62D
:10DDF00001031A684AF61003C0F601039B88104617
:10DE000019464FF00002F5F769F844F6C043C2F234
:10DE10000003FA881A8040F6D860C2F2000044F687
:10DE2000C041C2F200014FF001024FF00103F3F7CD
:10DE3000D1FA4AF61003C0F601031A684AF6100335
:10DE4000C0F601039B88104619464FF00102F5F712
:10DE500045F807F10807BD4680BD00BF80B582B018
:10DE600000AF0346FB804AF60003C0F601031A68C0
:10DE70004AF60003C0F601039B88104619464FF08E
:10DE80000102F5F72BF84AF67003C0F601031A6891
:10DE90004AF67003C0F601039B88104619464FF0FE
:10DEA0000002F5F71BF84AF61003C0F601031A68E2
:10DEB0004AF61003C0F601039B88104619464FF03E
:10DEC0000002F5F70BF844F6C043C2F20003FA88EB
:10DED0001A8040F6D860C2F2000044F6C041C2F297
:10DEE00000014FF001024FF00103F3F773FA4AF615
:10DEF0001003C0F601031A684AF61003C0F60103C6
:10DF00009B88104619464FF00102F4F7E7FF07F12E
:10DF10000807BD4680BD00BF80B500AF4AF60803C4
:10DF2000C0F601031A684AF60803C0F601039B888D
:10DF3000104619464FF00102F4F7D0FF4FF00500EC
:10DF4000FEF734F94AF60803C0F601031A684AF6E8
:10DF50000803C0F601039B88104619464FF00002E3
:10DF6000F4F7BCFF4FF01400FEF720F94AF608035F
:10DF7000C0F601031A684AF60803C0F601039B883D
:10DF8000104619464FF00102F4F7A8FF4FF0960033
:10DF9000FEF70CF94AF61003C0F601031A684AF6B8
:10DFA0001003C0F601039B88104619464FF000028B
:10DFB000F4F794FF4FF0EF00FFF7F2FE4FF003008D
:10DFC000FFF74CFF4FF08000FFF748FF4FF00200D3
:10DFD000FFF744FF4FF0CF00FFF7E2FE4FF00000E5
:10DFE000FFF73CFF4FF0C100FFF738FF4FF0300064
:10DFF000FFF734FF4FF0ED00FFF7D2FE4FF0640063
:10E00000FFF72CFF4FF00300FFF728FF4FF012003F
:10E01000FFF724FF4FF08100FFF720FF4FF0E800EB
:10E02000FFF7BEFE4FF08500FFF718FF4FF000002E
:10E03000FFF714FF4FF07800FFF710FF4FF0CB0011
:10E04000FFF7AEFE4FF03900FFF708FF4FF02C004E
:10E05000FFF704FF4FF00000FFF700FF4FF0340020
:10E06000FFF7FCFE4FF00200FFF7F8FE4FF0F7005D
:10E07000FFF796FE4FF02000FFF7F0FE4FF0EA00AA
:10E08000FFF78EFE4FF00000FFF7E8FE4FF00000B4
:10E09000FFF7E4FE4FF0C000FFF782FE4FF02300D1
:10E0A000FFF7DCFE4FF0C100FFF77AFE4FF01000E3
:10E0B000FFF7D4FE4FF0C500FFF772FE4FF03E00B1
:10E0C000FFF7CCFE4FF02800FFF7C8FE4FF0C70067
:10E0D000FFF766FE4FF08600FFF7C0FE4FF03600F8
:10E0E000FFF75EFE4FF04800FFF7B8FE4FF03A0032
:10E0F000FFF756FE4FF05500FFF7B0FE4FF0B100AE
:10E10000FFF74EFE4FF00000FFF7A8FE4FF018009B
:10E11000FFF7A4FE4FF0B600FFF742FE4FF00800F5
:10E12000FFF79CFE4FF08200FFF798FE4FF02700AC
:10E13000FFF794FE4FF0F200FFF732FE4FF00000C1
:10E14000FFF78CFE4FF02600FFF72AFE4FF001008C
:10E15000FFF784FE4FF0E000FFF722FE4FF00F00C4
:10E16000FFF77CFE4FF03100FFF778FE4FF02B00F9
:10E17000FFF774FE4FF00C00FFF770FE4FF00E003B
:10E18000FFF76CFE4FF00800FFF768FE4FF04E00FF
:10E19000FFF764FE4FF0F100FFF760FE4FF037002D
:10E1A000FFF75CFE4FF00700FFF758FE4FF010003E
:10E1B000FFF754FE4FF00300FFF750FE4FF00E0044
:10E1C000FFF74CFE4FF00900FFF748FE4FF000004C
:10E1D000FFF744FE4FF0E100FFF7E2FD4FF00000D3
:10E1E000FFF73CFE4FF00E00FFF738FE4FF0140033
:10E1F000FFF734FE4FF00300FFF730FE4FF0110041
:10E20000FFF72CFE4FF00700FFF728FE4FF031001C
:10E21000FFF724FE4FF0C100FFF720FE4FF048004B
:10E22000FFF71CFE4FF00800FFF718FE4FF00F003D
:10E23000FFF714FE4FF00C00FFF710FE4FF0310017
:10E24000FFF70CFE4FF03600FFF708FE4FF00F000F
:10E25000FFF704FE4FF01100FFF7A2FD4FF078002A
:10E26000FDF7A4FF4FF02900FFF79AFD80BD00BF26
:10E2700080B582B000AFF880B9807A803B804FF0E3
:10E280002A00FFF78DFDFB884FEA13239BB2184647
:10E29000FFF7E4FDFB88DBB29BB21846FFF7DEFD1B
:10E2A0007B884FEA13239BB21846FFF7D7FD7B8884
:10E2B000DBB29BB21846FFF7D1FD4FF02B00FFF702
:10E2C0006FFDBB884FEA13239BB21846FFF7C6FDCC
:10E2D000BB881846FFF7C2FD3B884FEA13239BB269
:10E2E0001846FFF7BBFD3B881846FFF7B7FD4FF018
:10E2F0002C00FFF755FD07F10807BD4680BD00BFA4
:10E3000090B597B014AF0346FB804AF60003C0F601
:10E3100001031A684AF60003C0F601039B88104601
:10E3200019464FF00102F4F7D9FD4AF61003C0F682
:10E3300001031A684AF61003C0F601039B881046D1
:10E3400019464FF00002F4F7C9FD44F6C043C2F28B
:10E350000003FA881A8040F6D864C2F2000444F63A
:10E36000C443C2F20003119344F6C043C2F2000357
:10E3700012934FF001031393694604F110024FF01A
:10E380004403084611461A4604F054F994E80F0075
:10E39000F9F7A4FF4AF61003C0F601031A684AF61B
:10E3A0001003C0F601039B88104619464FF0010286
:10E3B000F4F794FD07F10C07BD4690BD90B597B0FA
:10E3C00014AF13460246FA800A46BA807B80B7F93A
:10E3D0000630002B79DB40F63273C2F200031B8853
:10E3E000B7F906201BB29A426FDAB7F90430002B56
:10E3F0006BDB40F63873C2F200031B88B7F90420C8
:10E400001BB29A4261DAF888B988FB8803F10103EC
:10E410009AB2BB8803F101039BB2FFF729FF4AF6CA
:10E420000003C0F601031A684AF60003C0F60103B0
:10E430009B88104619464FF00102F4F74FFD4AF64B
:10E440001003C0F601031A684AF61003C0F6010370
:10E450009B88104619464FF00002F4F73FFD44F642
:10E46000C043C2F200037A881A8040F6D864C2F230
:10E47000000444F6C443C2F20003119344F6C043BF
:10E48000C2F2000312934FF001031393694604F1A3
:10E4900010024FF04403084611461A4604F0CAF829
:10E4A00094E80F00F9F71AFF4AF61003C0F60103CB
:10E4B0001A684AF61003C0F601039B8810461946F5
:10E4C0004FF00102F4F70AFD00E000BF07F10C076E
:10E4D000BD4690BD90B597B014AFF880B9807A80F2
:10E4E0003B8040F63273C2F200031B88B7F9062066
:10E4F0001BB29A4280F2948040F63873C2F2000355
:10E500001B88B7F904201BB29A4280F28980B7F9C0
:10E510000420B7F90230D31803F1FF3240F6387304
:10E52000C2F200031B881BB29A4209DB40F6387323
:10E53000C2F200031B889AB2BB88D31A9BB27B80BD
:10E54000F888B988FA88BC887B88E3189BB203F105
:10E55000FF339BB2FFF78CFE4AF60003C0F60103BF
:10E560001A684AF60003C0F601039B881046194654
:10E570004FF00102F4F7B2FC4AF61003C0F60103B3
:10E580001A684AF61003C0F601039B881046194624
:10E590004FF00002F4F7A2FC24E044F6C043C2F2BC
:10E5A00000033A881A8040F6D864C2F2000444F6A8
:10E5B000C443C2F20003119344F6C043C2F2000305
:10E5C00012934FF001031393694604F110024FF0C8
:10E5D0004403084611461A4604F02CF894E80F004C
:10E5E000F9F77CFEB7F90230002B0CBF00230123A2
:10E5F000DBB27A8802F1FF327A80002BCDD14AF665
:10E600001003C0F601031A684AF61003C0F60103AE
:10E610009B88104619464FF00102F4F75FFC00E0BA
:10E6200000BF07F10C07BD4690BD00BF90B597B085
:10E6300014AFF880B9807A803B8040F63273C2F222
:10E6400000031B88B7F906201BB29A4280F294801F
:10E6500040F63873C2F200031B88B7F904201BB2DE
:10E660009A4280F28980B7F90620B7F90230D318B0
:10E6700003F1FF3240F63273C2F200031B881BB273
:10E680009A4209DB40F63273C2F200031B889AB249
:10E69000FB88D31A9BB27B80F888B988FA887B887C
:10E6A000D3189BB203F1FF339AB2BB88FFF7E0FDAA
:10E6B0004AF60003C0F601031A684AF60003C0F6E2
:10E6C00001039B88104619464FF00102F4F706FC3F
:10E6D0004AF61003C0F601031A684AF61003C0F6A2
:10E6E00001039B88104619464FF00002F4F7F6FB31
:10E6F00024E044F6C043C2F200033A881A8040F690
:10E70000D864C2F2000444F6C443C2F20003119379
:10E7100044F6C043C2F2000312934FF00103139377
:10E72000694604F110024FF04403084611461A46A8
:10E7300003F080FF94E80F00F9F7D0FDB7F902303D
:10E74000002B0CBF00230123DBB27A8802F1FF32D9
:10E750007A80002BCDD14AF61003C0F601031A6867
:10E760004AF61003C0F601039B88104619464FF085
:10E770000102F4F7B3FB00E000BF07F10C07BD4650
:10E7800090BD00BF90B597B014AFF880B9807A8083
:10E790003B8040F63273C2F200031B88B7F90620B3
:10E7A0001BB29A4280F2BB8040F63873C2F200037B
:10E7B0001B88B7F904201BB29A4280F2B080B7F9E7
:10E7C0000620B7F90230D31803F1FF3240F6327356
:10E7D000C2F200031B881BB29A4209DB40F6327377
:10E7E000C2F200031B889AB2FB88D31A9BB27B80CB
:10E7F000B7F90420B7F90030D31803F1FF3240F61F
:10E800003873C2F200031B881BB29A4209DB40F640
:10E810003873C2F200031B889AB2BB88D31A9BB22A
:10E820003B80F888B988FA887B88D3189BB203F1BB
:10E83000FF339AB2BC883B88E3189BB203F1FF33E5
:10E840009BB2FFF715FD4AF60003C0F601031A68F4
:10E850004AF60003C0F601039B88104619464FF0A4
:10E860000102F4F73BFB4AF61003C0F601031A68F5
:10E870004AF61003C0F601039B88104619464FF074
:10E880000002F4F72BFB3B88BB8033E07B88FB80E6
:10E8900028E044F6C043C2F200033A8B1A8040F6E7
:10E8A000D864C2F2000444F6C443C2F200031193D8
:10E8B00044F6C043C2F2000312934FF001031393D6
:10E8C000694604F110024FF04403084611461A4607
:10E8D00003F0B0FE94E80F00F9F700FDFB8803F1A8
:10E8E000FF33FB80B7F90630002BD2DCBB8803F185
:10E8F000FF33BB80B7F90430002BC7DC4AF61003A6
:10E90000C0F601031A684AF61003C0F601039B889B
:10E91000104619464FF00102F4F7E0FA00E000BF9C
:10E9200007F10C07BD4690BD80B582B000AF03462D
:10E93000FB804FF03700FFF733FAFB884FEA1323D1
:10E940009BB21846FFF78AFAFB88DBB29BB21846E7
:10E95000FFF784FA07F10807BD4680BD80B582B095
:10E9600000AF13460246FA800A46BA807B80FA88D6
:10E97000BB88D2187B88D318B3F5A07F2BD14FF07A
:10E980003300FFF70DFAFB884FEA13239BB21846BA
:10E99000FFF764FAFB88DBB29BB21846FFF75EFA1A
:10E9A000BB884FEA13239BB21846FFF757FABB8880
:10E9B000DBB29BB21846FFF751FA7B884FEA13236C
:10E9C0009BB21846FFF74AFA7B88DBB29BB2184627
:10E9D000FFF744FA00E000BF07F10807BD4680BD1D
:10E9E00080B584B000AF0346FB714FF03600FFF7EF
:10E9F000D7F9FB7903F00303FB60FB68032B57D8BF
:10EA000001A252F823F000BF19EA00083FEA00080B
:10EA100065EA00088BEA00084FF04800FFF71EFA8D
:10EA200040F63273C2F200034FF0F0021A8040F653
:10EA30003873C2F200034FF4A0721A8038E04FF02E
:10EA40002800FFF70BFA40F63273C2F200034FF4CE
:10EA5000A0721A8040F63873C2F200034FF0F00241
:10EA60001A8025E04FF08800FFF7F8F940F632737E
:10EA7000C2F200034FF0F0021A8040F63873C2F27F
:10EA800000034FF4A0721A8012E04FF0E800FFF785
:10EA9000E5F940F63273C2F200034FF4A0721A8017
:10EAA00040F63873C2F200034FF0F0021A8000BF44
:10EAB00007F11007BD4680BD80B584B000AFF88077
:10EAC000B9807A803B80FB88FB810CE0B7F90E00AF
:10EAD000B7F90410B7F900203B8BFFF7FBFCFB896B
:10EAE00003F10103FB81B7F90E20B7F90610B7F95E
:10EAF0000230CB189A42E9DB07F11007BD4680BD12
:10EB000080B584B002AF0346FB8040F63273C2F298
:10EB100000031A8840F63873C2F200031B8812B251
:10EB20001BB2F98800914FF000004FF00001FFF791
:10EB300029FE07F10807BD4680BD00BF80B58CB037
:10EB400000AFF880B9807A803B80B7F90420B7F92C
:10EB500000309A420BDDBB887B843B88BB807B8C7A
:10EB60003B80FB883B847B88FB803B8C7B80B7F9B8
:10EB70000020B7F93C309A420BDDBB8FFB833B880A
:10EB8000BB87FB8B3B803B8FBB837B883B87BB8BEF
:10EB90007B80B7F90420B7F900309A420BDDBB88BF
:10EBA0007B833B88BB807B8B3B80FB883B837B8864
:10EBB000FB803B8B7B80B7F90420B7F93C309A424D
:10EBC00037D1FB88BB85BB8DFB85B7F90220B7F930
:10EBD0002E309A4202DA7B88FB8507E0B7F90220E3
:10EBE000B7F92C309A4201DD7B88BB85B7F9382014
:10EBF000B7F92E309A4202DA3B8FFB8507E0B7F96E
:10EC00003820B7F92C309A4201DD3B8FBB85BA8D95
:10EC1000FB8DD31A9BB203F101039BB29BB2B7F9F0
:10EC20002E00B7F904101AB2B7F84030FFF7FEFC17
:10EC3000D9E07A88FB88D31A9BB2FB823A88BB88DA
:10EC4000D31A9BB2BB823A8FFB88D31A9BB27B82CA
:10EC5000BA8FBB88D31A9BB23B823A8F7B88D31A78
:10EC60009BB2FB81BA8F3B88D31A9BB2BB814FF01A
:10EC70000003FB844FF00003BB84B7F90020B7F911
:10EC80003C309A4202D13B883B8504E03B8803F14B
:10EC9000FF339BB23B85BB887B8540E0B7F92620DC
:10ECA000B7F9143092FBF3F39AB2FB88D3189BB2F6
:10ECB000FB85B7F92420B7F9103092FBF3F39AB231
:10ECC000FB88D3189BB2BB85FA8CFB8AD3189BB206
:10ECD000FB84BA8C7B8AD3189BB2BB84B7F92E20F5
:10ECE000B7F92C309A4205DDFB8D7B81BB8DFB850E
:10ECF0007B89BB85BA8DFB8DD31A9BB203F10103CF
:10ED00009BB29BB2B7F92E00B7F92A101AB2B7F826
:10ED10004030FFF78BFC7B8D03F101037B85B7F956
:10ED20002A20B7F928309A42B8DDB7F92A20B7F976
:10ED30000030D31A9BB2FA8902FB03F39BB2FB8427
:10ED4000B7F92A20B7F90430D31A9BB27A8A02FBAA
:10ED500003F39BB2BB8440E0B7F92620B7F90C302F
:10ED600092FBF3F39AB27B88D3189BB2FB85B7F979
:10ED70002420B7F9103092FBF3F39AB2FB88D31832
:10ED80009BB2BB85FA8CFB89D3189BB2FB84BA8CEF
:10ED90007B8AD3189BB2BB84B7F92E20B7F92C30ED
:10EDA0009A4205DDFB8D3B81BB8DFB853B89BB8595
:10EDB000BA8DFB8DD31A9BB203F101039BB29BB2B8
:10EDC000B7F92E00B7F92A101AB2B7F84030FFF79A
:10EDD0002DFC7B8D03F101037B85B7F92A20B7F960
:10EDE0003C309A42B8DD07F13007BD4680BD00BF18
:10EDF00090B589B000AFBA600246FA810A46BA817E
:10EE0000FB80F889B989FA89FB88D3189BB203F192
:10EE1000FF339AB2BC893B8EE3189BB203F1FF33F8
:10EE20009BB2FFF725FA4AF60003C0F601031A6801
:10EE30004AF60003C0F601039B88104619464FF0BE
:10EE40000102F4F74BF84AF61003C0F601031A6802
:10EE50004AF61003C0F601039B88104619464FF08E
:10EE60000002F4F73BF84FF00003FB832CE0B7F906
:10EE70001E304FEA4303BA68D3181A88BB8E13407A
:10EE80009BB24FEA13239BB2DBB23B75B7F91E303E
:10EE90004FEA4303BA68D3181B88DAB2BB8EDBB2E1
:10EEA0001340DBB27B7507F1140340F6D860C2F261
:10EEB000000019464FF002024FF00103F2F78AFA00
:10EEC000FB8B03F10103FB83B7F91E20B7F9063072
:10EED000B7F9301001FB03F39A42C8DB4AF610037E
:10EEE000C0F601031A684AF61003C0F601039B88B6
:10EEF000104619464FF00102F3F7F0FF07F124071F
:10EF0000BD4690BDB0B584B002AF0346FB71FB793E
:10EF10000A2B1DD140F63773C2F200031B784FEA6B
:10EF2000C3039AB240F6B453C2F200031B889BB2EB
:10EF3000D3189BB29AB240F6B453C2F200031A80BF
:10EF400040F63473C2F200034FF000021A807FE0F3
:10EF5000FB790D2B7CD040F63473C2F20003198884
:10EF600040F6B453C2F200031A8840F6CE73C2F2E0
:10EF700000031C8840F6CC73C2F200031D8840F6E3
:10EF80003773C2F20003187809B212B2FB79009508
:10EF90000190084611461A46234600F05DF840F6F7
:10EFA0003773C2F200031B781A464FEA4202D318A5
:10EFB0004FEA43039AB240F63473C2F200031B884F
:10EFC0009BB2D3189BB29AB240F63473C2F20003DC
:10EFD0001A8040F63673C2F200031B78002B37D03C
:10EFE00040F63473C2F200031B8819B240F6327344
:10EFF000C2F200031B8818B240F63773C2F2000356
:10F000001B781A4613464FEA82029B1A4FEA4303C3
:10F01000C31899421CDD40F63773C2F200031B7817
:10F020004FEAC3039AB240F6B453C2F200031B88FE
:10F030009BB2D3189BB29AB240F6B453C2F200030B
:10F040001A8040F63473C2F200034FF000021A80B7
:10F0500007F10807BD46B0BD90B587B002AFF88094
:10F06000B980FA703B804FF00003FB73BDE097F965
:10F070000F30052B03D14FF00003BB730FE0FA787C
:10F0800013464FEA83039B181A4697F90F30D2189C
:10F090004AF6B813C0F60103D3181B78BB734FF0C0
:10F0A00000037B7398E0BB7B03F00103DBB2002B12
:10F0B00043D097F82430012B16D197F90F309AB22C
:10F0C000FB88D3189BB29AB297F90D3099B2BB88DE
:10F0D000CB189BB29BB211B21AB23B8808461146BC
:10F0E0001A46FFF76BF96FE097F90F309BB297F86C
:10F0F000242092B202FB03F39AB2FB88D3189BB28E
:10F1000098B297F90D309BB297F8242092B202FB87
:10F1100003F39AB2BB88D3189BB299B297F8243004
:10F120009AB297F824309BB200B209B212B21BB265
:10F130003C880094FFF7C0FC46E03A8C3B889A423A
:10F1400042D097F82430012B16D197F90F309AB29C
:10F15000FB88D3189BB29AB297F90D3099B2BB884D
:10F16000CB189BB29BB211B21AB23B8C0846114627
:10F170001A46FFF723F927E097F90F309BB297F86B
:10F18000242092B202FB03F39AB2FB88D3189BB2FD
:10F1900098B297F90D309BB297F8242092B202FBF7
:10F1A00003F39AB2BB88D3189BB299B297F8243074
:10F1B0009AB297F824309BB200B209B212B21BB2D5
:10F1C0003C8C0094FFF778FCBB7B4FEA5303BB7386
:10F1D0007B7B03F101037B7397F90D30072B7FF7DE
:10F1E00062AFFB7B03F10103FB7397F90F30052B33
:10F1F0007FF73DAF07F11407BD4690BD80B483B0E3
:10F2000000AF02460B46FA80BB8040F63473C2F270
:10F210000003FA881A8040F6B453C2F20003BA8899
:10F220001A8007F10C07BD4680BC704780B483B0DC
:10F2300000AF0346FB71FB79002B01D0FA7901E0A6
:10F240004FF0010240F63773C2F200031A7007F163
:10F250000C07BD4680BC704780B483B000AF024647
:10F260000B46FA80BB8040F6CE73C2F20003FA88E8
:10F270001A8040F6CC73C2F20003BA881A8007F1F4
:10F280000C07BD4680BC704780B483B000AF034616
:10F29000FB7140F63673C2F20003FA791A7007F177
:10F2A0000C07BD4680BC704780B485B000AF786065
:10F2B00079807A703B704FF00003FB737B687A882B
:10F2C0001A807A684BF2B463C0F6010353607B681E
:10F2D0007A789A707B683A78DA707B681B88B3F525
:10F2E000807F2ED0B3F5807F04DC102B47D0402BDD
:10F2F00036D053E0B3F5806F14D0B3F5805F4DD1B5
:10F300007B684FF001029A817B684FF00102DA813D
:10F310007A684AF6B463C0F6010393607B68294AB1
:10F320001A613FE07B684FF004029A817B684FF0DE
:10F330000402DA817B681F4A9A607B68224A1A615C
:10F3400030E07B684FF010029A817B684FF010022A
:10F35000DA817B68184A9A607B681C4A1A6121E04E
:10F360007B684FF040029A817B684FF04002DA815F
:10F370007B68124A9A607B68154A1A6112E07B68C2
:10F380004FF480729A817B684FF48072DA817B68D7
:10F390000B4A9A607B680F4A1A6103E04FF0FF0343
:10F3A000FB7300BFFB7B5BB2184607F11407BD4639
:10F3B00080BC7047BAAE0108D2AE010832AF010876
:10F3C000B2B00108000080390000803A0000803BA4
:10F3D0000000803C0000803D80B4C1B000AFF86008
:10F3E0007A600A467A813B817B89C7F8F430D7F886
:10F3F000F430C7F8E430D7F8F4304FEA9303C7F895
:10F40000F4304FF00003C7F8F8304FF00003C7F8AE
:10F41000FC30D7F8F430C7F8F030D7F8F820D7F838
:10F42000F430D318C7F8E030D7F8E020D7F8F4303C
:10F43000D318C7F8DC30D7F8DC20D7F8F430D3186D
:10F44000C7F8D830D7F8F8304FEAC303FA68D318B2
:10F450001B68C7F8D430D7F8F8304FEAC30303F17C
:10F460000403FA68D3181B68C7F8D030D7F8E03027
:10F470004FEAC303FA68D3181B68C7F8CC30D7F833
:10F48000E0304FEAC30303F10403FA68D3181B68A2
:10F49000C7F8C830D7F8DC304FEAC303FA68D3188E
:10F4A0001B68C7F8C430D7F8DC304FEAC30303F158
:10F4B0000403FA68D3181B68C7F8C030D7F8D830EF
:10F4C0004FEAC303FA68D3181B68C7F8BC30D7F8F3
:10F4D000D8304FEAC30303F10403FA68D3181B685A
:10F4E000C7F8B83097ED357AD7ED317A77EE277ACD
:10F4F000C7ED2D7A97ED337AD7ED2F7A77EE277A0D
:10F50000C7ED2C7A97ED347AD7ED307A77EE277AFB
:10F51000C7ED2B7A97ED327AD7ED2E7A77EE277AF0
:10F52000C7ED2A7AD7F8FC20D7F8FC30D318C7F8F3
:10F53000A430D7F8A4304FEAC3037A68D3181B6805
:10F54000C7F8A030D7F8A4304FEAC30303F104038F
:10F550007A68D3181B68C7F89C3097ED357AD7EDD9
:10F56000317A77EE677AC7ED267A97ED337AD7ED61
:10F570002F7A77EE677AC7ED257A97ED347AD7ED53
:10F58000307A77EE677AC7ED247A97ED327AD7ED45
:10F590002E7A77EE677AC7ED237AD7F8F8304FEAFC
:10F5A000C303FA68D31897ED2D7AD7ED2C7A77EE4E
:10F5B000277AC3ED007AD7F8F8304FEAC30303F196
:10F5C0000403FA68D31897ED2B7AD7ED2A7A77EEF1
:10F5D000277AC3ED007A97ED267AD7ED237A77EE76
:10F5E000277AC7ED227A97ED247AD7ED257A77EE40
:10F5F000677AC7ED217A97ED2D7AD7ED2C7A77EEE1
:10F60000677AC7ED207A97ED2B7AD7ED2A7A77EED5
:10F61000677AC7ED1F7A97ED267AD7ED237A77EED2
:10F62000677AC7ED1E7A97ED257AD7ED247A77EEC3
:10F63000277AC7ED1D7AD7F8FC304FEAC3037A6802
:10F64000D3181B683B67D7F8FC304FEAC30303F1BC
:10F6500004037A68D3181B68FB66D7F8A420D7F890
:10F66000FC30D318BB66BB6E4FEAC3037A68D3186D
:10F670001B687B66BB6E4FEAC30303F104037A6821
:10F68000D3181B683B6697ED227AD7ED1C7A67EE9C
:10F69000277AC7ED177A97ED217AD7ED1C7A67EEB6
:10F6A000277AC7ED167A97ED207AD7ED287A67EE9C
:10F6B000277AC7ED157A97ED1F7AD7ED287A67EE8E
:10F6C000277AC7ED147A97ED1E7AD7ED197A67EE8F
:10F6D000277AC7ED137A97ED1D7AD7ED197A67EE81
:10F6E000277AC7ED127A97ED217AD7ED1B7A67EE6C
:10F6F000277AC7ED117A97ED227AD7ED1B7A67EE5C
:10F70000277AC7ED107A97ED1F7AD7ED277A67EE43
:10F71000277AC7ED0F7A97ED207AD7ED277A67EE33
:10F72000277AC7ED0E7A97ED1D7AD7ED187A67EE36
:10F73000277AC7ED0D7A97ED1E7AD7ED187A67EE26
:10F74000277AC7ED0C7A97ED177AD7ED117A77EE15
:10F75000277AC7ED177A97ED167AD7ED107A77EEFC
:10F76000677AC7ED167A97ED157AD7ED0F7A77EEAF
:10F77000277AC7ED157A97ED147AD7ED0E7A77EEE2
:10F78000677AC7ED147A97ED137AD7ED0D7A77EE95
:10F79000277AC7ED137A97ED127AD7ED0C7A77EEC8
:10F7A000677AC7ED127AD7F8E0304FEAC303FA68F8
:10F7B000D3187A6D1A60D7F8E0304FEAC30303F12B
:10F7C0000403FA68D3183A6D1A60D7F8DC304FEAB0
:10F7D000C303FA68D318FA6D1A60D7F8DC304FEA21
:10F7E000C30303F10403FA68D318BA6D1A60D7F89B
:10F7F000D8304FEAC303FA68D318FA6C1A60D7F806
:10F80000D8304FEAC30303F10403FA68D318BA6C83
:10F810001A603B89D7F8FC20D318C7F8FC30D7F81A
:10F82000F83003F10103C7F8F830D7F8F03003F1EE
:10F83000FF33C7F8F030D7F8F030002B7FF4EDAD90
:10F840003B894FEA83033B817B894FEA93039BB259
:10F85000C7F8EC303DE2D7F8F430C7F8E430D7F819
:10F86000F4304FEA9303C7F8F4304FF00003C7F8C1
:10F87000FC304FF00003C7F8F030D7F8FC20D7F881
:10F88000FC30D318C7F8A430D7F8A420D7F8FC3040
:10F89000D318BB66D7F8FC304FEAC3037A68D31895
:10F8A0001B683B67D7F8FC304FEAC30303F104033E
:10F8B0007A68D3181B68FB66D7F8A4304FEAC303F5
:10F8C0007A68D3181B68C7F8A030D7F8A4304FEA7D
:10F8D000C30303F104037A68D3181B68C7F89C308C
:10F8E000BB6E4FEAC3037A68D3181B687B66BB6E96
:10F8F0004FEAC30303F104037A68D3181B683B661D
:10F900003B89D7F8FC20D318C7F8FC30D7F8F03083
:10F91000C7F8F830D7F8F820D7F8F430D318C7F87C
:10F92000E030D7F8E020D7F8F430D318C7F8DC304F
:10F93000D7F8DC20D7F8F430D318C7F8D830D7F888
:10F94000F8304FEAC303FA68D3181B68C7F8D430FD
:10F95000D7F8F8304FEAC30303F10403FA68D31869
:10F960001B68C7F8D030D7F8E0304FEAC303FA6815
:10F97000D3181B68C7F8CC30D7F8E0304FEAC30380
:10F9800003F10403FA68D3181B68C7F8C830D7F826
:10F99000DC304FEAC303FA68D3181B68C7F8C430D9
:10F9A000D7F8DC304FEAC30303F10403FA68D31835
:10F9B0001B68C7F8C030D7F8D8304FEAC303FA68DD
:10F9C000D3181B68C7F8BC30D7F8D8304FEAC30348
:10F9D00003F10403FA68D3181B68C7F8B83097ED31
:10F9E000357AD7ED317A77EE677AC7ED267A97EDDB
:10F9F000337AD7ED2F7A77EE677AC7ED257A97EDD0
:10FA0000347AD7ED307A77EE677AC7ED247A97EDBE
:10FA1000327AD7ED2E7A77EE677AC7ED237A97EDB3
:10FA2000357AD7ED317A77EE277AC7ED2D7A97EDD3
:10FA3000337AD7ED2F7A77EE277AC7ED2C7A97EDC8
:10FA4000347AD7ED307A77EE277AC7ED2B7A97EDB7
:10FA5000327AD7ED2E7A77EE277AC7ED2A7A97EDAC
:10FA6000267AD7ED237A77EE277AC7ED227A97EDBB
:10FA7000247AD7ED257A77EE677AC7ED217A97ED6C
:10FA80002D7AD7ED2C7A77EE677AC7ED207A97ED4D
:10FA90002B7AD7ED2A7A77EE677AC7ED1F7A97ED42
:10FAA000267AD7ED237A77EE677AC7ED1E7A97ED3F
:10FAB000257AD7ED247A77EE277AC7ED1D7AD7F825
:10FAC000F8304FEAC303FA68D31897ED2D7AD7EDD3
:10FAD0002C7A77EE277AC3ED007AD7F8F8304FEA20
:10FAE000C30303F10403FA68D31897ED2B7AD7ED1B
:10FAF0002A7A77EE277AC3ED007A97ED227AD7ED4E
:10FB00001C7A67EE277AC7ED177A97ED217AD7ED41
:10FB10001C7A67EE277AC7ED167A97ED207AD7ED33
:10FB2000287A67EE277AC7ED157A97ED1F7AD7ED19
:10FB3000287A67EE277AC7ED147A97ED1E7AD7ED0B
:10FB4000197A67EE277AC7ED137A97ED1D7AD7ED0C
:10FB5000197A67EE277AC7ED127A97ED217AD7EDF9
:10FB60001B7A67EE277AC7ED117A97ED227AD7EDE7
:10FB70001B7A67EE277AC7ED107A97ED1F7AD7EDDB
:10FB8000277A67EE277AC7ED0F7A97ED207AD7EDBF
:10FB9000277A67EE277AC7ED0E7A97ED1D7AD7EDB3
:10FBA000187A67EE277AC7ED0D7A97ED1E7AD7EDB2
:10FBB000187A67EE277AC7ED0C7A97ED177AD7EDAA
:10FBC000117A77EE277AC7ED177A97ED167AD7ED87
:10FBD000107A77EE677AC7ED167A97ED157AD7ED3A
:10FBE0000F7A77EE277AC7ED157A97ED147AD7ED6D
:10FBF0000E7A77EE677AC7ED147A97ED137AD7ED20
:10FC00000D7A77EE277AC7ED137A97ED127AD7ED52
:10FC10000C7A77EE677AC7ED127AD7F8E0304FEAC0
:10FC2000C303FA68D3187A6D1A60D7F8E0304FEA48
:10FC3000C30303F10403FA68D3183A6D1A60D7F8C6
:10FC4000DC304FEAC303FA68D318FA6D1A60D7F8AC
:10FC5000DC304FEAC30303F10403FA68D318BA6D2A
:10FC60001A60D7F8D8304FEAC303FA68D318FA6C91
:10FC70001A60D7F8D8304FEAC30303F10403FA68D7
:10FC8000D318BA6C1A60D7F8F820D7F8E430D31834
:10FC9000C7F8F8307A89D7F8F8309A423FF63AAE8A
:10FCA000D7F8F03003F10103C7F8F030D7F8F4309B
:10FCB00003F1FF32D7F8F0309A42BFF4DEAD3B8952
:10FCC0004FEA83033B81D7F8EC304FEA9303C7F840
:10FCD000EC30D7F8EC30042B3FF6BDAD7B894FEA12
:10FCE00093039BB2C7F8F030FB68C7F8E830D7F849
:10FCF000E8301B68C7F8D430D7F8E8305B68C7F83D
:10FD0000D030D7F8E8309B68C7F8CC30D7F8E83067
:10FD1000DB68C7F8C830D7F8E8301B69C7F8C430CB
:10FD2000D7F8E8305B69C7F8C030D7F8E8309B698E
:10FD3000C7F8BC30D7F8E830DB69C7F8B83097EDC2
:10FD4000357AD7ED317A77EE277AC7ED2D7A97EDB0
:10FD5000357AD7ED317A77EE677AC7ED267A97ED67
:10FD6000347AD7ED307A77EE277AC7ED2B7A97ED94
:10FD7000347AD7ED307A77EE677AC7ED247A97ED4B
:10FD8000337AD7ED2F7A77EE277AC7ED2C7A97ED75
:10FD9000327AD7ED2E7A77EE277AC7ED2A7A97ED69
:10FDA000337AD7ED2F7A77EE677AC7ED257A97ED1C
:10FDB000327AD7ED2E7A77EE677AC7ED237A97ED10
:10FDC0002D7AD7ED2C7A77EE277AC7ED0B7A97ED5F
:10FDD0002B7AD7ED2A7A77EE277AC7ED0A7A97ED54
:10FDE0002D7AD7ED2C7A77EE677AC7ED097A97ED01
:10FDF0002B7AD7ED2A7A77EE677AC7ED087A97EDF6
:10FE0000267AD7ED237A77EE277AC7ED077A97ED32
:10FE1000247AD7ED257A77EE677AC7ED067A97EDE3
:10FE2000267AD7ED237A77EE677AC7ED057A97EDD4
:10FE3000257AD7ED247A77EE277AC7ED047AD7F8BA
:10FE4000E830FA6A1A60D7F8E83003F10403BA6AB6
:10FE50001A60D7F8E83003F108037A6A1A60D7F815
:10FE6000E83003F10C033A6A1A60D7F8E83003F17E
:10FE70001003FA691A60D7F8E83003F11403BA697D
:10FE80001A60D7F8E83003F118037A691A60D7F8D6
:10FE9000E83003F11C033A691A60D7F8E83003F13F
:10FEA0002003C7F8E830D7F8F03003F1FF33C7F884
:10FEB000F030D7F8F030002B7FF419AF07F58277D8
:10FEC000BD4680BC704700BF80B4C3B000AFF860CF
:10FED00007F1040002601A463B4683ED000A0B4618
:10FEE0007B8107F108031A807B89C7F8FC30D7F8BB
:10FEF000FC30C7F8EC30D7F8FC304FEA9303C7F872
:10FF0000FC304FF00003C7F800314FF00003C7F892
:10FF10000431D7F8FC30C7F8F830D7F80021D7F80B
:10FF2000FC30D318C7F8E830D7F8E820D7F8FC3011
:10FF3000D318C7F8E430D7F8E420D7F8FC30D3184A
:10FF4000C7F8E030D7F800314FEAC303FA68D31896
:10FF50001B68C7F8DC30D7F800314FEAC30303F160
:10FF60000403FA68D3181B68C7F8D830D7F8E43010
:10FF70004FEAC303FA68D3181B68C7F8D430D7F820
:10FF8000E4304FEAC30303F10403FA68D3181B6893
:10FF9000C7F8D030D7F8E8304FEAC303FA68D3186F
:10FFA0001B68C7F8CC30D7F8E8304FEAC30303F139
:10FFB0000403FA68D3181B68C7F8C830D7F8E030D4
:10FFC0004FEAC303FA68D3181B68C7F8C430D7F8E0
:10FFD000E0304FEAC30303F10403FA68D3181B6847
:10FFE000C7F8C03097ED377AD7ED357A77EE277AB4
:10FFF000C7ED2F7A97ED337AD7ED317A77EE277AFE
:020000040801F1
:10000000C7ED2E7A97ED367AD7ED347A77EE277AE8
:10001000C7ED2D7A97ED327AD7ED307A77EE277AE1
:10002000C7ED2C7AD7F80421D7F80431D318C7F8D4
:10003000AC30D7F8AC304FEAC30307F104021268C2
:10004000D3181B68C7F8A830D7F8AC304FEAC30301
:1000500003F1040307F104021268D3181B68C7F800
:10006000A43097ED377AD7ED357A77EE677AC7ED1A
:10007000287A97ED337AD7ED317A77EE677AC7ED44
:10008000277A97ED367AD7ED347A77EE677AC7ED2F
:10009000267A97ED327AD7ED307A77EE677AC7ED28
:1000A000257AD7F800314FEAC303FA68D31897EDE1
:1000B0002F7AD7ED2E7A77EE277AC3ED007AD7F82C
:1000C00000314FEAC30303F10403FA68D31897ED34
:1000D0002D7AD7ED2C7A77EE277AC3ED007A97ED5B
:1000E000287AD7ED257A77EE677AC7ED247A97EDEF
:1000F000267AD7ED277A77EE277AC7ED237A97ED20
:100100002F7AD7ED2E7A77EE677AC7ED227A97EDC0
:100110002D7AD7ED2C7A77EE677AC7ED217A97EDB5
:10012000287AD7ED257A77EE277AC7ED207A97EDF2
:10013000267AD7ED277A77EE677AC7ED1F7AD7F858
:1001400004314FEAC30307F104021268D3181B6895
:10015000BB67D7F804314FEAC30303F1040307F187
:1001600004021268D3181B687B67D7F8AC20D7F855
:100170000431D3183B673B6F4FEAC30307F1040216
:100180001268D3181B68FB663B6F4FEAC30303F189
:10019000040307F104021268D3181B68BB6697EDCD
:1001A000247AD7ED1E7A67EE277AC7ED197A97ED94
:1001B000237AD7ED1E7A67EE277AC7ED187A97ED86
:1001C000227AD7ED2A7A67EE277AC7ED177A97ED6C
:1001D000217AD7ED2A7A67EE277AC7ED167A97ED5E
:1001E000207AD7ED1B7A67EE277AC7ED157A97ED5F
:1001F0001F7AD7ED1B7A67EE277AC7ED147A97ED51
:10020000237AD7ED1D7A67EE277AC7ED137A97ED3B
:10021000247AD7ED1D7A67EE277AC7ED127A97ED2B
:10022000217AD7ED297A67EE277AC7ED117A97ED13
:10023000227AD7ED297A67EE277AC7ED107A97ED03
:100240001F7AD7ED1A7A67EE277AC7ED0F7A97ED06
:10025000207AD7ED1A7A67EE277AC7ED0E7A97EDF6
:10026000197AD7ED137A77EE677AC7ED197A97ED99
:10027000187AD7ED127A77EE277AC7ED187A97EDCC
:10028000177AD7ED117A77EE677AC7ED177A97ED7F
:10029000167AD7ED107A77EE277AC7ED167A97EDB2
:1002A000157AD7ED0F7A77EE677AC7ED157A97ED65
:1002B000147AD7ED0E7A77EE277AC7ED147AD7F84D
:1002C000E8304FEAC303FA68D318FA6D1A60D7F81A
:1002D000E8304FEAC30303F10403FA68D318BA6D98
:1002E0001A60D7F8E4304FEAC303FA68D3187A6E7D
:1002F0001A60D7F8E4304FEAC30303F10403FA6845
:10030000D3183A6E1A60D7F8E0304FEAC303FA68A0
:10031000D3187A6D1A60D7F8E0304FEAC30303F1BF
:100320000403FA68D3183A6D1A6007F108031B88B2
:10033000D7F80421D318C7F80431D7F8003103F1F6
:100340000103C7F80031D7F8F83003F1FF33C7F8DD
:10035000F830D7F8F830002B7FF4DFAD07F1080351
:1003600007F1080212884FEA82021A807B894FEA5D
:1003700093039BB2C7F8F4304FE2D7F8FC30C7F8CC
:10038000EC30D7F8FC304FEA9303C7F8FC304FF05D
:100390000003C7F804314FF00003C7F8F830D7F86E
:1003A0000421D7F80431D318C7F8AC30D7F8AC2003
:1003B000D7F80431D3183B67D7F804314FEAC303A9
:1003C00007F104021268D3181B68BB67D7F8043121
:1003D0004FEAC30303F1040307F104021268D318C0
:1003E0001B687B67D7F8AC304FEAC30307F1040200
:1003F0001268D3181B68C7F8A830D7F8AC304FEA9A
:10040000C30303F1040307F104021268D3181B6845
:10041000C7F8A4303B6F4FEAC30307F10402126828
:10042000D3181B68FB663B6F4FEAC30303F1040359
:1004300007F104021268D3181B68BB6607F10803B2
:100440001B88D7F80421D318C7F80431D7F8F8303F
:10045000C7F80031D7F80021D7F8FC30D318C7F817
:10046000E830D7F8E820D7F8FC30D318C7F8E430E4
:10047000D7F8E420D7F8FC30D318C7F8E030D7F825
:1004800000314FEAC303FA68D3181B68C7F8DC30A1
:10049000D7F800314FEAC30303F10403FA68D31815
:1004A0001B68C7F8D830D7F8E8304FEAC303FA68BA
:1004B000D3181B68C7F8CC30D7F8E8304FEAC3032D
:1004C00003F10403FA68D3181B68C7F8C830D7F8DB
:1004D000E4304FEAC303FA68D3181B68C7F8D43076
:1004E000D7F8E4304FEAC30303F10403FA68D318E2
:1004F0001B68C7F8D030D7F8E0304FEAC303FA687A
:10050000D3181B68C7F8C430D7F8E0304FEAC303EC
:1005100003F10403FA68D3181B68C7F8C03097EDDD
:10052000377AD7ED357A77EE677AC7ED287A97ED87
:10053000337AD7ED317A77EE677AC7ED277A97ED80
:10054000367AD7ED347A77EE677AC7ED267A97ED6B
:10055000327AD7ED307A77EE677AC7ED257A97ED64
:10056000377AD7ED357A77EE277AC7ED2F7A97ED80
:10057000337AD7ED317A77EE277AC7ED2E7A97ED79
:10058000367AD7ED347A77EE277AC7ED2D7A97ED64
:10059000327AD7ED307A77EE277AC7ED2C7A97ED5D
:1005A000287AD7ED257A77EE677AC7ED247A97ED2A
:1005B000267AD7ED277A77EE277AC7ED237A97ED5B
:1005C0002F7AD7ED2E7A77EE677AC7ED227A97EDFC
:1005D0002D7AD7ED2C7A77EE677AC7ED217A97EDF1
:1005E000287AD7ED257A77EE277AC7ED207A97ED2E
:1005F000267AD7ED277A77EE677AC7ED1F7AD7F894
:1006000000314FEAC303FA68D31897ED2F7AD7ED7C
:100610002E7A77EE277AC3ED007AD7F800314FEAC9
:10062000C30303F10403FA68D31897ED2D7AD7EDCD
:100630002C7A77EE277AC3ED007A97ED247AD7EDFE
:100640001E7A67EE277AC7ED197A97ED237AD7EDF0
:100650001E7A67EE277AC7ED187A97ED227AD7EDE2
:100660002A7A67EE277AC7ED177A97ED217AD7EDC8
:100670002A7A67EE277AC7ED167A97ED207AD7EDBA
:100680001B7A67EE277AC7ED157A97ED1F7AD7EDBB
:100690001B7A67EE277AC7ED147A97ED237AD7EDA8
:1006A0001D7A67EE277AC7ED137A97ED247AD7ED96
:1006B0001D7A67EE277AC7ED127A97ED217AD7ED8A
:1006C000297A67EE277AC7ED117A97ED227AD7ED6E
:1006D000297A67EE277AC7ED107A97ED1F7AD7ED62
:1006E0001A7A67EE277AC7ED0F7A97ED207AD7ED61
:1006F0001A7A67EE277AC7ED0E7A97ED197AD7ED59
:10070000137A77EE677AC7ED197A97ED187AD7EDF5
:10071000127A77EE277AC7ED187A97ED177AD7ED28
:10072000117A77EE677AC7ED177A97ED167AD7EDDB
:10073000107A77EE277AC7ED167A97ED157AD7ED0E
:100740000F7A77EE677AC7ED157A97ED147AD7EDC1
:100750000E7A77EE277AC7ED147AD7F8E8304FEAA9
:10076000C303FA68D318FA6D1A60D7F8E8304FEA75
:10077000C30303F10403FA68D318BA6D1A60D7F8FB
:10078000E4304FEAC303FA68D3187A6E1A60D7F8D8
:10079000E4304FEAC30303F10403FA68D3183A6E56
:1007A0001A60D7F8E0304FEAC303FA68D3187A6DBD
:1007B0001A60D7F8E0304FEAC30303F10403FA6884
:1007C000D3183A6D1A60D7F80021D7F8EC30D31857
:1007D000C7F800317A89D7F800319A423FF63AAE2D
:1007E000D7F8F83003F10103C7F8F830D7F8FC3038
:1007F00003F1FF32D7F8F8309A42BFF4D0AD07F1D9
:10080000080307F1080212884FEA82021A80D7F81B
:10081000F4304FEA9303C7F8F430D7F8F430042BE0
:100820003FF6ABAD7B894FEA93039BB2C7F8F83034
:10083000FB68C7F8F030D7F8F0301B68C7F8DC3039
:10084000D7F8F0305B68C7F8D830D7F8F0309B683D
:10085000C7F8CC30D7F8F030DB68C7F8C830D7F825
:10086000F0301B69C7F8D430D7F8F0305B69C7F8AF
:10087000D030D7F8F0309B69C7F8C430D7F8F030E3
:10088000DB69C7F8C03097ED377AD7ED357A77EE68
:10089000277AC7ED2F7A97ED377AD7ED357A77EE4D
:1008A000677AC7ED287A97ED367AD7ED347A77EE06
:1008B000277AC7ED2D7A97ED367AD7ED347A77EE31
:1008C000677AC7ED267A97ED337AD7ED317A77EEEE
:1008D000277AC7ED2E7A97ED327AD7ED307A77EE18
:1008E000277AC7ED2C7A97ED337AD7ED317A77EE08
:1008F000677AC7ED277A97ED327AD7ED307A77EEBF
:10090000677AC7ED257A97ED2F7AD7ED2E7A77EEB5
:10091000277AC7ED0D7A97ED2D7AD7ED2C7A77EE01
:10092000277AC7ED0C7A97ED2F7AD7ED2E7A77EEEE
:10093000677AC7ED0B7A97ED2D7AD7ED2C7A77EEA3
:10094000677AC7ED0A7A97ED287AD7ED257A77EEA0
:10095000677AC7ED097A97ED267AD7ED277A77EE91
:10096000277AC7ED087A97ED287AD7ED257A77EEC2
:10097000277AC7ED077A97ED267AD7ED277A77EEB3
:10098000677AC7ED067A3B4697ED0D7AD3ED007A8C
:1009900067EE277AC7ED137A3B4697ED0C7AD3EDD5
:1009A000007A67EE277AC7ED127A3B4697ED0B7A0D
:1009B000D3ED007A67EE277AC7ED117A3B4697EDC3
:1009C0000A7AD3ED007A67EE277AC7ED107A3B46B4
:1009D00097ED097AD3ED007A67EE277AC7ED0F7AA3
:1009E0003B4697ED087AD3ED007A67EE277AC7ED9C
:1009F0000E7A3B4697ED077AD3ED007A67EE277AB9
:100A0000C7ED057A3B4697ED067AD3ED007A67EE9F
:100A1000277AC7ED047AD7F8F030FA6C1A60D7F865
:100A2000F03003F10403BA6C1A60D7F8F03003F128
:100A300008037A6C1A60D7F8F03003F10C033A6CB3
:100A40001A60D7F8F03003F11003FA6B1A60D7F888
:100A5000F03003F11403BA6B1A60D7F8F03003F1E9
:100A600018037A691A60D7F8F03003F11C033A6969
:100A70001A60D7F8F03003F12003C7F8F030D7F848
:100A8000F83003F1FF33C7F8F830D7F8F830002B0F
:100A90007FF4D1AE07F58677BD4680BC704700BFB6
:100AA00080B582B000AF786039607B689B78012B9D
:100AB0000ED17B6819887B685A687B689B89786847
:100AC000D0ED047A3868B0EE670AFFF7FDF908E068
:100AD0007B6819887B685A687B689B893868FEF751
:100AE0007BFC7B68DB78012B08D17B6819887B68ED
:100AF000DA897B689B68386800F004F807F108071A
:100B0000BD4680BD80B489B000AFF8607B600B4605
:100B10007B8113463B814FF00003BB837B894FEA07
:100B200053037B837B894FEA53039BB203F1010399
:100B30003B834FF00003FB83E5E0FA8BBB8B9A42CB
:100B400080F08880FB8B4FEAC303FA68D3181B68D8
:100B50007B61FB8B4FEAC303FA68D318BA8B4FEA69
:100B6000C202F9688A1812681A60BB8B4FEAC30385
:100B7000FA68D3187A691A60FB8B4FEAC30303F152
:100B80000403FA68D3181B687B61FB8B4FEAC3032D
:100B900003F10403FA68D318BA8B4FEAC20202F1D8
:100BA0000402F9688A1812681A60BB8B4FEAC30303
:100BB00003F10403FA68D3187A691A60FA8B3B8B45
:100BC000D3184FEAC303FA68D3181B687B61FA8B0A
:100BD0003B8BD3184FEAC303FA68D318B98B3A8B0F
:100BE0008A184FEAC202F9688A1812681A60BA8B2A
:100BF0003B8BD3184FEAC303FA68D3187A691A609B
:100C0000FA8B3B8BD3184FEAC30303F10403FA6852
:100C1000D3181B687B61FA8B3B8BD3184FEAC30355
:100C200003F10403FA68D318B98B3A8B8A184FEA98
:100C3000C20202F10402F9688A1812681A60BA8BBB
:100C40003B8BD3184FEAC30303F10403FA68D318AC
:100C50007A691A60FB8B03F101034FEAC303FA6858
:100C6000D3181B687B61FB8B03F101034FEAC303BD
:100C7000FA68D318B98B7A8B8A184FEAC202F968DE
:100C80008A1812681A60BA8B7B8BD3184FEAC30399
:100C9000FA68D3187A691A60FB8B03F101034FEAF3
:100CA000C30303F10403FA68D3181B687B61FB8B51
:100CB00003F101034FEAC30303F10403FA68D318F5
:100CC000B98B7A8B8A184FEAC20202F10402F968E2
:100CD0008A1812681A60BA8B7B8BD3184FEAC30349
:100CE00003F10403FA68D3187A691A607B681B88D9
:100CF000BB833B894FEA43037A68D3187B60FB8B45
:100D000003F10203FB83FA8B7B8BA3F102039A426C
:100D10007FF613AF07F12407BD4680BC704700BFC4
:100D200080B582B000AF87ED010A3860D7ED017A57
:100D3000F5EEC07AF1EE10FAD4BF00230123DBB246
:100D4000002B0BD097ED010A00F07EF9F0EE407A0F
:100D50003B68C3ED007A4FF0000304E03B68054AAE
:100D60001A604FF0FF035BB2184607F10807BD4653
:100D700080BD00BF0000000080B588B000AFF86003
:100D8000B9607A607B684FEA9303FB619BE0FB6884
:100D90001B68BB61FB6803F10403FB60FB681B6815
:100DA0007B61FB6803F10403FB6097ED067AD7EDE6
:100DB000067A27EE277AD7ED056AD7ED057A66EE33
:100DC000A77A77EE277ABB68BA6802F10402BA60A4
:100DD000B0EE670A1846FFF7A3FFFB681B68BB610C
:100DE000FB6803F10403FB60FB681B687B61FB6825
:100DF00003F10403FB6097ED067AD7ED067A27EE40
:100E0000277AD7ED056AD7ED057A66EEA77A77EEF1
:100E1000277ABB68BA6802F10402BA60B0EE670ACA
:100E20001846FFF77DFFFB681B68BB61FB6803F199
:100E30000403FB60FB681B687B61FB6803F1040330
:100E4000FB6097ED067AD7ED067A27EE277AD7ED85
:100E5000056AD7ED057A66EEA77A77EE277ABB6842
:100E6000BA6802F10402BA60B0EE670A1846FFF7EA
:100E700057FFFB681B68BB61FB6803F10403FB6061
:100E8000FB681B687B61FB6803F10403FB6097ED63
:100E9000067AD7ED067A27EE277AD7ED056AD7EDE1
:100EA000057A66EEA77A77EE277ABB68BA6802F110
:100EB0000402BA60B0EE670A1846FFF731FFFB691B
:100EC00003F1FF33FB61FB69002B7FF460AF7B68AC
:100ED00003F00303FB6129E0FB681B68BB61FB684F
:100EE00003F10403FB60FB681B687B61FB6803F193
:100EF0000403FB6097ED067AD7ED067A27EE277A92
:100F0000D7ED056AD7ED057A66EEA77A77EE277AF0
:100F1000BB68BA6802F10402BA60B0EE670A18460C
:100F2000FFF7FEFEFB6903F1FF33FB61FB69002B5A
:100F3000D2D107F12007BD4680BD00BFD0B52DED51
:100F4000048BB0EE408AF0EE608A3C4C8AB000F030
:100F5000D7F894F90030B0EE409AF0EE609A013381
:100F600035D0B0EE480AF0EE680A00F02BFB0028FE
:100F70002DD051EC180B0022002300F0DBFF30BB1A
:100F80002F4B24780193002308938DED028B8DED78
:100F9000048B002C23D000270026CFF6F07751ECED
:100FA000180B00220023CDE9066700F09BFF002804
:100FB00025D002239C42009336D0684600F03AFBCD
:100FC000002831D0089B002B27D19DED069BB0EE69
:100FD000490AF0EE690A0AB0BDEC048BD0BD4FF6A9
:100FE000FF774FF06046CCF2EF7751EC180B002200
:100FF0000023CDE9066700F075FF0028D9D1012351
:10100000022C009315D0684600F014FB88B10D48FF
:1010100000F012FB8DED060BD4E701F005FB089BF9
:101020009DED069B0360D2E701F0FEFA22230360E8
:10103000C8E701F0F9FA21230360E8E7580000202F
:10104000B4360208F436020810B52DED028B294C97
:101050008AB0B0EE408A00F067FA94F900300133AC
:10106000F0EE408A2FD0B0EE480A00F0EDFA50B30F
:10107000B5EEC08AF1EE10FA25D5012300931E4B80
:1010800018EE100A01930023089300F06FFC2478F7
:10109000CDE90401CDE90201DCB1002000210246C6
:1010A0000B4600F0E1FD022CCDE9060117D101F05D
:1010B000BBFA21230360089BBBB9DDE9060100F000
:1010C0006BFF08EE900AB0EE680A0AB0BDEC028B26
:1010D00010BD0022002343EC172B8DED067B6846E4
:1010E00000F0A8FA0028E6D1E1E701F09DFA089B9C
:1010F0000360E2E758000020B83602080000000054
:101100002DE9F04F53EC102BB3F5801F87B0194633
:1011100067DA23F00043134300F00B81002951EC00
:10112000100BC0F2948100230022C4F2503300F06F
:1011300071FC4FF6FF720B46C7F6EF72934241EC1B
:10114000100B6FF0350753DC23F07F4445F66476CF
:1011500024F47004C0F20906A61906F4801686F07D
:101160007E521D1582F4E002002351EC100BC3F6F1
:10117000F07342EA0401002200F098FAA5F57E75AA
:10118000A31C073D23F47003ED190022022B05EB8D
:10119000165582468B4636DC002300F0A3FE00285D
:1011A00000F0D280002D00F05D81284600F0CCFBDD
:1011B000C9A3D3E9002304460D4600F02BFCC8A3C5
:1011C000D3E9002306460F462046294600F022FCBC
:1011D00002460B463046394600F06AFA41EC100BE5
:1011E0000EE04FF6FF72C7F6EF7200279342ABDDB9
:1011F00051EC100B02460B4600F05AFA41EC100B72
:1012000007B0BDE8F08F4FF0804300F051FA02467E
:101210000B465046594600F027FDCDE9000128460F
:1012200000F092FBCDE90201DDE9000102460B4628
:1012300000F0F0FB02460B468046894600F0EAFBD0
:10124000A9A3D3E9002306460F4600F0E3FBA8A3B9
:10125000D3E9002300F02CFA32463B4600F0DAFBDB
:10126000A5A3D3E9002300F023FA32463B4600F061
:10127000D1FBA3A3D3E9002300F01AFA42464B4660
:1012800000F0C8FBA0A3D3E900238046894630467E
:10129000394600F0BFFB9EA3D3E9002300F008FA13
:1012A00032463B4600F0B6FB9BA3D3E9002300F097
:1012B000FFF932463B4600F0ADFB02460B46404686
:1012C000494600F0F5F94EF686334BF65102CFF65B
:1012D000F973C0F20602E318121B1343002B0646F3
:1012E0000F465BDD00230022C3F6E07350465946EB
:1012F00000F090FB52465B4600F08CFB804689462E
:10130000002D6FD132463B4600F0D2F9DDE90023D3
:1013100000F080FB02460B464046494600F0C6F905
:1013200002460B465046594600F0C0F941EC100BFE
:1013300066E700210020CCF250310022002300F0AB
:1013400093FC41EC100B5BE752465B465046594616
:1013500000F060FB72A3D3E9002306460F46504617
:10136000594600F057FB0B4600210246C3F6E071D8
:10137000002000F09BF902460B463046394600F04B
:1013800049FB06460F46002D6FD15046594632465E
:101390003B4600F08BF941EC100B31E7002D00F0DB
:1013A0008A804DA3D3E90023DDE9020100F032FB7E
:1013B00032463B46804689465046594600F076F90B
:1013C000DDE9002300F026FB45A3D3E90023044612
:1013D0000D46DDE9020100F01DFB02460B462046EA
:1013E000294659E03CA3D3E90023DDE9020100F0DE
:1013F00011FB3246CDE904013B464046494600F028
:1014000057F9DDE9002300F005FB35A3D3E90023FC
:1014100004460D46DDE9020100F0FCFA02460B46E7
:101420002046294600F044F902460B46404649460C
:1014300000F03CF952465B4600F038F902460B4694
:10144000DDE9040100F032F941EC100BD8E6024668
:101450000B4600F02BF90022002300F005FC41ECC4
:10146000100BCDE69FED1A0BCAE6284600F06CFA89
:1014700019A3D3E9002304460D4600F0CBFA18A3C4
:10148000D3E90023804689462046294600F0C2FA67
:1014900002460B463046394600F008F952465B4694
:1014A00000F004F902460B464046494600F0FEF8BB
:1014B00041EC100BA4E632463B465046594600F03C
:1014C000F5F8DDE9002300F0A5FA29E7AFF3008085
:1014D00000000000000000000000E0FE422EE63F99
:1014E000763C7935EF39EA3D44523EDF12F1C23F96
:1014F000DE03CB966446C73F599322942449D23FDA
:10150000935555555555E53F9FC678D0099AC33F29
:10151000AF788E1DC571CC3F04FA97999999D93F40
:10152000555555555555D53F10EE103A23F000420C
:10153000B2F1FF4F70B42FD262B3002B3ADBD91552
:10154000B2F5000F2BD323F07F43A1F17F0223F4E8
:101550000003D10743F4000348BF5B000025561089
:101560005B0019212C464FF08072A018984202DCD3
:1015700084181B1AAD185B0052080139F5D113B15C
:1015800005F001035D196D1005F17C5505EBC6559D
:1015900000EE105A70BC704700EE000AFAE713F430
:1015A00000020CD15B0001321802FBD5C2F101022E
:1015B0008918C8E730EE400A80EE000AEAE7012207
:1015C0008918C0E753EC102B10461A4663B1B3F1EB
:1015D000004F09D04FF6FF73A2F58011C7F6DF73F5
:1015E000994205D8042070470028F3D102207047A3
:1015F00002F1FE4101F570019942F3D94FF6FF73F4
:10160000C0F20F039A4201D80320704702F1004153
:101610009942F9D90023C7F6F0739A4204D012F523
:10162000801F01D000207047D0F1010038BF00209A
:10163000704700BF002070479FED010B704700BF4F
:10164000000000000000F87F10EE103A0BB90220F5
:101650007047B3F1004FFAD0A3F500016FF00142DB
:10166000914201D80420704703F1FF419142F9D91A
:101670004FF6FE72591EC0F27F02914201D803203C
:10168000704703F1004101399142F8D9B3F1FF4F9E
:1016900005D013F5000F14BF002001207047012072
:1016A000704700BF81F0004102E000BF83F00043BB
:1016B00030B54FEA41044FEA430594EA050F08BFED
:1016C00090EA020F1FBF54EA000C55EA020C7FEAB1
:1016D000645C7FEA655C00F0E2804FEA5454D4EB2E
:1016E0005555B8BF6D420CDD2C4480EA020281EAF8
:1016F000030382EA000083EA010180EA020281EA30
:101700000303362D88BF30BD11F0004F4FEA013181
:101710004FF4801C4CEA113102D0404261EB410190
:1017200013F0004F4FEA03334CEA133302D0524216
:1017300063EB430394EA050F00F0A780A4F10104D2
:10174000D5F1200E0DDB02FA0EFC22FA05F280180C
:1017500041F1000103FA0EF2801843FA05F35941F2
:101760000EE0A5F120050EF1200E012A03FA0EFC71
:1017700028BF4CF0020C43FA05F3C01851EBE3719B
:1017800001F0004507D54FF0000EDCF1000C7EEBB8
:1017900000006EEB0101B1F5801F1BD3B1F5001FF6
:1017A0000CD349085FEA30004FEA3C0C04F1010415
:1017B0004FEA445212F5800F80F09A80BCF1004F3E
:1017C00008BF5FEA500C50F1000041EB045141EAC0
:1017D000050130BD5FEA4C0C404141EB010111F4C1
:1017E000801FA4F10104E9D191F0000F04BF01466C
:1017F0000020B1FA81F308BF2033A3F10B03B3F14A
:1018000020020CDA0C3208DD02F1140CC2F10C02D9
:1018100001FA0CF021FA02F10CE002F11402D8BF37
:10182000C2F1200C01FA02F120FA0CFCDCBF41EA03
:101830000C019040E41AA2BF01EB0451294330BDD2
:101840006FEA04041F3C1CDA0C340EDC04F11404AF
:10185000C4F1200220FA04F001FA02F340EA030086
:1018600021FA04F345EA030130BDC4F10C04C4F1CC
:10187000200220FA02F001FA04F340EA03002946AC
:1018800030BD21FA04F0294630BD94F0000F83F4F6
:10189000801306BF81F480110134013D4EE77FEAD9
:1018A000645C18BF7FEA655C29D094EA050F08BF25
:1018B00090EA020F05D054EA000C04BF1946104606
:1018C00030BD91EA030F1EBF0021002030BD5FEA4A
:1018D000545C05D14000494128BF41F0004130BD72
:1018E00014F580043CBF01F5801130BD01F00045C6
:1018F00045F0FE4141F470014FF0000030BD7FEA39
:10190000645C1ABF194610467FEA655C1CBF0B4633
:10191000024650EA013406BF52EA033591EA030F4A
:1019200041F4002130BD00BF90F0000F04BF002142
:10193000704730B54FF4806404F132044FF0000575
:101940004FF0000150E700BF90F0000F04BF0021EE
:10195000704730B54FF4806404F1320410F0004554
:1019600048BF40424FF000013EE700BF42004FEA4F
:10197000E2014FEA31014FEA02701FBF12F07F43CC
:1019800093F07F4F81F06051704792F0000F14BFC9
:1019900093F07F4F704730B54FF4607401F000450D
:1019A00021F0004120E700BF50EA010208BF704764
:1019B00030B54FF000050AE050EA010208BF704759
:1019C00030B511F0004502D5404261EB41014FF4C2
:1019D000806404F132045FEA915C3FF4DCAE4FF0C6
:1019E00003025FEADC0C18BF03325FEADC0C18BFAD
:1019F000033202EBDC02C2F1200300FA03FC20FAFE
:101A000002F001FA03FE40EA0E0021FA02F114444A
:101A1000C1E600BF70B54FF0FF0C4CF4E06C1CEA5F
:101A200011541DBF1CEA135594EA0C0F95EA0C0FD4
:101A300000F0DEF82C4481EA030621EA4C5123EA47
:101A40004C5350EA013518BF52EA033541F4801176
:101A500043F4801338D0A0FB02CE4FF00005E1FB29
:101A600002E506F00042E0FB03E54FF00006E1FB73
:101A700003569CF0000F18BF4EF0010EA4F1FF04B6
:101A8000B6F5007F64F5407404D25FEA4E0E6D41F6
:101A900046EB060642EAC62141EA55514FEAC52007
:101AA00040EA5E504FEACE2EB4F1FD0C88BFBCF583
:101AB000E06F1ED8BEF1004F08BF5FEA500E50F134
:101AC000000041EB045170BD06F0004646EA0101FA
:101AD00040EA020081EA0301B4EB5C04C2BFD4EB2C
:101AE0000C0541EA045170BD41F480114FF0000E25
:101AF000013C00F3AB8014F1360FDEBF002001F093
:101B0000004170BDC4F10004203C35DA0C341BDC0C
:101B100004F11404C4F1200500FA05F320FA04F0DE
:101B200001FA05F240EA020001F0004221F0004112
:101B300010EBD37021FA04F642EB06015EEA430E85
:101B400008BF20EAD37070BDC4F10C04C4F12005B5
:101B500000FA04F320FA05F001FA04F240EA020068
:101B600001F0004110EBD37041F100015EEA430E39
:101B700008BF20EAD37070BDC4F1200500FA05F259
:101B80004EEA020E20FA04F301FA05F243EA0203D8
:101B900021FA04F001F0004121FA04F220EA0200E7
:101BA00000EBD3705EEA430E08BF20EAD37070BD2D
:101BB00094F0000F0FD101F00046400041EB01010D
:101BC00011F4801F08BF013CF7D041EA060195F0EF
:101BD000000F18BF704703F00046520043EB0303A9
:101BE00013F4801F08BF013DF7D043EA0603704796
:101BF00094EA0C0F0CEA135518BF95EA0C0F0CD0A1
